:10000000D804002035E900002DE900002FE90000A8
:1000100031E9000031E9000031E900000000000092
:1000200000000000000000000000000031E90000B6
:1000300031E900000000000031E9000031E9000072
:1000400031E9000031E9000031E9000031E9000048
:1000500031E9000031E9000031E9000031E9000038
:1000600031E9000031E9000031E9000031E9000028
:1000700031E9000031E9000031E9000031E9000018
:1000800031E9000031E9000031E9000031E9000008
:1000900031E9000031E9000031E9000031E90000F8
:1000A00031E9000031E9000031E9000031E90000E8
:1000B00031E9000031E9000031E9000031E90000D8
:1000C00031E9000031E9000031E9000031E90000C8
:1000D00031E9000031E9000031E9000031E90000B8
:1000E00031E9000031E9000031E9000031E90000A8
:1000F000FF230370FF3B8370643343707047FF231B
:100100000370F53B83705A334370643BC370704790
:1001100038B50025044645700430FFF7F0FF04F1C0
:100120000800FFF7E5FFFF23642223702373627347
:10013000A373E27323746274A374E274072395FBC0
:10014000F3F3643BC835237563750434B5F5C86FA4
:10015000F4D138BD13B504460C490FF029F82046F8
:100160000FF084F80A4B201819784A1C1A700123E2
:1001700000220093134600F0B9FD0023238263821E
:10018000A382A375E3750023A3611CBD8C06010047
:10019000E102002013B5044611490FF009F820468A
:1001A0000FF064F80F4B201819784A1C1A700022BF
:1001B00001230093134600F099FD002204F11C0076
:1001C0002282A274E27422756275A275E2752276AB
:1001D0006276A276E27602B0BDE81040FFF788BFF3
:1001E00098060100E402002000230370437083702E
:1001F000C370704738B50025FF230446437005706F
:100200008570C5700430FFF77AFF04F10800FFF72E
:100210006FFF04F10C00FFF76BFF2582658238BD8C
:10022000FF2310B50370FF3B044643708370C37017
:100230000430FFF764FF04F10800BDE81040FFF749
:1002400057BFFF2310B50370FF3B04464370837014
:10025000C3700430FFF753FF04F10800BDE81040FD
:10026000FFF746BFFF2310B50370FF3B0446437002
:100270008370C3700430FFF742FF04F10800FFF7FA
:1002800037FF04F10C00BDE81040FFF731BFFF233A
:1002900010B50370FF3B044643708370C370043095
:1002A000FFF72DFF04F10800FFF722FF04F10C0017
:1002B000BDE81040FFF71CBF13B504460D490EF012
:1002C00077FF20460EF0D2FF0B4B201819784A1CFE
:1002D0001A70012300220093134600F007FD00234B
:1002E00004F114002382A374E37402B0BDE810404B
:1002F000FFF7FEBE9F060100E2020020002303700C
:1003000043708370C3708380C3800381438100F195
:1003100020030022828102309842FAD170470023E4
:1003200043708370C370C21802330021202B918068
:10033000F9D170470023037043708370C370704716
:1003400038B50446FFF7F6FF201DFFF7F3FF04F171
:1003500008000025FFF7EEFF04F10C00FFF7EAFFAD
:1003600025746574A574E57425756575A575E575C1
:1003700004F11800FFF7BCFE25776577A577E577D0
:100380002584658484F8245084F8255084F8265008
:1003900084F8275038BD00002DE9F34100240646BB
:1003A00046F8044B05463A4930460EF001FF304608
:1003B0000EF05CFF374E2818317801274B1C22467F
:1003C000337005F1140823460430009700F08EFCCA
:1003D0002F4940460EF0ECFE40460EF047FF3178C4
:1003E0002818CB192246337005F12408234614300F
:1003F000009700F07BFC264940460EF0D9FE4046AF
:100400000EF034FF31782818CB192246337005F1ED
:10041000340823462430009700F068FC1C4940460D
:100420000EF0C6FE40460EF021FF31782818CB1999
:100430002246337005F1440823463430009700F01B
:1004400055FC134940460EF0B3FE40460EF00EFF39
:1004500031782818CB192246337005F5A278234647
:100460004430009700F042FC094940460EF0A0FEDF
:1004700040460EF0FBFE31782818CB193370224627
:10048000234600F5A270009700F030FCBDE8FC8127
:10049000A7060100E302002000230380438083803D
:1004A000C380704738B50546002405EBC40001340D
:1004B000FFF7F2FF042CF8D138BD00234370C3705E
:1004C0004371C371704770B500250446056005711E
:1004D00045718571C571A81C04EB80000135FFF7DB
:1004E00083FE102DF7D1103D0C2000FB0540013597
:1004F0004830FFF795FE102DF6D1103D0C2000FB83
:100500000540013500F58470FFF79BFE102DF5D1F5
:10051000103D142000FB0540013500F5E470FFF7A5
:1005200069FE102DF5D1103D342000FB054001354A
:1005300000F54270FFF7ECFD402DF5D1403D28015C
:1005400000F58050083020180135FFF78BFE102D84
:10055000F5D1103D280100F58850083020180135EC
:10056000FFF795FE102DF5D104F5905505F1080023
:10057000FFF7C4FE05F13400FFF7C0FE04F5935009
:1005800004F59454FFF7CBFE201DFFF7C8FE04F1DD
:100590002800BDE87040FFF790BF00230370437050
:1005A0008370C370704710B50446FFF7A8FD0022A2
:1005B000A280E28022726272A272E27210BD0022F8
:1005C00002608280C280027242728272C2720C30F9
:1005D000FFF795BDF7B5044631490EF0E9FD204619
:1005E0000EF044FE2F4D0022297801264B1C2B7063
:1005F00004F1180713462018009600F077FB2849ED
:1006000038460EF0D5FD38460EF030FE297800222F
:100610008B1918302B70201800251346009600F017
:1006200065FB84F8285084F8295084F82A5084F80F
:100630002B50680120182C300135FFF7ABFD402D01
:10064000F7D1403D182000FB054000F502600C305A
:100650000135FFF731FE402DF4D1403D1C2000FB59
:10066000054000F562600C300135FFF773FD202D69
:10067000F4D104F58C502C3004F51054FFF723FF0F
:1006800004F15C00FFF79BFF04F16C00FFF797FF9C
:1006900004F17C0003B0BDE8F040FFF784BF00BF69
:1006A000B0060100E002002010B50446FFF7FAFE94
:1006B00004F12000FFF744FE04F14800BDE81040BB
:1006C000FFF76ABE0D4A002310B513700C4A0446AA
:1006D00013700C4A04F5125413700B4A13700B4A32
:1006E0001370FFF777FF04F10800FFF756FF04F1DE
:1006F0000C00BDE81040FFF7D7BF00BFE1020020AB
:10070000E4020020E2020020E3020020E0020020D8
:100710002DE9F04193F900406425E602361B96FB73
:10072000F5F6541EB04213F8244001DC30B207E065
:1007300064B2E602341B94FBF5F4A042A8BF20B2D9
:1007400000262AE093F90040E5022D1B642495FB66
:10075000F4F5A8421FDB93F9047003F1040C4FEA8F
:10076000C728C7EB080797FBF4F7B84213DC93F9E7
:100770000130401BDA02D31A9CF9012093FBF4F3F9
:10078000D602B21A92FBF4F4E41A60437F1B90FB8A
:10079000F7F5ED1805E001360433541EA642D1DB0F
:1007A00000256943642391FBF3F000B2BDE8F081BA
:1007B0000378FF2B1AD0FE2B1AD0FD2B01D14078E5
:1007C00017E03F2B05D80C4A5B019B189A7952B26F
:1007D00000E0002290F9023090F901006432C01A62
:1007E0005043C82190FBF1F0C01802E0002000E067
:1007F000642040B2704700BF080D00200278034615
:10080000FF2A17D0FE2A13D03F2A13D80E495201CF
:100810005218917990F9020049B288420ADC907925
:1008200093F9012040B28242B4BF0020012002E0CF
:10083000012000E0002093F90330012B04BFC0F138
:100840000100C0B2704700BF080D002010B5174866
:1008500000F0A2FA154800F59A51083100F090FC1A
:10086000124800F58E51083100F0D6FB0F4800F514
:100870009451083100F064FC0C4800F5A452083291
:1008800000F5006100F008FD094800F5CC51083181
:1008900000F0A8FD064800F5D451083100F0D4FD61
:1008A0000348BDE8104000F005BE00BFFC0C00206E
:1008B000FC14002010B500230D4A342101FB032253
:1008C000FE2402F5A452FD2182F8343082F838402B
:1008D00082F83C10FD3982F83E10643182F83D10F8
:1008E00082F840300133402B82F84110E4D110BD32
:1008F000D00C002070B59F499F480EF059FC9F49CD
:100900009F480EF055FC9F499F480EF051FC9F49AF
:100910009F480EF04DFC9F499F480EF049FC9F4BAD
:1009200042F2B962DA62012003F594534FF49672F1
:1009300083F865003C21A3F860204FF41675FF2270
:100940004FF49676A3F8625083F8641083F8682019
:1009500083F87500A3F870600138A3F8725083F82B
:10096000741083F878201946834B142202FB00325E
:10097000FE2502F59A52013082F838500024642690
:10098000013D102882F83E4082F83D6082F83C50DC
:1009900082F8424082F8416082F84050E4D1224619
:1009A0000C2404FB0234FE2504F58E5484F83850E0
:1009B0000020D13D013284F83E0084F83D50D0350E
:1009C000102A84F83C50EBD10C2404FB0034FE25A3
:1009D00004F5945484F838500022B33D013084F873
:1009E0003E2084F83D50B235102884F83C50EBD1BD
:1009F000342000FB0230FE2500F5A45080F838506A
:100A000000249A3D013280F83E4080F83D509935EF
:100A1000402A80F83C50EBD104F506720332FE20E8
:100A200003EB0212107204F58072013203EB021222
:100A3000013402F58C52FE386426FD25102C82F814
:100A40002E0082F82D6082F82C5082F8320082F855
:100A5000316082F83050DFD100F50A720332FE2493
:100A600003EB0212147200F58872013203EB0212DA
:100A7000013002F58C52FE3C6426FD25102882F8D8
:100A80002E4082F82D6082F82C5082F8324082F895
:100A9000316082F83050DFD122462C2505FB02352B
:100AA000082405F50E5585F834400126083C85F8E4
:100AB000354085F836604FF496762E8740F2DC5646
:100AC000AE874FF47A7605F13000EE8742F6E065A6
:100AD00045812046162404FB020404F58E541C3480
:100AE0000130002603EB440410282681F2D10132A4
:100AF000022AD2D1023A242000FB0230082400F559
:100B00001050C473F7344473FF3C8473204612249E
:100B100004FB020404F5905404340130002503EB77
:100B2000440410282581F2D10132022AE3D10024A5
:100B3000182000FB043001340022FD25402C80F8F1
:100B4000422880F8412880F84058F1D15001181807
:100B5000383001240472941C640100251C1945726C
:100B6000A5726572FD35257254B2032C18DC26245B
:100B700017E000BF40070100D00C00205107010022
:100B8000A831002056070100B8310020EE290100ED
:100B9000E83100205B070100E80C0020501E002017
:100BA00027240132402AC471D0D12B3A83F83F2048
:100BB000013283F85F20013283F87F20013283F80D
:100BC0009F20FD20183A83F84A2083F8492083F8B3
:100BD000480083F86A2083F8692083F8680083F866
:100BE0008A2083F8892083F8880083F8AA2083F874
:100BF000A92083F8A8002F3881F8550081F8570004
:100C000081F859009C3881F85B00313881F8542014
:100C100081F85600013081F85800013081F85A00FF
:100C2000911C4901002559188D7151010132591843
:100C3000402A81F83E508D87F2D12A4CFFF73AFEC8
:100C40000123237284F8533084F85130033384F83D
:100C50005230FB3384F82C5084F8345084F82D50F3
:100C600084F8355084F82E5084F8365084F83830A3
:100C700084F8393084F83A3084F8303084F83130F0
:100C800084F83230F73B84F83C301A3384F84B3028
:100C90003226183B84F8493004F1880084F84A5021
:100CA000114984F8483084F850600EF081FA8023AE
:100CB00026226020A4F84C30A4F84E0084F840604E
:100CC00084F842203E3284F8415084F8465084F83B
:100CD0004520993284F8442084F83D3084F83E5011
:100CE00070BD00BF5031002063070100F0B500293E
:100CF00085B005DA2D244942047009B22C3C00E08D
:100D0000002400250BE04FF00A0C91FBFCF70CFBD4
:100D100017110135303106F80C1CEDB239B204AFB1
:100D2000092907EB0506EEDC303106F80C1C691CBE
:100D300003E0302605F80C6C0131C9B204AE9942CB
:100D400006EB0105F5D99142F3D3002205F80C2CEE
:100D50000A460DE09A4203D12E2101550134E4B236
:100D600004AFB91811F80D1C013A01550134E4B271
:100D7000002AEFD1025505B0F0BD000010B50024E7
:100D8000E0B20DF041FA034B23F814000134202C9B
:100D9000F6D110BDD8040020F0B5002585B004467A
:100DA0002F4694F91530EEB2042B24D1043B237561
:100DB000A37D013BDBB2632B01D90123A375E17D48
:100DC000A37DA27C51B958B251B24118632901DC0C
:100DD0009B183DE06423A374633B0AE050B259B210
:100DE000411A11F1630F01DBD31A31E09C23A37484
:100DF0009C3BE37563E094F914208AB9022B5ED121
:100E000094F91630002B5ED1A37C5AB2632A04DC1D
:100E1000142701335743A37455E00123A37552E00F
:100E2000754A012B32F815703FB213D117F5027FC6
:100E300001DA9B330CE0B7F5027F01DD642307E0A4
:100E400007F5F877033740F2E6339F4237D800239F
:100E5000A37434E0022B14D117F1640F05DAA37CDC
:100E60005AB212F1630F2ADB05E0642F27DDA37C61
:100E70005AB2632A23DC4FF4FA7297FBF2F7FB189D
:100E8000E6E7032B1FD1642F07DD94F916308BB9E9
:100E900094F912205AB9643309E017F1640F09DAA2
:100EA00094F9163033B994F9122002B99C33A37423
:100EB000012303E06337C62F01D80023A37594F9FB
:100EC000123014275F43032E1DD84C4A05F5926358
:100ED000013302EBC303DA8812B2BF1A002F07DD19
:100EE0001A8912B2002A0EDDFA02D71B1B8907E00D
:100EF00009D09A8812B2002A05DA414A9B885743E2
:100F00001BB297FBF3F7237F3F2B03D9FE2B01D0B6
:100F1000FD2B24D104F11C00FFF74AFC94F91B308F
:100F2000012B15D19B338DF804308DF805309C3B97
:100F300064218DF808308DF80900032238B201AB26
:100F40008DF80C108DF80D10FFF7E2FB074606E058
:100F5000C302181A642390FBF3F000B23F1894F90F
:100F60001A30012B264B08BF7F429F42B8BF1F4655
:100F700040F2FF739F42A8BF1F46224B33F8152053
:100F800012B297421DD0032E0BD91F4A16701F4A6A
:100F90001278A2B194F91520042A10D01C4A1670B8
:100FA0000DE033F81500282200B297FBF2F190FB18
:100FB000F2F2914203D0144A1670144A127823F8C0
:100FC000157094F9143027827BB194F9153063B908
:100FD000143397FBF3F31BB2642BA8BF64236FF0A9
:100FE00063029342B8BF1346A37401352034402DE9
:100FF0007FF4D7AE05B0F0BDD8040020D00C00209F
:1010000001F8FFFFE6020020E2010020A1310020EC
:10101000E3010020000000002DE9F3470D46002405
:101020002B5D2E193F2B76D8301DFFF7E7FB0128EB
:1010300071D106F10800FFF7BBFB824600286AD099
:101040002E5D394F7301FB18988F00B20FF0DEF858
:1010500036490FF0E3F94FF07E5180460FF0E6FA83
:1010600028B9404632490FF0C3FA18B904E04FF0EE
:101070007E5801E0DFF8B8802B195B78013BDBB2CA
:10108000012B06D840460EF081FCCDE90001404618
:1010900008E040460EF07AFCCDE9000140464146AA
:1010A0000FF008F941460FF005F9014640460EF0F1
:1010B000F7FF0EF06BFC8046504689460FF0A6F80D
:1010C0000EF064FC00221B4B0EF0DEFD02460B46C8
:1010D000404649460EF0AEFC02460B46DDE90001F3
:1010E0000EF0F4FA0EA3D3E900230EF0A3FC0EF0E9
:1010F0003BFF73017601FB18BF1998873837BA8810
:1011000040F2FF7312B29A4204DCBA880A4B12B260
:101110009A4200DABB800C34C02C81D1BDE8FC8738
:101120000000000000FC9F40D00C002000E0FF44C5
:10113000000080BF0000594001F8FFFFAFF30080BE
:10114000F8B504460E460025735D77193F2B12D87B
:10115000381DFFF753FB01280DD107F10800FFF7F9
:1011600027FB735D64215B01E318B3F91020424350
:1011700092FBF1F21A820C35C02DE5D1F8BD0000CA
:101180002DE9F843044688460D46002708EB07067C
:1011900073783F2B76D8281DFFF730FB01286CD1E0
:1011A00005F10800FFF704FB814605F10C00FFF78D
:1011B000FFFA18F80720737892B95B01E318B3F9C6
:1011C00010202B8A19B209EB010C624503DD99440A
:1011D000A5F810904BE0091A8A4248DA1B1A45E03C
:1011E0005B01E318B3F91030142B10DD03FB09F396
:1011F00040F2FF7293FBF2F3B2785BB2002A28D080
:10120000698A08B21018984224DA521810E013F1D3
:10121000140F11DA43431F4A93FBF2F3B2785BB227
:1012200042B1698A5B4208B2801A984212DD8A1A7A
:101230006A820FE05B420CE0B37853B16A8A11B264
:10124000C81A002801DDD31A03E0CB424CBF9B181B
:1012500000236B822B8A6A8AD2180E4B2A8212B222
:101260009A4203DB40F2FF739A4200DD2B827378CF
:101270002A8A5B01E3181A8204E073785B01E318A1
:101280001B8A2B8214371435B7F5A07F7FF47EAF0D
:10129000BDE8F88301F8FFFF2DE9F84F16468146B7
:1012A0000F460B4601F5C0620021198218339342A4
:1012B000FAD134460025735D3F2B00F28B80201D50
:1012C000FFF79CFA012840F0858004F10800FFF741
:1012D0006FFA237B80463F2B1CD894F90D20CAB1AE
:1012E0004FF0180A0AFB037A735D08225B014B4436
:1012F000B3F91000414604F11403BAF810B0FFF737
:1013000007FA94F90D306422434393FBF2F39B44B4
:10131000AAF810B0A37B3F2B1CD894F90F20CAB1B8
:101320004FF0180A0AFB037A735D08225B014B44F5
:10133000B3F91000414604F11403BAF810B0FFF7F6
:10134000E7F994F90F306422434393FBF2F39B4493
:10135000AAF810B0237C3F2B1CD894F91120CAB1F5
:101360004FF0180A0AFB037A735D08225B014B44B5
:10137000B3F91000414604F11403BAF810B0FFF7B6
:10138000C7F994F911306422434393FBF2F39B4471
:10139000AAF810B0A37C3F2B1CD894F91320CAB133
:1013A0004FF0180A0AFB037A735D08225B014B4475
:1013B000B3F91000414604F11403BAF810B0FFF776
:1013C000A7F994F913306422434393FBF2F39B444F
:1013D000AAF810B034353434B5F5506F7FF46BAFE4
:1013E000BDE8F88F2DE9F04104460E460025735DF7
:1013F00006EB05083F2B21D808F10400FFF7FEF9A2
:1014000001281BD1725D182707FB0242138A19B20B
:10141000002902DD08F1080002E073B108F10C00B8
:10142000FFF7C6F9735D642207FB0347B7F9103075
:10143000434393FBF2F33B8200E013821035B5F592
:10144000807FD4D1BDE8F081F8B504460E46002572
:10145000735D77193F2B28D8381DFFF7CFF9012886
:1014600023D107F10800FFF7A3F9735D182202FBEF
:101470000343C2026421121A92FBF1F2B3F9101075
:1014800007F10C009142C8BF1A82FFF791F9735D12
:10149000182202FB0343C2026421821A92FBF1F27A
:1014A000B3F910109142B8BF1A821035B5F5807F9C
:1014B000CED1F8BD70B5044600F5C066237DB4F901
:1014C00010503F2B03D9FE2B01D0FD2B0AD104F184
:1014D0001400FFF76DF9C3021B1A642293FBF2F3A9
:1014E0001BB2ED1894F91230012B084B08BF6D4266
:1014F0009D42B8BF1D4640F6FE139D42A8BF1D4643
:1015000025821834B442D9D170BD00BF02F6FFFF66
:101510007047000070B5284CB4B0A04205460E4696
:1015200047D3264902A80DF043FE02A80DF09EFE07
:101530000022291B02AB0124181809B2134600949B
:10154000FFF7D4FB1E4902A80DF00EFE02A80DF015
:101550008DFE02AB0022181831B213460094FFF73B
:10156000C5FB013C11E0164902A80DF0FDFD02A8E3
:101570000DF07CFE01230093002202AB295D1818B8
:101580001346FFF7B3FB0134E4B2B442EBD30C498A
:1015900002A80DF0E9FD00200CF070FE02A9002069
:1015A0000CF074FE00200CF093FE002005490CF0B6
:1015B0006DFE002034B070BDD00C0020E0090100A9
:1015C000B81B0100EC29010010B50CF085F90446A8
:1015D0000CF084FB844207D20CF080FB041B04EB6C
:1015E000D4746010C0B210BD002010BD10B50CF056
:1015F000C7F904460CF072FB844207D20CF06EFB74
:10160000041B04EBD4746010C0B210BD002010BDE8
:1016100038B505460CF062FB044628460CF0B0F9DC
:10162000201AC0B238BD08B592F900300BB10023C2
:1016300000E00123137010460121FFF76BFF01202A
:1016400008BD00002DE9F04F8BB014460D460CF09C
:1016500045FB06460CF044FB0027721E431E012189
:10166000D2B2DBB200913846394601970297039710
:101670000BF0F0FF0CF032FB06460CF031FBFF21C3
:10168000721E431E01910291039138463946D2B22F
:10169000DBB200970BF0DEFF20460DF0E7FDA14E18
:1016A000013096F80080804502D8B8F10F0F00D9BC
:1016B0003770FF272046FFF787FF3B46032122466E
:1016C000009701970CF0C2F9974B93F80090984659
:1016D000B9F1000F78D1012D0CD120460DF0C6FDD7
:1016E0003778904D874202D201372F7035E085F868
:1016F000009032E0022D0AD133788A4D13B1013BBC
:101700002B702AE020460DF0B1FD287025E0033D46
:10171000EDB2012D21D835784DB920460DF0A6FD4A
:10172000411C89B22046FFF7F5FE012059E16F1EEA
:10173000E35D2B2B01D1023302E02D2B02D1023BC2
:10174000E3550AE020460DF091FD854203D92023A0
:10175000E35504F8059088F80050357875B973485A
:10176000FFF732FF05460CF0BBFAFF23A0F113018F
:10177000009301932846C9B26C4A12E020460DF04E
:1017800075FD854211D96A48FFF71EFF05460CF02A
:10179000A7FAFF23A0F10B01654A009301932846A5
:1017A000C9B20CF053F9002513E16248FFF70CFFB2
:1017B00005460CF095FAFF23A0F10B01009301936D
:1017C0002846C9B25B4AECE75A48FFF7FDFE81465E
:1017D0000CF086FAA0F10B01C9B24846554A3B46C7
:1017E000009701970CF032F9012D0DD198F80030D7
:1017F000013BE25C2B2A0FD02D2A11D0382A01D8C8
:10180000013214E0302212E0022D12D198F800309B
:10181000013BE25C2B2A01D1023208E02D2A01D1E2
:10182000023A04E0302A01D9013A00E03922E254B8
:10183000B9E7033DEDB2012DB5D898F800305A1E36
:10184000A15C202901D12039A1543370002388F8EC
:101850000030A8E7635D60190022059036488DF8D6
:101860001C308DF81D200CF037F8337800F1020A97
:10187000013B9D425FFA8AFA40F09980635D05FB67
:101880000AF9202B0ED10CF02BFA09F105094108B9
:10189000FF235FFA89F0C9B2284A009301930CF044
:1018A000D5F830E00DF1280B0BF80C3D04900CF04E
:1018B00017FA09F10509FF275FFA89F941085A4625
:1018C000C9B23B464846009701970CF0BFF80CF0B0
:1018D00007FA83460CF004FADDF810C043084FEA1B
:1018E0005B0BA9F102020020ABF10201E1440B33D2
:1018F0000090C9B2D0B2DBB25FFA89F201970297C9
:1019000003970BF0A7FE98F80030002B5FD0059AE4
:1019100013785A1ED2B22B2B8DF81C2010D1023313
:1019200015E000BF9C03002067030020E8090100C8
:10193000ED090100F1090100C60D0100F6090100E1
:101940002D2B01D1023B02E02F2A02D839238DF83A
:101950001C300CF0C5F905FB0AFA41080AF1050A2A
:1019600008395FFA8AFAFF2307AA5046C9B20093E2
:1019700001930CF06BF8059803785A1CD2B22B2B0C
:101980008DF81C2001D1023306E02D2B01D1023B42
:1019900002E0392A02D930238DF81C300CF0A0F96E
:1019A000FF23410808310093019350460BE00CF0EF
:1019B00097F905FB0AFAFF230AF1050A410800938B
:1019C00001935FFA8AF0C9B207AA0CF03FF801351B
:1019D000EDB220460DF04AFC01308542FFF43AAFEB
:1019E00000200BB0BDE8F08F70B5012386B006462D
:1019F0000D461446B2F9001002A800930922013BDB
:101A0000FFF774F9294602AAFF233046FFF71AFEB2
:101A1000054602A80DF046FB02A80DF043FB20602E
:101A2000284606B070BD70B5012386B00D46064647
:101A3000B2F90010144600930522013B03A8FFF7FA
:101A400055F92946FF2303AA3046FFF7FBFD05465B
:101A500003A80DF027FBB0F5803F02DB00232380B5
:101A600003E003A80DF01EFB2080284606B070BDE1
:101A700070B50D46B2F9001086B00029064614462E
:101A80004FF0010304DA009303A80622013B07E0AC
:101A90002B228DF80C2000930DF10D00253A002328
:101AA000FFF724F92946FF2303AA3046FFF7CAFDB2
:101AB000054603A80DF0F6FAB0F5FA4F02DD4FF433
:101AC000FA4307E003A80DF0EDFA10F5FA4F03DA38
:101AD00048F20033238003E003A80DF0E3FA2080EE
:101AE000284606B070BD00002DE9F04F8BB01446BB
:101AF0000D460CF0F3F806460CF0F2F80027721EC3
:101B0000431E0121D2B2DBB200913846394601971B
:101B1000029703970BF09EFD0CF0E0F806460CF0E0
:101B2000DFF8FF21721E431E019102910391384696
:101B30003946D2B2DBB200970BF08CFD20460DF097
:101B400095FB994E013096F80080804502D8B8F197
:101B50000F0F00D93770FF272046FFF735FD3B46B2
:101B600003212246009701970BF070FF8F4B93F8EB
:101B700000809946B8F1000F71D1012D0DD120469A
:101B80000DF074FB377801308742874D02D2013760
:101B90002F702DE085F800802AE0022D0BD13378DC
:101BA000814D13B1013B2B7022E020460DF05EFB0E
:101BB000013028701CE0033DEDB2012D18D83578B6
:101BC0004DB920460DF052FB411C89B22046FFF76B
:101BD000A1FC012052E120460DF048FB854205D9C9
:101BE0006319202203F8012C04F8058089F80050BD
:101BF000357875B96E48FFF7E7FC05460CF070F8CC
:101C0000FF23A0F10B01009301932846C9B2684A53
:101C100012E020460DF02AFB854211D96548FFF7F6
:101C2000D3FC05460CF05CF8FF23A0F10B01614AE0
:101C3000009301932846C9B20BF008FF002515E177
:101C40005D48FFF7C1FC05460CF04AF8FF23A0F100
:101C50000B01009301932846C9B2574AECE7564856
:101C6000FFF7B2FC80460CF03BF8A0F10B01C9B2C3
:101C70004046514A3B46009701970BF0E7FE012D85
:101C800009D199F80030013BE25C7E2A01D801328B
:101C90000CE020220AE0022D0AD199F80030013B25
:101CA000E25C202A01D9013A00E07F22E254C5E734
:101CB000033DEDB2012DC1D899F800305A1EA15C48
:101CC000202901D12039A1543370002389F8003034
:101CD000B4E760190590635D002238488DF81C3028
:101CE0008DF81D200BF0F8FD337800F10208013B60
:101CF0009D425FFA88F840F0A780635D05FB08FA13
:101D0000202B0ED10BF0ECFF0AF1050A4108FF234E
:101D10005FFA8AF0C9B22A4A009301930BF096FE4B
:101D200030E00DF1280B0BF80C3D04900BF0D8FFC0
:101D30000AF1050AFF275FFA8AFA41085A46C9B232
:101D40003B465046009701970BF080FE0BF0C8FF12
:101D500083460BF0C5FFDDF810C043084FEA5B0B6C
:101D6000AAF102020020ABF10201E2440B33009021
:101D7000C9B2D0B2DBB25FFA8AF201970297039739
:101D80000BF068FC99F80030002B6DD005FB08FBC8
:101D9000C8F1000C5FFA8CFC0BF1050BE2465FFA10
:101DA0008BFB0027A44628E0810300208703002046
:101DB000E8090100ED090100F1090100C60D01006B
:101DC000F6090100059A0AAC1378013BDB1B04F805
:101DD0000C3DCDF810C00BF083FF41080BEB08025F
:101DE0001039FF23D0B2C9B22246009301930137C4
:101DF0000BF02CFEDDF810C0FFB2D344AF425FFA07
:101E00008BFBDFD16446002719E005980DF1280A05
:101E100003780133FB180AF80C3D0BF061FF7A19C7
:101E200002FB08F2410805321031FF23D0B2C9B2DB
:101E30005246009301930BF009FE0137FFB2C5F142
:101E40000E039F42E1DB0FE00BF04AFF05FB08F8B1
:101E5000410808F10508FF235FFA88F0C9B207AA14
:101E6000009301930BF0F2FD0135EDB220460DF029
:101E7000FDF901308542FFF42CAF00200BB0BDE826
:101E8000F08F00BF13B50E4B0C4693F848300A2B69
:101E900009D9811CFF230220C9B222460093019375
:101EA0000BF0D4FD0AE0074B22461978FF234118B6
:101EB000C9B20220009301930BF0A8FD1CBD00BF26
:101EC00050310020D1000020F7B5124F054697F899
:101ED00048300C460A2B104E09D90846FFF798FBEC
:101EE000327897F84830D2438018073B07E008461D
:101EF000FFF78EFB3378094FDB43C0183B78ED18B2
:101F0000E9B2FF232246C0B2009301930BF07EFD9D
:101F1000FEBD00BF5031002030000020D100002065
:101F200030B5012387B0144600220546009303A86C
:101F3000134609B2FEF7DAFE284603A92246FFF748
:101F4000C3FF07B030BD000037B50C4605460BF0A7
:101F5000C5FE0C4B013593F848200B4B083A197815
:101F60006FF012035B1A02EBD27205EB6201C0182C
:101F700000230093C9B2E2B20133C0B20BF0AEF954
:101F80003EBD00BF503100203000002030B5054676
:101F900087B01C46002923D1012A06D13F4903A856
:101FA0000DF006F92846242166E0022A02D103A892
:101FB0003B4924E0032A02D103A83A4958E0042A05
:101FC00002D103A8384906E0052A02D103A83749FF
:101FD00015E0374903A80DF0EBF828462B214BE01C
:101FE000012929D1012A06D1324903A80DF0E0F8D0
:101FF0002846252140E0022A04D12F4903A80DF0EC
:10200000D7F844E0032A06D12C4903A80DF0D0F8F4
:102010002846272130E0042A02D103A8284906E0F7
:10202000052A02D103A82749E9E7274903A80DF0AB
:10203000BFF828462A211FE0022908D1032A26D109
:10204000224903A80DF0B4F82846282114E00329FA
:1020500008D1032A1BD11E4903A80DF0A9F8284670
:10206000292109E004290BD1032A10D1194903A819
:102070000DF09EF8284626212246FFF765FF0BE06B
:1020800001230022009303A81346FEF72FFE2846E3
:1020900003A92246FFF718FF07B030BDFC09010075
:1020A000030A01000B0A0100120A0100150A0100CF
:1020B00025100100140F01001D0A01004B12010040
:1020C000220A0100260A01001D1001002D0A01004C
:1020D000340A01003B0A010030B5012387B01446E1
:1020E00000220546009303A8134609B2FEF7FEFD41
:1020F00003A805490DF038F8284603A92246FFF742
:10210000E3FE07B030BD00BF4E0A010013B5064B19
:102110000C46197822464118FF230320C9B20093C8
:1021200001930BF0ADFC1CBDD100002013B5064B94
:102130000C46197822464118FF230320C9B20093A8
:1021400001930BF083FC1CBDD100002070B50E463E
:10215000097888B03F290546144604D8164B490132
:1021600002A8C91805E00331C9B202291FD81349D2
:1021700002A80DF01DF83046FEF71AFB104906467E
:1021800002A80CF0F1FF02A80DF070F80123002264
:10219000009302AB181831B21346FEF7A7FD0949A8
:1021A00002A80CF0E1FF284602A9224600E00649F9
:1021B000FFF78AFE08B070BDFC0C0020400A010049
:1021C000111001004E0A0100470A010070B50D46CA
:1021D000097886B03F290446164613D8104B4901AA
:1021E0006846C9180CF0E4FF2846FEF707FB10B15B
:1021F00068460C4901E00C4968460CF0B5FF2046E2
:10220000694608E02846FEF7F9FA10B1204607496A
:1022100001E0074920463246FFF756FE06B070BD82
:10222000FC0C0020500A0100560A01005D0A010062
:10223000660A0100F0B5054685B01A4E01B3327842
:1022400000F109070024FFB20123C2F12E0200931E
:10225000204629463B46D2B20194029403940BF0E7
:1022600025F93278FF23C2F12E02019302930393E2
:1022700020462946D2B23B4600940BF0EBF90FE022
:10228000327800F10903C2F12E0201200090019181
:10229000029103910846D2B22946DBB20BF006F94F
:1022A00005B0F0BD30000020F0B5054685B00C4605
:1022B0001D4E21B30BF012FD327805F10907D24310
:1022C0000024FFB2012382182946009320463B4692
:1022D000D2B20194029403940BF0E8F80BF0FEFCE8
:1022E0003278FF23D243821801930293039320464E
:1022F0002946D2B23B4600940BF0ACF911E00BF04A
:10230000EDFC32780121D243821805F109030091D6
:1023100020462946D2B2DBB20194029403940BF01A
:10232000C5F805B0F0BD00BF3000002070B50C4608
:10233000224605490546FFF7A5FD28463D212246D0
:10234000BDE87040FFF700BEE80901000A460149F8
:10235000FFF798BDE8090100012809D118480023BA
:1023600003701078013988420ADA0130107025E0D4
:1023700002280AD1124B02381870137813B1013BAE
:1023800013701BE00139117018E0032807D1197888
:10239000FF290CBF1278FF221A7001220CE063287B
:1023A00005D91A78FF2AF8D164381870F5E704289F
:1023B00004D100221A700132024B1A7000207047BB
:1023C00075030020900000202DE9F04115463F4A9A
:1023D00088B012780446012A0F463D4E25D1B6F842
:1023E00000C040F6736E1FFA8CFCF44517D8DFF876
:1023F000E4E0DEF854C04FF47A7EBCFBFEF80EFB3E
:1024000018CEBEF5FA7F0AD9FF2705EB000E009221
:102410005B180197029703975FFA8EF22DE0012176
:1024200000912A19DB19013921E0B6F800E041F2E8
:1024300018021FFA8EFE964514D9264AD2F854E0A7
:102440004FF47A72BEFBF2FC02FB1CE2B2F5FA7F9B
:1024500008D901270097013F2A185B1801970297B6
:10246000039709E0012100912A19DB19FE3101913E
:102470000291039120463946D2B2DBB20BF016F836
:102480003188642389B2B1FBF3F10022633B09B2C6
:1024900005A80093FEF72AFC05A80BF01DFA0E4BC9
:1024A0002D1A197805EBD575C1F10A0101EBD1712F
:1024B00004EB65044910FF23E0B2C9B205AA0093FA
:1024C00001930BF0C3FA08B0BDE8F081E6010020EB
:1024D000D203002050310020F400002001460148C2
:1024E0000CF066BE580500202DE9F0434B1EDBB210
:1024F000012B144685B00746744B754A0BD81878E3
:10250000884208D1734805786EB2022E01DC01358D
:102510000570062009E0127850B2002803DD6C48EF
:10252000013A027002E06B4A002010700129197014
:102530000CD1684B22781B7859B2C1F156018A42FE
:1025400001DA01330BE08BB156230FE0022911D1E0
:10255000604B22781B7859B28A4203DDDB43D218E4
:10256000227004E00BB9563300E0002323702046AC
:10257000012106E0042907D1237820465B4223701D
:102580000339FEF7C7FF07E0032905D120460239CA
:10259000FEF7C0FF012095E00BF0A0FB05460BF015
:1025A0009FFB6A1F431F00260A21D2B2DBB205201F
:1025B0004FF00108CDF800800196029603960BF0CB
:1025C00049F80BF08BFB05460BF08AFB6A1F431F93
:1025D000FF250A21D2B2DBB20520009601950295B3
:1025E00003950BF037F83846FEF7EEFF81460BF007
:1025F00077FB81082B464846C9B23A4600950195BB
:102600000BF024FA237843450CD90BF069FB2278B0
:10261000A0F11001023A0A20C9B2D2B24346009694
:102620000AF05CFE23786BB10BF05AFB227841086C
:1026300000230231013A00931320C9B2D2B2013310
:102640000AF04CFE0BF04AFB05460BF049FB032158
:102650006D08B0FBF1F1EB1F06310025D8B22278EE
:102660000123C9B200950AF039FE2378552B10D802
:102670000BF034FB06460BF033FB22784108223E78
:1026800002310132F0B2C9B2D2B2012300950AF090
:1026900025FE2378542B11D80BF020FB05460BF0B8
:1026A0001FFB2278A0F110010023193D0232009394
:1026B000E8B2C9B2D2B201330AF010FE3846FFF7D1
:1026C0000DFF002005B0BDE8F08300BF73030020BC
:1026D0006D0300208C0300201FB50BF0FFFA0123CF
:1026E000A0F1230200212220D2B2009309330191EC
:1026F000029103910AF0DAFE0BF0F0FA0446144856
:102700000BF0EAF8433C8442124C10DC1048FEF710
:102710006DFF23780E4AC3F10A0303EBD3735910FC
:10272000C9B2FF23009301930BF070F90FE0084842
:10273000FEF74AFF2378064AC3F10A0303EBD3737B
:102740005910C9B2FF23009301930BF07FF91FBD0D
:1027500058050020F400002030B5254D4EF66023CA
:10276000696D89B0B1FBF3F101240222002305A8B1
:1027700009B20094FEF7BAFA1E4905A80CF0F4FC61
:1027800005A80CF073FD6A6D4FF47A73B2FBF3F297
:102790003C23B2FBF3F103FB112305AA19B2101875
:1027A000002302220094FEF7A1FA00200146222213
:1027B0000A2301900290039000940AF077FE05A886
:1027C0000BF0DEF80C4BC0F12200197800EBD07052
:1027D000C1F10A0101EBD17120412141FF23C9B2AE
:1027E00005AAC0B2009301930BF010F909B030BDF7
:1027F00050310020E6090100F40000202DE9F043EB
:1028000089B0064688460BF069FA04460BF068FA70
:10281000621F431F002501270A21D2B2DBB2052027
:1028200001950295039500970AF014FF0BF056FAF4
:1028300004460BF055FA621F431FFF240A21D2B24F
:10284000DBB2052000950194029403940AF002FF84
:102850003046FEF7B9FE81460BF042FA30FA07F136
:102860000639324623464846C9B2009401940BF01B
:10287000EDF80FFA88F12A462B4605A80097FEF7D7
:1028800035FA05A8FEF7A0FE05460BF029FA30FA46
:1028900007F106312846C9B205AA234600940194DF
:1028A0000BF0D4F83046FFF719FE09B0BDE8F0830D
:1028B000012970B50646144611D1156828460DF059
:1028C00065F81DA3D3E900230DF026FB28B12846A7
:1028D0004FF07E510DF0E6FB12E01B4B13E0022996
:1028E00017D1156828460DF051F815A3D3E9002338
:1028F0000DF030FB30B128464FF07E510DF0D0FB8B
:10290000206001E0114B236020460421FEF702FE07
:1029100007E0032905D110460131FEF7FBFD012038
:1029200070BD20680DF08CFE01463046FFF766FF53
:10293000002070BDAFF3008085EB51B8FE87C34027
:1029400085EB51B8FE87C3C0F63F1CC6F63F1C4658
:10295000F8B54B1EDBB2012B154604462A4B2B4A19
:102960000BD81878884208D12948067877B2312FD9
:1029700001DC02360670062009E0127850B2002809
:1029800003DD2248013A027002E0214A0020107063
:10299000012919700CD11E4B2A781B7859B2C1F14C
:1029A000FF018A4201DA01330BE08BB1FF230FE014
:1029B000022911D1164B2A781B7859B28A4203DDBD
:1029C000DB43D2182A7004E00BB9FF3300E0002388
:1029D0002B702846012106E0042907D12B782846D0
:1029E0005B422B700339FEF795FD07E0032905D103
:1029F00028460239FEF78EFD0120F8BD20462978D1
:102A0000FFF7FCFE0020F8BD780300207F030020C4
:102A1000A1030020F8B54B1EDBB2012B154604467E
:102A20002D4B2E4A0BD81878884208D12C480678AE
:102A300077B2312F01DC02360670062009E01278E9
:102A400050B2002803DD2548013A027002E0244A12
:102A500000201070012919700FD1214B2A781B78A2
:102A600050B259B2C1F17F01884201DA01330FE05F
:102A70000BB9813313E07F2311E0022913D1184BE6
:102A80002A781B7851B258B27E38884203DCDB4387
:102A9000D2182A7004E00BB97F3300E081232B7039
:102AA0002846012106E0042907D12B7828465B42FD
:102AB0002B700339FEF72EFD07E0032905D12846C8
:102AC0000239FEF727FD0120F8BD204695F90010D8
:102AD000FFF794FE0020F8BDA50300206A03002044
:102AE0008803002030B51A4B85B093F84A3005466C
:102AF000072B04D905B0BDE83040FFF7EFBC0BF061
:102B0000EDF80123821F00240A21009305201E33C3
:102B1000D2B20194029403940AF09CFD0BF0DEF80B
:102B2000821F0A211F2300940520FF34D2B2019492
:102B3000029403940AF08EFD2846FEF745FD11210C
:102B40002A462346009401940AF080FF05B030BD68
:102B5000503100202DE9F0475A4F8CB0002201255A
:102B60001346804609B204A807F512540095FEF7F3
:102B7000BDF894F84A30072B3BD90BF0B1F894F824
:102B80004AA081460BF0AAF806460BF0A9F86FEAB6
:102B90000A0A431ED144721E00205FFA89F1D2B2A4
:102BA000DBB200950190029003900AF053FD04A857
:102BB000FEF70AFD05460BF093F8434B94F84A20C4
:102BC0001B7894F84A104FEA4818CB1A03EBD373DA
:102BD000C2EB63014118FF232846C9B204AA474447
:102BE000009301930AF032FF07F12C00FFF776FC07
:102BF00064E00BF073F8A0F10A020A2000262123FA
:102C00000146D2B200950196029603960AF022FD83
:102C10000BF064F84FEA4818A0F10A0207EB080924
:102C20000A20FF2401462123D2B209F12C09009683
:102C30000194029403940AF00DFD4846FEF7C4FC8B
:102C40000D214A462346009401940AF0FFFE04A891
:102C5000FEF7BAFC4744172104AA234638370094EC
:102C600001940AF0F3FE0F20FA792B4601460096F4
:102C70000AF034FBBB79642B07D10BF02FF81E3818
:102C80000096C0B20F21422215E0BC793CB90BF08E
:102C900025F81E380094C0B20F2143220BE0BB7907
:102CA0005BB213F1640F09D10BF018F81E380096CF
:102CB000C0B20F2144222B460AF010FB0CB0BDE835
:102CC000F08700BFD00C0020F4000020F0B585B0E4
:102CD0000E4605460BF002F804460BF001F8002101
:102CE0000091AB310191A4F10A022231A0F10C0351
:102CF0000A20FF24D2B2DBB20291014603940AF00B
:102D0000A9FC0AF0EBFF07460AF0EAFF0121009157
:102D10004231019122390291A7F10C021239A0F13E
:102D20000C030C200391D2B20146DBB20AF092FCF4
:102D30002846FEF749FC14212A46234600940194B4
:102D40000AF084FE3046FEF73FFC07460AF0C8FF53
:102D50004108C9B2384632462346009401940AF02D
:102D600075FE284605B0BDE8F040FFF7B7BB000090
:102D70002DE9F04F8BB004469DF850000F460992A4
:102D800005469B4608900AF0ABFF704E6FF00909AC
:102D900096F84A304FF00A08C3EB090981442046EF
:102DA000FFF79CFB0AF09AFF04460AF099FF96F899
:102DB0004A30621E01210024C31AD2B22046DBB27F
:102DC000009141460194029403940AF043FC0AF0F6
:102DD00087FF96F84A306FF00A02D21A5FFA89F933
:102DE000B9FBFBFCB9FBF8FA02EB0009CCEB0909D3
:102DF00005FB09F90BF1FF3B0CF1060199FBFBF90F
:102E0000CDF810C08944CDF81CB00AF067FFDFF898
:102E100048B15FFA89F99BF80010A14508BF4FF04F
:102E20000109C1F101014118C9B205910AF056FF2B
:102E300006900AF055FF069B96F84A2003F1FF3EE4
:102E40006FF0010305999B1AC3180122DBB20846F3
:102E5000009241465FFA8EF20194029403940AF0C4
:102E6000F9FB0AF03BFF9BF800100AF1FF3AC1F1B1
:102E700001014118C9B205910AF030FF06900AF02D
:102E80002FFF069B96F84A2003F1FF3E6FF00103E7
:102E900005999B1AC3185FFA8EF2DBB208460094BC
:102EA0004146FF340194029403940AF0D3FB0AF0E4
:102EB00015FF9BF800805FFA8AFAC8F10308804486
:102EC0000AF00EFF96F84A6083460AF007FFDDF825
:102ED00010C06FF009039B1BCCEB030159446943FD
:102EE000079BC21E91FBF3F101200C315FFA88F8B9
:102EF00009F10103C9B20090DBB24046D2B201949D
:102F0000029403940AF0A6FB3B78AB4284BF089975
:102F10003970554506D93B7853449D42C4BFCAEB2E
:102F200005053D703B78099A01339A44084B82F8B5
:102F300000A01B78074AC3F10A0303EBD3735B10AD
:102F4000013313700BB0BDE8F08F00BF503100208B
:102F5000F4000020D1000020300000202DE9F04FC7
:102F600089B09DF848C00E466446CDF814C007925B
:102F70009A4605460AF0B4FE3F4F6FF0090897F8ED
:102F80004A304FF00A09C3EB080880442846FFF78F
:102F9000A5FA0AF0A5FE97F84A300025C31A49465B
:102FA00031222846DBB24FF0010B019502950395C3
:102FB000CDF800B00AF04EFB0AF092FE97F84A30C6
:102FC0004946C31A30222C20DBB20095FF3501950B
:102FD000029503950AF03EFB0AF082FE97F84A300C
:102FE00098FBF9F8069381460AF07AFE069B97F85B
:102FF0004A206FF00D01C91A6FF00E039B1A1B18BF
:1030000049446143634391FBFAF193FBFAF30C31BA
:103010000F332D202F22DBB2C9B2CDF800B00195BD
:10302000029503950AF016FB337808F1FF38DDF8B6
:1030300014C0A3425FFA88F888BF86F800C04445F0
:1030400006D9337843449C42C4BFC8EB04043470AF
:1030500033780A4A01339844079B83F80080084B71
:103060001B78C3F10A0303EBD3735B1001331370B6
:1030700009B0BDE8F08F00BF50310020D100002022
:10308000F40000202DE9F04F87B09DF840409DF8F6
:1030900044809DF848A005908B461D46174608EBD6
:1030A00003090AEB0406E2B901235FFA89F9F6B2D3
:1030B0000093019202920392284621464A463346E3
:1030C0000AF0F4F9BBF1010F6CD1FF2301930293D5
:1030D0000393284621464A46334600970AF0E6F90C
:1030E00060E001235FFA89F9F6B2002700932846D1
:1030F00021464A4633460197029703970AF0D6F9CC
:10310000BBF1010F0AD1FF230193029303932846D9
:1031100021464A46334600970AF0C8F9B8F13C0FF9
:1031200030D905EB58085FFA88F8E31CFF274046C2
:1031300021464246DBB20097019702970AF043FB13
:10314000F11E33464046C9B2424604EB5A06F6B277
:103150000097019702970AF036FBEA1C2846314691
:10316000D2B233460097019702970AF02CFBA9F1DF
:103170000300C0B231464A46334600970197029792
:103180000AF021FBBAF1280F0CD9A81CA11C059A42
:10319000FF23C0B2C9B21093119307B0BDE8F04F3E
:1031A0000AF034BC07B0BDE8F08F00002DE9F04F05
:1031B000814693B09DF878500D9199F900109B4687
:1031C0006943C823680891FBF3F14118C9B29DF81F
:1031D0007C80069199F901104FEA580A01FB08F129
:1031E00091FBF3F39DF8706053449DF87470DBB26B
:1031F00011460890079391480122334600970195A4
:10320000CDF80880FFF73EFF0BFB05F0089940F66C
:10321000FE7C90FBFCF08B191818C0B208EB07037A
:10322000FF2402463946DBB2CDF814C00094019465
:1032300002940AF0C8FA642108224B465846FDF76A
:1032400067FA08FB00F1DDF814C00AEB070391FBF5
:10325000FCF15918C9B2AA193046D2B20B460094F3
:10326000019402940AF0AFFAFF3C03E0CDF81CC0D1
:10327000CDF818B019F904B0C8230BFB05FB089A68
:103280009BFBF3FB934409EB040292F901C03C2D34
:103290000CFB08FC9CFBF3FCD4445FFA8BFB5FFA4D
:1032A0008CFC1BD90CEB07030BEB0602D2B2DBB292
:1032B000002002F1FF3E591E00900132FF30013321
:1032C000019002900390C9B25FFA8EF0D2B2DBB2E5
:1032D000CDF814C00AF0EAF8DDF814C0069B079A8E
:1032E0009819D1190CEB07030BEB06024FF0FF0EF8
:1032F000C0B2C9B2D2B2DBB20434CDF814C0CDF83A
:1033000000E0CDF804E0CDF808E00AF05CFA202CEB
:10331000DDF814C0AAD10D9B002009EB83030693AE
:103320000790B346B9460D99079A91427CD1069B06
:10333000069993F9002091F901C06A430CFB08FC3F
:10334000C823089892FBF3F28218D2B29CFBF3FCDC
:10335000D44402EB0B035FFA8CFCDBB20C920CEB57
:103360000907DA1E0333FFB2DBB2D2B20A93F91EA9
:10337000FB1CFF240992DBB200261046C9B20A9A50
:103380000B930096019402940394CDF814C00AF0B4
:103390008DF8642D48D9069A012392F900100FA8E0
:1033A000324600933346FDF7A1FC25490FA80BF0E8
:1033B000DBFE0FA80BF05AFF069A012392F90110C9
:1033C0000FAA0093101833463246FDF78FFC0C9B72
:1033D0000898DDF814C0834215D3D4450AD30FA84A
:1033E0000AF07AFA09990094081A0194A7F10B01DE
:1033F000C0B214E00FA80AF06FFA099A0094101AEC
:103400000194C0B204E0D44504D20A980094019417
:103410000B9905E00A98A7F10B0100940194C9B239
:103420000FAA23460AF012FB0798431CDBB2082BB5
:1034300007937FF478AF13B0BDE8F08FCF0A010097
:10344000700A01002DE9F0430446994610F8043B48
:1034500085B03F2B0D4616469DF8308012D8FDF7FB
:10346000CDF90246204610F8143B0F495B015B186A
:103470009F88FF2100950196CDF80890CDF80C802B
:103480003BB20CE0FDF7BAF9009502460196CDF883
:103490000890CDF80C8004F11400FF210023FFF701
:1034A00085FE05B0BDE8F083080D002073B50C461D
:1034B0000546084611461E460BF07AFE0F49204687
:1034C0000BF052FE20460BF0D1FE002201230093A8
:1034D000314613462018FDF709FC094920460BF038
:1034E00043FE20460AF04CFA0A23093090FBF3F021
:1034F0004343D8B2A84238BF28467CBD720A0100B7
:10350000E10A01002DE9F04F85B01F469DF838A073
:10351000002380468C4693461C462149342202FBF8
:10352000031202F5A452303212798946424501D184
:103530000134E4B20133402BEFD16CB300252E46A9
:1035400034226A4309EB020303F5A45330331B7999
:1035500043451CD11248BAFBF4F38018023B0BF12F
:103560000102C7EB0C01B218DBB200F5A4500093C6
:1035700034303B46C9B2D2B2CDF80CC0FFF762FF7F
:103580000A2393FBF4F3F618DDF80CC0F6B201350C
:10359000402DD5D10B2000E0204605B0BDE8F08FCE
:1035A000D00C002010B500230C4A342101FB03216C
:1035B00001F5A45292F840403832844208D0927A01
:1035C000824205D001F5A6521179814218BF927945
:1035D0000133402BE8D1002010BD00BFD00C0020EB
:1035E0002DE9F04F8DB007469DF8580089461646E4
:1035F0009B4603909DF85CA00AF070FB5E4B5F4A0F
:103600001978342303FB072303F5A45393F83440BC
:1036100090463F2C00F2AB8093F84020411A01EB1A
:10362000D171CBEB610438333F2AE4B219D81A7A4E
:10363000182101FB02825B7A02F50262204604A98E
:103640000C325BB2FFF732FF0446C0EB0900FF23E8
:10365000C0B2314604AA0093019308250AF0D6F9B6
:1036600000E00025342303FB078303F5A45393F8FC
:10367000422038333F2A1BD89A7A4049182000FB51
:103680000212DB7A02F50262204604A90C325BB218
:10369000FFF70CFFA9190446C0EB0900FF23C0B2D5
:1036A000C9B204AA009301930AF0B0F90835EDB24B
:1036B000342303FB078303F5A6531A793F2A1BD84B
:1036C0001A792E49182000FB02125B7902F502627A
:1036D000204604A90C325BB2FFF7E8FEA9190446A4
:1036E000C0EB0900FF23C0B2C9B204AA0093019342
:1036F0000AF08CF90835EDB2342303FB078303F598
:10370000A6539A793F2A19D89A791C49182000FBA8
:103710000212DB7902F50262204604A90C325BB288
:10372000FFF7C4FEA9190446C0EB0900FF23C0B28D
:10373000C9B204AA009301930AF068F9342303FB89
:10374000078703980634E4B2C4EB0909831EDBB291
:10375000CBEB0901721C07F5A45000933430C9B2B9
:10376000D2B25B460B34FFF76DFEE0B200E0002002
:103770000DB0BDE8F08F00BF30000020D00C00205D
:103780002DE9F04F91B09DF868B09DF86C509DF810
:10379000709009900892644801220593CDF800B01A
:1037A0000195CDF80890FFF76DFC4FEA5903079398
:1037B000059B6A0802EB03080692079A002702EBB2
:1037C0000B0A5FFA88F85FFA8AFABC463C46CDF8E5
:1037D0003CB02E4678E02046CDF810C00CF012FD2B
:1037E000054630460CF00EFD4FF07C510CF062FDAA
:1037F000014628460CF012FE054609FB04F090FB3A
:10380000F6F00CF0B1F8CDE90A01294628460CF093
:1038100051FD29460CF04EFD014628460CF040FCB7
:10382000834607980CF0F2FC014658460CF042FD26
:10383000014628460CF034FC0CF0A8F8CDE90C0148
:1038400009980CF0DFFC0CF0A1F80022374B0CF0CB
:103850001BFA02460B46DDE90C010CF0EBF80246C0
:103860000B46DDE90A010BF033FF0CF0A5FBDDF898
:1038700010C05FFA80FB07EB0A010CEB080004EBB9
:1038800008020BEB0A03FF25C0B2C9B2D2B2DBB209
:1038900000950195029509F096FFDDF810C0C7EB81
:1038A0000A01CCEB0800C4EB0802CBEB0A03DBB245
:1038B000C0B2C9B2D2B200950195029509F083FF5A
:1038C000631CA4465F46DCB2069B9C4283D3089AE5
:1038D000354602FB06F0C826DDF83CB090FBF6F05A
:1038E00080445FFA88F009EB0B03FF245946024637
:1038F000DBB200940194029409F065FF089B1A94CE
:1039000003FB09F9059B99FBF6F6B244EA185FFA46
:103910008AF11846D2B20B461B941C9411B0BDE834
:10392000F04F09F050BF00BF740A01000000594079
:103930002DE9F04F89B09DF84C509DF850809DF8CE
:1039400054709DF858A006910792194601222B4603
:103950009DF948900197CDF80080CDF808A0FFF7B9
:1039600091FB069A4FEA5A0B02FB0BF10BEB080690
:103970006FF06303F6B205EB570C91FBF3F15FFABE
:103980008CFC7118FF24284662463346C9B2CDF834
:1039900010C000940194029409F015FF079A7B1956
:1039A000DBB2059302FB0BF34FF0640BDDF810C0A4
:1039B00009FB07F793FBFBF3F31860463146059AC2
:1039C000DBB200940194029409F0FDFEC823DDF8F7
:1039D00010C097FBF3F7BC445FFA8CF00AEB0803C6
:1039E0000246DBB2414600940194029409F0EBFEDA
:1039F000B9F1000FD5BF069A079B02FB09F903FB3B
:103A000009F999FBFBFB4FFA8BFB0AFB0BFBC82365
:103A10009BFBF3FB5E443733F1B2059A1293139389
:103A2000149328460B4609B0BDE8F04F09F0CBBE11
:103A30002DE9F04F834689B00846BDF948909DF8BE
:103A40004C509DF850809DF854709DF858A0144635
:103A50001E46FCF7ADFE06902046FCF7A9FE314657
:103A60000790012258462B460197CDF80080CDF8EB
:103A700008A0FFF707FB069A4FEA5A0B0BFB02F16F
:103A80000BEB08066FF06303F6B205EB570C91FBE6
:103A9000F3F15FFA8CFC7118FF2428466246334626
:103AA000C9B2CDF810C000940194029409F08BFEC5
:103AB000079A7B19DBB205930BFB02F34FF0640B03
:103AC000DDF810C009FB07F793FBFBF3F318604622
:103AD0003146059ADBB200940194029409F073FE1A
:103AE000DDF810C040F6FE7397FBF3F7BC445FFAB5
:103AF0008CF00AEB08030246DBB2414600940194C5
:103B0000029409F060FEB9F1000FCBBF079B069A43
:103B100009FB03F909FB02F999FBFBFB0FFA8BFB8D
:103B20000AFB0BFB40F6FE739BFBF3FB5E44FF239B
:103B3000F1B2059A12931393149328460B4609B0D9
:103B4000BDE8F04F09F03FBE2DE9F04F8BB01446B1
:103B50009DF8602007460846BDF950A09DF85450D6
:103B60009DF858909DF85C801E460792FCF720FE59
:103B700008902046FCF71CFE079B099002933846EC
:103B8000314601222B46CDF80480CDF80090FFF796
:103B900079FA08994FEA580B0BFB01F20BEB05077A
:103BA0006FF06303FFB292FBF3F2BA18D2B2059240
:103BB000079AFF244FEA520C0CFB01F20CEB0906AA
:103BC000F6B292FBF3F3F318DBB2069305981946AD
:103BD0003A463346CDF810C000940194029409F09F
:103BE000F2FD06992846059A0B460094019402942A
:103BF00009F0E9FD0999DDF810C00BFB01F30CFB9E
:103C000001FC4FF0640B93FBFBF39CFBFBFCFB18EC
:103C1000B4445FFA8CFCDBB20593384631461A4651
:103C20006346CDF810C000940194029409F0CBFDD6
:103C3000DDF810C008EB05030AFB08F8DBB26146AB
:103C4000069305981A46634600940194029409F07D
:103C5000BAFD40F6FE73079A98FBF3F84744F8B2B2
:103C600002EB09034946DBB2024600940194029438
:103C700009F0A9FDBAF1000FCBBF099B08990AFB17
:103C800003FA0AFB01FA079A9AFBFBFB0FFA8BFB7C
:103C900002FB0BFB40F6FE739BFBF3FB5E44FF2332
:103CA000F1B2069A14931593169328460B460BB05F
:103CB000BDE8F04F09F087BD2DE9F04F8DB00A93B4
:103CC0009DF85C309DF858900B93002306460F46F4
:103CD00009921D46FF2E09D1484A0C2101FB0322FF
:103CE00002F5945230321279BA420ED0FF2F0ED123
:103CF000DAB296420BD1414A0C2101FB062202F5B1
:103D00009452303212793F2A01D80135EDB2013395
:103D1000102BDFD1002D6CD00024A046FF2E09D13E
:103D2000364B0C2202FB043303F5945330331B79DA
:103D3000BB420ED0FF2F57D1E3B29E4254D12F4B3E
:103D40000C2202FB063303F5945330331B793F2BCF
:103D50004AD84FF00C0B0BFB04FBDFF8A0A00BF5CF
:103D600094530AEB03023C32104607930892FCF787
:103D70001FFD089A014610460691FCF719FD079BA6
:103D80000246534403F138000892FCF737FDD34450
:103D900003460BF5945030300079DDF824E0400103
:103DA00082449AF83E00069940B20090C9EB0E009A
:103DB000DDF828E0C0B201900EF101004044DDF8CA
:103DC0002CE0C0B20290BEFBF5F00238C0B2049005
:103DD000089A0B48CDF80C90FFF7AAFD0A2393FB35
:103DE000F5F398445FFA88F80134102C96D10B2033
:103DF00000E028460DB0BDE8F08F00BFD00C0020D9
:103E0000790A01002DE9F04F89B006469DF84C0073
:103E100006939DF8489000230F46059207901D4693
:103E2000FF2E09D1444A0C2101FB032202F58E52D8
:103E300030321279BA420ED0FF2F0ED1DAB296424A
:103E40000BD13D4A0C2101FB062202F58E52303285
:103E500012793F2A01D80135EDB20133102BDFD1A1
:103E6000002D65D00024A046FF2E09D1324B0C2234
:103E700002FB043303F58E5330331B79BB420ED063
:103E8000FF2F50D1E3B29E424DD12B4B0C2202FBAF
:103E9000063303F58E5330331B793F2B43D84FF055
:103EA0000C0B0BFB04FBDFF890A00BF58E530AEB19
:103EB00003003C300493FCF77BFC049B8446534492
:103EC00003F13800CDF810C0FCF798FCD3440BF593
:103ED0008E5330331B79DDF814E05B019A44C9EB53
:103EE0000E03DDF818E001460EF101004044DDF854
:103EF0001CE0C0B29AF83E200090AEF10200DDF85E
:103F000010C090FBF5F0C0B20290DBB25FFA8CF00B
:103F100052B2CDF80490FFF733FC0A2393FBF5F37C
:103F200098445FFA88F80134102C9DD10B2000E0F2
:103F3000284609B0BDE8F08FD00C00202DE9F04FE5
:103F40008DB00A939DF85C309DF858900B93002338
:103F500006460F4609921D46FF2E09D1484A1421F4
:103F600001FB032202F59A5230325279BA420ED046
:103F7000FF2F0ED1DAB296420BD1414A142101FB38
:103F8000062202F59A52303252793F2A01D8013581
:103F9000EDB20133102BDFD1002D6DD00024A046EF
:103FA000FF2E09D1364B142202FB043303F59A533A
:103FB00030335B79BB420ED0FF2F58D1E3B29E4223
:103FC00055D12F4B142202FB063303F59A5330339D
:103FD0005B793F2B4BD84FF0140B0BFB04FBDFF846
:103FE000A0A00BF59A5303F138025244101D089318
:103FF0000792FCF7DDFB079A014602F108000691E3
:10400000FCF7D6FB089B0246534403F138000792A5
:10401000FCF7F4FBD34403460BF59A50303040795B
:10402000DDF824E0400182449AF83E00069940B24F
:104030000090C9EB0E00DDF828E0C0B201900EF14F
:1040400001004044DDF82CE0C0B20290BEFBF5F068
:104050000238C0B20490079A0A48CDF80C90FFF7D6
:1040600067FC0A2393FBF5F398445FFA88F8013460
:10407000102C95D10B2000E028460DB0BDE8F08F44
:10408000D00C0020820A01002DE9F04F8DB00A9378
:104090009DF85C309DF858900B93002306460F4620
:1040A00009921D46FF2E08D103F5067241490332DD
:1040B00001EB02121279BA420DD0FF2F0DD1DAB204
:1040C00096420AD106F506723A49033201EB021212
:1040D00012793F2A01D80135EDB20133102BE1D11D
:1040E000002D63D00024A046FF2E08D104F50673EE
:1040F000304A033302EB03131B79BB420DD0FF2F71
:104100004FD1E3B29E424CD106F50673294A0333E0
:1041100002EB03131B793F2B43D82201DFF894A055
:1041200002F5065204F5067B38320BF1030B5244BC
:104130000AEB0B1B02F108010BF108000432089195
:104140000792FCF75BFB03469BF804004FF0180E48
:104150000EFB00A000F5026070448088DDF824E0CA
:1041600000B20090C9EB0E00DDF828E0C0B201906B
:104170000EF101004044DDF82CE0C0B20290BEFB1D
:10418000F5F00238C0B2049008990B48079ACDF8B0
:104190000C90FFF74DFC0A2393FBF5F398445FFA6C
:1041A00088F80134102C9FD10B2000E028460DB078
:1041B000BDE8F08FD00C0020890A01002DE9F04FF6
:1041C0008DB00A939DF85C309DF858900B930023B6
:1041D00006460F4609921D46FF2E08D103F50A72C6
:1041E0004149033201EB02121279BA420DD0FF2F7E
:1041F0000DD1DAB296420AD106F50A723A49033273
:1042000001EB021212793F2A01D80135EDB20133D8
:10421000102BE1D1002D63D00024A046FF2E08D141
:1042200004F50A73304A033302EB03131B79BB42D4
:104230000DD0FF2F4FD1E3B29E424CD106F50A7349
:10424000294A033302EB03131B793F2B43D8220186
:10425000DFF894A002F50A5204F50A7B38320BF11C
:10426000030B52440AEB0B1B02F108010BF108008F
:10427000043208910792FCF7C1FA03469BF8040048
:104280004FF0180E0EFB00A000F50260704480880D
:10429000DDF824E000B20090C9EB0E00DDF828E064
:1042A000C0B201900EF101004044DDF82CE0C0B234
:1042B0000290BEFBF5F00238C0B2049008990B489A
:1042C000079ACDF80C90FFF73FFC0A2393FBF5F318
:1042D00098445FFA88F80134102C9FD10B2000E03D
:1042E00028460DB0BDE8F08FD00C00208D0A0100EB
:1042F0002DE9F04F91B017469DF86C20804607924B
:104300000022099113468D48342101FB020101F579
:10431000A45191F838408146444503D03831097999
:10432000414501D101339BB20132402AEBD1403AE1
:104330000C2101FB029101F58E5191F838004045A6
:1043400003D038310979414501D101339BB20132A3
:10435000102AEDD1103A0C2101FB029101F5945184
:1043600091F83800404503D038310979414501D1F1
:1043700001339BB20132102AEDD1103A142101FB16
:10438000029101F59A5191F83800404507D091F813
:104390003C003831404502D0097A414501D1013312
:1043A0009BB20132102AE9D1103A02F506710331AD
:1043B00009EB0111097A41450FD0604802F580717F
:1043C000013100EB011101F58C5191F82C002831DD
:1043D000404502D0097A414501D101339BB20132F7
:1043E000102AE2D1103A02F50A71033109EB0111EA
:1043F000097A41450FD0514802F58871013100EB2F
:10440000011101F58C5191F82C002831404502D062
:10441000097A414501D101339BB20132102AE2D120
:10442000002B00F00A85042B28BF04230593059A6E
:10443000042393FBF2F3023B099EDBB24FF0000B27
:10444000C2460693B8461C465D463746342606FBF0
:104450000B9606F5A45696F838303036534532D1CF
:1044600037490AA80AF0A4FE3179344B490159189A
:104470002C310AA80AF078FE0AA809F081FAA7F1FF
:104480000A0604EB0801301AFF23C9B20AAAC0B217
:104490000093019309F0BAFA059A082393FBF2F30B
:1044A0000AA8E41809F06CFAA842E4B203D90AA8F1
:1044B00009F066FA0546082C05D90F3F7F1B069CBC
:1044C00007F0FF070025342000FB0BF009EB000C80
:1044D0000CF5A45C9CF83C3053455BD1174B002293
:1044E000181810AE00F5A45006F8182D3C30CDF881
:1044F0000CC00492FCF75CF9049A01230146009376
:1045000030461346FCF7F2FB0E4930460AF02CFE0B
:10451000DDF80CC0094A9CF83410304649015118A6
:104520002C310AF021FE079AA7F10A0308935AB129
:10453000304609F025FA089B181A0AE0D00C002032
:10454000960A0100950A0100304609F019FA089A06
:10455000101A04EB0801FF23C9B23246C0B200931F
:10456000019309F053FA059A082393FBF2F30AA882
:10457000E41809F005FAA842E4B203D90AA809F040
:10458000FFF90546082C05D90F3F7F1B069C07F055
:10459000FF0700250BF1010BBBF1400F7FF456AF75
:1045A0003E46ABF1400B37460C2606FB0B9606F554
:1045B0008E5696F838303036534532D18A490AA89B
:1045C0000AF0F6FD3179894B490159182C310AA8B6
:1045D0000AF0CAFD0AA809F0D3F9A7F10A0604EB0C
:1045E0000801301AFF23C9B20AAAC0B2009301938E
:1045F00009F00CFA059A082393FBF2F30AA8E418D1
:1046000009F0BEF9A842E4B203D90AA809F0B8F942
:104610000546082C05D90F3F7F1B069C07F0FF07B6
:1046200000250C2000FB0BF009EB000C0CF58E5C58
:104630009CF83C30534555D16C4B0022181810AEF5
:1046400000F58E5006F8182D3C30CDF80CC00492C1
:10465000FCF7AEF8049A0123014600933046134656
:10466000FCF744FB624930460AF07EFDDDF80CC0E1
:104670005E4A9CF834103046490151182C310AF03A
:1046800073FD079AA7F10A0308932AB1304609F08F
:1046900077F9089B181A04E0304609F071F9089A76
:1046A000101A04EB0801FF23C9B23246C0B20093CE
:1046B000019309F0ABF9059A082393FBF2F30AA8DA
:1046C000E41809F05DF9A842E4B203D90AA809F098
:1046D00057F90546082C05D90F3F7F1B069C07F0AC
:1046E000FF0700250BF1010BBBF1100F7FF45CAF4E
:1046F0003E46ABF1100B37460C2606FB0B9606F533
:10470000945696F838303036534532D139490AA894
:104710000AF04EFD3179354B490159182C310AA860
:104720000AF022FD0AA809F02BF9A7F10A0604EB0A
:104730000801301AFF23C9B20AAAC0B2009301933C
:1047400009F064F9059A082393FBF2F30AA8E41828
:1047500009F016F9A842E4B203D90AA809F010F941
:104760000546082C05D90F3F7F1B069C07F0FF0765
:1047700000250C2000FB0BF009EB000C0CF5945C01
:104780009CF83C3053455FD1184B0022181810AEEE
:1047900000F5945006F8182D3C30CDF80CC004926A
:1047A000FCF706F8049A01230146009330461346AD
:1047B000FCF79CFA104930460AF0D6FCDDF80CC034
:1047C0000A4A9CF834103046490151182C310AF03D
:1047D000CBFC079AA7F10A0308937AB1304609F097
:1047E000CFF8089B181A0EE09D0A0100D00C00209B
:1047F0009C0A0100A40A0100A30A0100304609F046
:10480000BFF8089A101A04EB0801FF23C9B2324618
:10481000C0B20093019309F0F9F8059A082393FBBD
:10482000F2F30AA8E41809F0ABF8A842E4B203D9FD
:104830000AA809F0A5F80546082C05D90F3F7F1BEB
:10484000069C07F0FF0700250BF1010BBBF1100FD1
:104850007FF452AF3E464746D046C1464FF0000A6D
:10486000B846BB4B142707FB0A3707F59A5797F84A
:10487000382030374A4531D1B6490AA80AF098FCA9
:104880007979B34B490159182C310AA80AF06CFC0C
:104890000AA809F075F8A6F10A0704EB0801381A0E
:1048A000FF23C9B20AAAC0B20093019309F0AEF87F
:1048B000059A082393FBF2F30AA8E41809F060F8BC
:1048C000A842E4B203D90AA809F05AF80546082C10
:1048D00004D90F3E761B069C06F0FF06142000FB51
:1048E0000AF09B4B03EB000C0CF59A5C9CF83C30F7
:1048F0004B4549D110AF4FF0000B07F818BD0CF134
:104900003C00CDF80CC0FBF753FF01235A4601468B
:10491000009338465B46FCF7E9F98F4938460AF0C0
:1049200023FCDDF80CC08A4B9CF835103846490151
:1049300059182C310AF018FC384609F021F8A6F174
:104940000A0B04EB0801C0EB0B00FF23C9B23A4687
:10495000C0B20093019309F059F8059A082393FB1C
:10496000F2F30AA8E41809F00BF8A842E4B203D95C
:104970000AA809F005F80546082C05D90F3E761B54
:10498000069C06F0FF060025142000FB0AF0704B81
:1049900003EB000C0CF59A5C9CF840304B454BD176
:1049A0006B4A10AF4FF0000B101807F818BD00F558
:1049B0009C50CDF80CC0FBF7FBFE01235A46014684
:1049C000009338465B46FCF791F9634938460AF094
:1049D000CBFBDDF80CC05E4B9CF835103846490126
:1049E00059182C310AF0C0FB384608F0C9FFA6F16F
:1049F0000A0B04EB0801C0EB0B00FF23C9B23A46D7
:104A0000C0B20093019309F001F8059A082393FBC3
:104A1000F2F30AA8E41808F0B3FFA842E4B203D9FD
:104A20000AA808F0ADFF0546082C05D90F3E761BF5
:104A3000069C06F0FF0600250AF1010ABAF1100FE4
:104A40007FF40FAFAAF1100A414B0AF5067703373E
:104A500003EB07173B7A4B4531D140490AA80AF0CE
:104A6000A7FB39793A4B490159182C310AA80AF0A9
:104A70007BFB0AA808F084FFA6F10A0704EB0801F3
:104A8000381AFF23C9B20AAAC0B20093019308F0F2
:104A9000BDFF059A082393FBF2F30AA8E41808F077
:104AA0006FFFA842E4B203D90AA808F069FF0546DF
:104AB000082C04D90F3E761B069C06F0FF060AF56B
:104AC00080700130DFF888B000010BEB000303F5C4
:104AD0008C5328331B794B4557D1584410AF0022D3
:104AE00000F58C5007F8182D2C300492FBF760FE6F
:104AF000049A01230146009338461346FCF7F6F862
:104B0000174938460AF030FB0AF5067303330BEBFE
:104B100003131B7938465B019B440BF12C010AF00F
:104B200023FB384608F02CFFA6F10A0B04EB080122
:104B3000C0EB0B00FF23C9B23A46C0B20093019309
:104B400008F064FF059A082393FBF2F30AE000BF24
:104B5000D00C0020AA0A0100A90A0100B00A010035
:104B6000AF0A01000AA8E41808F00AFFA842E4B25C
:104B700003D90AA808F004FF0546082C05D90F3E02
:104B8000761B069C06F0FF0600250AF580700130B2
:104B9000DFF8B8B200010BEB000303F58C532833A8
:104BA0001B7A4B454BD1584410AF002200F58C5076
:104BB00007F8182D30300492FBF7FAFD049A012310
:104BC0000146009338461346FCF790F89E49384654
:104BD0000AF0CAFA0AF5067303330BEB03131B79C9
:104BE00038465B019B440BF12C010AF0BDFA3846B4
:104BF00008F0C6FEA6F10A0B04EB0801C0EB0B009F
:104C0000FF23C9B23A46C0B20093019308F0FEFEFA
:104C1000059A082393FBF2F30AA8E41808F0B0FE03
:104C2000A842E4B203D90AA808F0AAFE0546082C57
:104C300005D90F3E761B069C06F0FF0600250AF1FB
:104C4000010ABAF1100F7FF4FFAEAAF1100A7F4BF0
:104C50000AF50A77033703EB07173B7A4B4531D147
:104C60007B490AA80AF0A4FA3979784B4901591806
:104C70002C310AA80AF078FA0AA808F081FEA6F1F9
:104C80000A0704EB0801381AFF23C9B20AAAC0B206
:104C90000093019308F0BAFE059A082393FBF2F300
:104CA0000AA8E41808F06CFEA842E4B203D90AA8E6
:104CB00008F066FE0546082C04D90F3E761B069CBC
:104CC00006F0FF060AF588700130DFF880B10001B8
:104CD0000BEB000303F58C5328331B794B454BD169
:104CE000584410AF002200F58C5007F8182D2C30D6
:104CF0000492FBF75DFD049A0123014600933846B8
:104D00001346FBF7F3FF534938460AF02DFA0AF52C
:104D10000A7303330BEB03131B7938465B019B4487
:104D20000BF12C010AF020FA384608F029FEA6F112
:104D30000A0B04EB0801C0EB0B00FF23C9B23A4693
:104D4000C0B20093019308F061FE059A082393FB1B
:104D5000F2F30AA8E41808F013FEA842E4B203D95B
:104D60000AA808F00DFE0546082C05D90F3E761B53
:104D7000069C06F0FF0600250AF588700130DFF872
:104D8000CCB000010BEB000303F58C5328331B7AE6
:104D90004B454BD1584410AF002200F58C5007F81A
:104DA000182D30300492FBF703FD049A01230146CD
:104DB000009338461346FBF799FF264938460AF018
:104DC000D3F90AF50A7303330BEB03131B79384647
:104DD0005B019B440BF12C010AF0C6F9384608F040
:104DE000CFFDA6F10A0B04EB0801C0EB0B00FF237B
:104DF000C9B23A46C0B20093019308F007FE059A83
:104E0000082393FBF2F30AA8E41808F0B9FDA842BE
:104E1000E4B203D90AA808F0B3FD0546082C05D969
:104E20000F3E761B069C06F0FF0600250AF1010ADC
:104E3000BAF1100F7FF40BAF00E0099E099B9E1B97
:104E4000F0B211B0BDE8F08FAF0A0100D00C002025
:104E5000B60A0100BB0A0100012908B5104605D1B8
:104E600013785AB2632A0ADC013307E002290BD116
:104E700013785AB212F1630F01DB013B0370012179
:104E8000FCF748FB002008BD0339C9B2012904D84A
:104E90000121FCF73FFB012008BD002008BD0000F8
:104EA0002DE9F041464B05461F7888B0FF2F084694
:104EB00016461C4663D1434F03213A46FDF74CFA90
:104EC000414C3B782846009321460DF11F020323F5
:104ED000FEF744F80A252478B8464BE0022C45D862
:104EE00098F8001028460B1B594241EB0301FDF7CF
:104EF000A1F9012C334F0AD0022C1DD03978284655
:104F0000D1F1010138BF0021FDF720FA2EE02F4931
:104F100003A80AF04DF903A80AF0A8F9002203AB90
:104F200096F90010181813460094FBF7DFFE3A7844
:104F3000284603A9012A14E0254903A80AF038F9F4
:104F400003A80AF093F901230022009303AB96F91A
:104F5000011018181346FBF7C9FE3A78284603A932
:104F6000022A14BF00220122FDF7E0F80A350134BD
:104F7000EDB2E4B29DF81F30A342AFD81CE0012F80
:104F800009D002D3022F17D108E0124A0120107075
:104F9000FF221A7011E0104B586802E00E4B0132EC
:104FA0009868FF23FFF758FF012805D1094B1870B7
:104FB000FF232370013800E0002008B0BDE8F08135
:104FC0003F010020720300206C030020FD0F010050
:104FD000C20A010090000020D40000202DE9F04F0B
:104FE0007B4B8BB01F788046FF2F0E4614461D4624
:104FF00064D1784F08463A461121FDF7ADF9764E57
:105000003B783146009381460DF12702404611233B
:10501000FDF7A4FF4FF00A08367832E039784046B1
:105020008B1B594241EB0301FDF704F93A783EB975
:10503000D2F10101404638BF0021FDF787F91AE09F
:10504000082E0AD8C6EB020CDCF1000240463146BD
:1050500042EB0C02FDF75AF80DE0C6EB020E5F4B77
:10506000A6F10901DEF10002404653F8211042EB9F
:105070000E02FDF75BF808F10A0801365FFA88F8BE
:10508000F6B29DF82730B342C8D83E7808F026FE25
:10509000074608F025FE013E32230B38F6B2009396
:1050A000333F283BC0B20193FFB203903146204604
:1050B00001220A3B0297FEF779F847E12FB9484AE7
:1050C00001201070FF221A7063E1092F0ED1002316
:1050D0001A46072192FBF1F16439C832E018E15415
:1050E0000433B2F5C86F4170F3D132E10A2F0ED10B
:1050F00000236422E118E2540433202B4A70F8D1D3
:105100007C33237063709C3B2371637121E10B2F0F
:105110001BD100226423A118A3540432202A4B700F
:10512000F8D17C3222706270627133322272CF3ACF
:10513000CE21627231206273323222742171207367
:10514000637423756375313A04E10C2F0BD100238E
:10515000E21892F90110043301EBD1714910202BB0
:105160005170F5D1F5E00D2F08D10023E2185178E8
:1051700004334942202B5170F8D1EAE00E2F12D1AE
:105180000023E21851780139517049B211F1640FCE
:1051900001DA9C2102E0642901DD642151700433AD
:1051A000202BEED1D5E00F2F1CD10023E21851782F
:1051B0000131517049B211F1640F01DA9C2102E012
:1051C000642901DD642151700433202BEED1C0E04D
:1051D000A8000020AC030020A40300205C000020F5
:1051E00090000020102F72D16B4FFF236B483A467E
:1051F000FDF7AEFB3B7884463E460BB901333B706E
:105200003378402B02D9644B40221A7096F8008004
:10521000634F342308F1FF3803FB087895F80090BA
:10522000CDF814C008F05AFD069008F059FD07901B
:1052300008F054FD834608F051FD824608F050FD09
:10524000069A079BD208D2B200920522B3FBF2F372
:1052500003EB43030BF1FF3BDBB2ABEB9A0A019389
:105260005FFA8AF302938308013B08F5A65809F117
:10527000FF39DBB208F108085FFA89F90393043AB1
:10528000002340464946FDF791FFDDF814C0BCF10C
:10529000010F63D10022134630780D21013801FB44
:1052A000003000F5A66007EB8000007AA05430784B
:1052B000013801FB003101F5A66107EB8101487A55
:1052C0000133A1180432082B4870E5D141E008F001
:1052D00005FD814608F004FD32230093A9F133094E
:1052E000283B0B38791E0193C0B25FFA89F3012283
:1052F0000293039000232046C9B2FDF757FF2B7895
:105300004046013B04EB83023146DBB2FFF7C8FDA8
:10531000012E81460DD1234604F11C011A7893F920
:10532000046050B28642B8BF1A7104338B42F5D183
:105330000CE0022E0AD10023E2181279E05651B295
:105340008842C8BFE25404331C2BF5D1B9F1010FD8
:1053500004D10122134B1A70FF232B700023E25655
:1053600012F1640F01DA9C2202E0642A01DD64225A
:10537000E254E21892F9011011F1640F01DA9C2154
:1053800002E0642901DD642151700433202BE6D151
:1053900000200BB0BDE8F08F6F030020C50A0100AC
:1053A000D00C0020900000202DE9F0434D4E85B038
:1053B00035788146FF2D144667D14B4F08463A4653
:1053C00043213346FCF7C8FFDFF83C813B780DF101
:1053D0000F020093484643234146FDF7C9FC434B67
:1053E0001A78FF2A04D01B7801272370357075E0E6
:1053F00098F800400A2542E0397828460B1B5942AC
:1054000041EB0301384EFCF74FFF3CB93278284698
:10541000D2F10102364938BF002208E0012C09D13F
:10542000327834492846012A14BF00220122FCF7B1
:1054300029FD20E0022C04D1327828462E49022A88
:10544000F2E7422C17D832782846C4EB020CDCF184
:10545000000242EB0C022949FCF714FD3278284B7C
:10546000C4EB020E6101DEF100022846194442EB52
:105470000E02FCF729FD0A350134EDB2E4B29DF8C5
:105480000F30A342B8D8002728E01E4B2DB9FF22C9
:10549000012722701F70327015E0012D0AD1FE2203
:1054A00022701D70FF23337020462946FCF732F826
:1054B0002F4613E0022D4FF0010706D1FD22227086
:1054C0001F70FF233370204605E0033D15701F70E9
:1054D000FF23337010463946FCF71CF8384605B0F8
:1054E000BDE8F083D000002068030020E201002026
:1054F000D50A0100E40A0100F40A0100000B0100D2
:105500009C0C0020900000207E030020F0B5334B5F
:10551000064610461A7885B0FF2A4DD1304C084611
:1055200022464121FCF718FF2E4D23783046009388
:1055300029460DF10F024123FDF71AFC0A262D78AA
:1055400034E0217830464B1B594241EB0301244F94
:10555000FCF7AAFE4DB93A783046D2F10102224951
:1055600038BF0022FCF78EFC1CE0402D1AD83A7898
:105570003046C5EB020CDCF1000242EB0C021B4989
:10558000FCF780FC1A4B6A1E182101FB02313A78A5
:105590000431C5EB020EDEF10002304642EB0E0292
:1055A000FCF792FC0A360135F6B2EDB29DF80F30E9
:1055B000AB42C6D800200FE00E4901241AB9FF32D1
:1055C00002700C7003E0013A02700C70FF221A7036
:1055D0002146FBF79FFF204605B0F0BD31000020BB
:1055E00096030020AE030020060B01000B0B010008
:1055F000F8140020900000202DE9F04F137889B0B6
:10560000FD2B064614460BD003F102095FFA89F917
:10561000B9F1010F94BF4FF002094FF0040901E006
:105620004FF003098F4D6F78FF2F40F0DA80084666
:105630002A4649466B1CFCF78FFE2B788A490DF1F0
:105640001F02304600934B46FDF792FB08F048FBE3
:10565000064608F043FB804608F042FBA6F10A012B
:1056600042460026DFF8308203464FF0010A3046FA
:10567000C9B2CDF800A001960296039607F016FF76
:1056800098F84A30002B3BD008F02AFB98F84A20C3
:105690000490059208F022FB834608F021FB059A4E
:1056A000049BD2439918431E0BF1FF32C9B2D2B208
:1056B0003046DBB2CDF800A001960296039607F0C3
:1056C000F5FE6A4E2B7856F82300FBF77DFF8246E5
:1056D00008F006FB664B98F84A201B7898F84A10A9
:1056E0000097CB1A03EBD373C2EB63012B784118FD
:1056F000019756F823205046C9B23B4608F0A6F958
:10570000594B0A261F7867E029783046CB1B59424F
:1057100041EB0301FCF7C8FD4F4559D22378FD2B1F
:10572000544B0ED1022F0CD14E4A304612781969D3
:10573000A2F1020CDCF1000242EB0C02FCF7A2FB2E
:105740002EE02A783046C7EB020EDEF1000242EB73
:105750000E0253F82710FCF795FB022F20D0414B87
:10576000032F1A7822D0012F2AD12178FF2902D1C4
:105770003046414912E0FE2902D130463F490DE052
:10578000FD2902D130463E4908E03F2904D83D4B6F
:1057900049013046C91801E03B493046012A12E070
:1057A0002A78304694F90110022A03E094F9021095
:1057B0003046032A14BF00220122FCF78DFC07E0CB
:1057C00032493046BA4214BF00220122FCF77CFB6A
:1057D0000A360137F6B2FFB29DF81F30BB4293D8AC
:1057E0003CE0032F3AD8DFE807F0020D242C284BC9
:1057F00001261E702046FF2304216B70FBF78AFEF2
:1058000030462CE01B4B22465868FF23FFF7CCFDA7
:10581000204F06463B78FF2B1AD008F0CFFC387893
:1058200008F0F2FC002801DD642300E09C23637093
:105830000EE0FD2B0F4B04F101020CBF18699868B4
:1058400002E00C4BA21CD868FF23FDF7E3F80646E4
:10585000012E03D10E4B1E70FF236B70002009B088
:10586000BDE8F08F42010020A0030020E0000020EE
:10587000F400002000000020D50A0100E40A010025
:10588000F40A0100FC0C0020120B0100D10D0100F4
:1058900090000020E2010020503100202DE9F04F5F
:1058A000137891B0FD2B0646154601D102331370D3
:1058B00095F80090924C09F1020967795FFA89F92D
:1058C000B9F1010F94BF4FF002094FF00509FF2F06
:1058D00040F0E8800846221D4946631DFCF73CFD68
:1058E000237988490DF13F02304600934B46FDF77E
:1058F0003FFA08F0F5F9064608F0F0F9804608F09E
:10590000EFF9A6F10A0142460026DFF8308203468D
:105910004FF0010A3046C9B2CDF800A001960296B8
:10592000039607F0C3FD98F84A30002B3BD008F0EF
:10593000D7F998F84A200490059208F0CFF98346E9
:1059400008F0CEF9059A049BD2439918431E0BF137
:10595000FF32C9B2D2B23046DBB2CDF800A0019618
:105960000296039607F0A2FD674E237956F82300AE
:10597000FBF72AFE824608F0B3F9644B98F84A20F8
:105980001B7898F84A100097CB1A03EBD373C2EB3D
:10599000630123794118019756F823205046C9B274
:1059A0003B4608F053F8574B0A261F7875E02179DB
:1059B0003046CB1B594241EB0301FCF775FC4F45C8
:1059C00067D24F4B30461A79514BC7EB020CDCF1D2
:1059D000000253F8271042EB0C02FCF753FA7B1E2F
:1059E000032B4DD8DFE803F0022E343F2978FF293E
:1059F00003D122793046474922E0FE2903D122799A
:105A0000304645491CE0A1F14003DBB2BD2B14D95F
:105A1000424B490107A8C91809F0CAFB2846FAF702
:105A2000EDFE10B107A83E4901E03E4907A809F084
:105A30009BFB2279304607A902E022793A49304699
:105A4000012A21E02279304695F90110022A04E06A
:105A5000227995F902103046032A14BF0022012250
:105A6000FCF73AFB15E022793046A2F1040EDEF194
:105A7000000295F9031042EB0E02FCF751FA08E020
:105A800022792A493046BA4214BF00220122FCF78B
:105A90001BFA0A360137F6B2FFB29DF83F30BB421F
:105AA00085D85AE0042F58D8DFE807F0030E2023EA
:105AB0004A001F4B01261E702846FF2304216371F4
:105AC000FBF728FD304649E0114B2A465868FF2372
:105AD000FFF76AFC174B06461B78FF2B37D008F000
:105AE0006DFB64236B70503BAB7030E012486A1C56
:105AF00002E0074BAA1CD868FF23FCF78BFF25E0C8
:105B000042010020A703002048000020F4000020EC
:105B1000BC000020660A01005D0A0100FC0C0020A8
:105B2000500A0100560A0100120B0100D10D0100BC
:105B300090000020E2010020C4000020503100202D
:105B4000084BEA1C1869FF23FBF76DFD0646012E82
:105B500003D1054B1E70FF236371002011B0BDE817
:105B6000F08F00BFBC000020900000202DE9F04F16
:105B7000814D8FB0804608F0B3F82B78FF2B40F0B2
:105B800060810A27A0F10C0696FBF7F6F6B27B4877
:105B9000FCF7A4FC4FEA460A794C402191FBFAF14C
:105BA00022462B4601314046FCF7D6FB08F096F81A
:105BB0000C3800EBD070401080B2069008F090F8DE
:105BC0002478A0F10B0508F089F8640095FBF6F540
:105BD0007443064608F084F80121431E721E00201B
:105BE0000091D2B23946DBB201900290039007F0E7
:105BF00031FD06990698C9B2E4B2400801F10803E4
:105C00005FFA80F9DBB204F1010B544409F1040896
:105C1000EAB201349944ED190D9409905FFA88F8BD
:105C20000A9107935FFA89F90B92EDB20C24FEE01A
:105C30000598544A4301D31838339B796FF06301B8
:105C40005BB28B42B8BF0B460699642BA8BF642396
:105C500003FB01F0C92190FBF1F10998002B0144ED
:105C600089B20C914FF0010301F104020ADD0093A7
:105C7000FE330193643B0293963B039340462146D7
:105C8000D2B208E00093FF230193FA3BD0B2029313
:105C900003932146424604F1020A5FFA8AFA2B4630
:105CA000FF2607F0D7FC9B27404621464246534635
:105CB00000960197029707F086FDAB1EDBB21946EE
:105CC0000893404642462B4600960197029707F0FC
:105CD0007AFD0C99089B081DC0B2514602460096F9
:105CE0000197029707F06FFD059B26485A0182181D
:105CF0002C321046049207F043FEA8EB50005146A8
:105D0000049A3346C0B20096019607F07FFE0A99C6
:105D100000230A1D042000932146D2B22B4601968F
:105D20000296039607F096FC164A4FEA4B13D318D7
:105D300038339B796FF063025BB29342B8BF13466E
:105D40000698642BA8BF642303FB00F1C92291FBD2
:105D5000F2F2099907988A1892B2002B05924FF037
:105D60000103024410DD009304330196029703936C
:105D700048462146D2B20FE03E010020190B010037
:105D8000A3030020D00C002000930523D0B201967D
:105D90000293039321464A462B46FF2607F05AFCFE
:105DA0009B27214648464A4653460197029700964C
:105DB00007F009FD2B46484608994A460197029785
:105DC000009607F000FD0799059A089B8818C0B255
:105DD0000246514601970297009607F0F4FC1E4BCD
:105DE0004FEA4B17DF192C37384607F0C9FDA9EBEE
:105DF000500051463A463346C0B20096019607F02D
:105E000005FE0A98002342000832214600930798B5
:105E10002B4602F0FE0201960296039607F01AFC4A
:105E20000B990BF1020B64186D18E4B2EDB20D9AE8
:105E300093450CD00BF1FF333F2B05937FF7F8AE62
:105E400005E0064B01201870FF232B7000E00020B6
:105E50000FB0BDE8F08F00BFD00C002090000020F4
:105E60002DE9F04F894D91B0804607F039FF2B782E
:105E7000FF2B40F072810A27A0F10C0696FBF7F683
:105E8000F6B28348FCF72AFB4FEA460A814C4021D0
:105E900091FBFAF122462B4601314046FCF75CFAB1
:105EA00007F01CFF0C3800EBD070401080B2089057
:105EB00007F016FF2478A0F10B0507F00FFF640030
:105EC00095FBF6F57443064607F00AFF0121431ED1
:105ED000721E00200091D2B23946DBB201900290CE
:105EE000039007F0B7FB08990898C9B2E4B24008DC
:105EF00001F108035FFA80F9DBB204F1010B5444AD
:105F000009F10408EAB201349944ED190F940B9099
:105F10005FFA88F80C9109935FFA89F90D92EDB256
:105F20000C2410E15C4A0798182303FB002303F5B7
:105F3000026318339B8814211BB293FBF1F3783969
:105F40008B42B8BF0B460899642BA8BF642303FBA0
:105F500001F0C92190FBF1F10B98002B014489B2AB
:105F60000E914FF0010301F104020ADD0093FE33AC
:105F70000193643B0293963B039340462146D2B281
:105F800008E00093FF230193FA3BD0B202930393FE
:105F90002146424604F1020A5FFA8AFA2B4607F0CC
:105FA00059FBFF269B274046214642465346009612
:105FB0000197029707F007FCAB1EDBB219460A9364
:105FC000404642462B4600960197029707F0FBFB9E
:105FD0000E990A9B081DC0B25146024600960197D1
:105FE000029707F0F0FB079B2B484FF0180C0CFBB7
:105FF000030202F502620C321046CDF814C006927C
:1060000007F0BEFCA8EB50005146069A3346C0B2DA
:106010000096019607F0FAFC0C9900230A1D042053
:1060200000932146D2B22B4601960296039607F0C2
:1060300011FB194ADDF814C008980CFB0B2C0CF569
:10604000026318339B8814221BB293FBF2F3783A55
:106050009342B8BF1346642BA8BF642303FB00F12F
:10606000C92291FBF2F20B9909988A1892B2002B7F
:1060700007924FF00103024410DD009304330196B0
:106080000297039348462146D2B20FE0D001002088
:10609000280B010077030020D00C0020009305237B
:1060A000D0B201960293039321464A462B46FF261F
:1060B00007F0D0FA9B27214648464A4653460197A7
:1060C0000297009607F07FFB2B4648460A994A46FE
:1060D00001970297009607F076FB0999079A0A9BA9
:1060E0008818C0B20246514601970297009607F001
:1060F0006AFB1F4B833F07FB0B3707F502670C3723
:10610000384607F03DFCA9EB500051463A4633466D
:10611000C0B20096019607F079FC0C98002342006B
:1061200008322146009309982B4602F0FE020196A0
:106130000296039607F08EFA0D990BF1020B641884
:106140006D18E4B2EDB20F9A93450CD00BF1FF330A
:106150003F2B07937FF7E6AE05E0064B0120187052
:10616000FF232B7000E0002011B0BDE8F08F00BFCE
:10617000D00C0020900000202DE9F04FAD4C95B0E0
:10618000A4F5125094F80890667AA57AFAF722FAE4
:10619000FAF7B0FB01238DF84930DB188DF84A304F
:1061A00001338DF84B3001338DF84C3001338DF8CD
:1061B0004D30013300278DF84E30013384F80890BC
:1061C0008DF8487066728DF84F30A5729A4C780140
:1061D00020182C309949013708F0EAFF402FF5D1FB
:1061E000403F182000FB074000F502600C30934947
:1061F000013708F0DDFF402FF3D10020342101FBEF
:106200000041FF2301F5A45181F8343001F130023F
:1062100038310B724FF0FE0E9B3B4B72013082F80F
:1062200008E0FD220A714B71643B4028824F8B715C
:10623000E4D187F84A3087F8493087F8482087F852
:106240006A3087F8693087F8682087F88A3087F8DD
:10625000893087F8882087F8AA3087F8A93087F82E
:10626000A82007F510572F3A87F8552087F85720B0
:1062700087F859209C3A87F85B2087F8543001331F
:1062800087F85630013387F85830013387F85A3091
:106290006B4B102D00F25A87DFE815F0110011004A
:1062A00011001100110011001F031F031F035807E5
:1062B0005807FC05FC055807C9068F06C9060022C9
:1062C000691E84F8282010460132042908D8DFE826
:1062D00001F007030303060084F8280002E002220D
:1062E00084F82820574853F8251008F061FFB9F1C9
:1062F000020F17D0B9F1030F1DD0B9F1000F4FF005
:10630000030A0CBF4FF0010C4FF0020C0CBF02202F
:106310000120CDF828A0CDF80CC0089018BF4FF090
:10632000000912E00021012203230A910392CDF813
:10633000209009930BE000274FF0020A4FF0010C68
:106340000A97CDF80CA0CDF820C0CDF8249009997B
:10635000480120183C492C3008F02AFF089A3B4994
:10636000500120182C3008F023FF039B38495801B6
:1063700020182C3008F01CFF0A9F3649780120189D
:106380002C3008F015FF3449344808F011FF9DF80F
:106390004A0033494001201800F5B67008F008FFA4
:1063A0003049314808F004FF3049314808F000FF17
:1063B0003049314808F0FCFE3049314808F0F8FE19
:1063C0003048314908F0F4FE00220123032E6DD835
:1063D000DFE806F0020E205C8DF8493002238DF8CC
:1063E0004A3001338DF84B308DF8482001331CE0E2
:1063F0008DF8483002238DF84930023B8DF84A3041
:1064000003338DF84B3001338DF84C3003338DF866
:106410004D304BE08DF8493003238DF84A30013B75
:106420008DF84B308DF8482002338DF84C30013315
:10643000EDE700BF50310020D00C0020120B01000E
:10644000F8000020E80C0020380B01003D0B010093
:10645000D3060100420B0100480B01007C0D002017
:10646000500B0100740A0100FC0E0020790A0100A3
:106470005C0F0020590B01003C0F00205C0B010059
:10648000BC0E0020DC0E0020630B01008DF84C30A8
:1064900002238DF8493001338DF84D3001338DF8EA
:1064A0004B3001338DF848208DF84A309DF848C0B4
:1064B0004FF0180808FB0CF904EB090000F5026026
:1064C0000C308149CDF82CC008F072FE9DF84900CF
:1064D0007E4908FB00F30D90E01800F502600C30D7
:1064E000069308F065FE9DF84AB0794908FB0B4019
:1064F00000F502600C3008F05BFE9DF84B707549AA
:1065000008FB074000F502600C3008F051FE9DF8D2
:106510004C10714E08FB01FA04EB0A0000F5026012
:106520000C910C306D4908F043FE9DF84D206C49EC
:1065300008FB02FC04EB0C0000F502600C300E922C
:10654000CDF814C008F034FE9DF84E006549109057
:1065500008FB004000F502600C3008F029FE9DF8B1
:106560004F10A14408FB014000F5026011910C306E
:106570005D4908F01DFE06F50E600C305B4908F021
:1065800017FE09F502620020FD214244A2449072E8
:10659000507211720AF50262424490725072117286
:1065A000069B4FF0FE09E31803F50263434498721B
:1065B00058721972DDF814C0644404F5026444444E
:1065C000A07260722172099A06F5A45484F83420EE
:1065D0000B9B06F5A652137064235370DDF830A0B0
:1065E00008F1840882F802A082F8038084F83890C9
:1065F00084F83C1084F83E8084F83D30DDF820C0FB
:10660000012D82F828C00D9C82F8344082F8353084
:10661000DDF838A006F5A95482F836A082F83730A4
:1066200082F82C9082F8301082F8328082F8313073
:10663000DDF828C006F5A85282F81CC082F8287040
:1066400082F8293084F8009082F8241082F826809D
:1066500082F82530039A06F5AA5C02F1020A06F5D3
:10666000AC5406F5AE5243D84FEA4A1A56440125B7
:10667000B57104258CF81050109E8CF81C608CF8B5
:106680001D308CF814908CF818108CF81A808CF847
:106690001930039F277184F810B0637484F8089050
:1066A000217384F83850DDF82CA082F804A05371CF
:1066B000DDF830C082F806C0D37184F83C901170C8
:1066C00090705370C9E000BF690B0100700B0100AE
:1066D000D3060100420B0100D00C0020770B010013
:1066E0007E0B0100480B01005C0B0100630B0100F5
:1066F0004FEA4A1A06EB0A074FF0010A87F806A08C
:106700000F97039F4FF00E0A8CF810708CF81CB096
:106710008CF81D308CF814908CF818108CF81A80B6
:106720008CF8193084F804A0DDF844C084F810C057
:10673000637484F80890217384F80E80637384F87E
:106740003870082717710737537184F83C7011703F
:1067500082F8028053700F9FFF243C720BF10A07EE
:1067600006F50654BC4606F5075784F834B084F89D
:10677000389084F83C1084F83E0084F83D3087F867
:1067800000C04B2784F842304FF0EC0984F8417088
:1067900006F50B5C06F50A5484F834B084F838A08A
:1067A00084F8399084F83A8084F83C1084F83E00EC
:1067B00084F83D808CF800104FF0140C84F84200EF
:1067C000042D84F8413084F844B084F848A084F85B
:1067D00049C00CF1A60C84F84A9084F84C1084F857
:1067E0004E0084F84DC084F8501084F8520084F8AC
:1067F000513032D1122482F83040099D82F82C5059
:10680000DDF834A082F838A082F839700E9D82F845
:106810003A50B52582F83B5082F8341082F83600A1
:1068200082F8353006F5B05282F82440DDF820A019
:1068300006F5B15686F800A0DDF82CC082F82CC011
:1068400082F82D700C9D82F82E5082F82F7082F8FD
:10685000281082F82A0082F82930864A099EFD21F4
:1068600000242D20102582F8346082F8385082F8F8
:106870003C1082F83E4082F83D00089F134603F822
:10688000407F1D7119729C725872DDF828A083F840
:106890000CA01D7419759C7558751334053082F859
:1068A000F46082F8F84082F8FC1082F8FE0019309B
:1068B00082F8FD0002F5807382F8007182F80441CD
:1068C00082F8081114229A72587283F80CA01C7472
:1068D00019759A75587500F077BC042284F8282041
:1068E000654853F8251008F063FCB9F1020F14D085
:1068F000B9F1030F18D0B9F1000F4FF0030CCDF828
:1069000020C00CBF012702270CBF4FF002084FF038
:10691000010818BF4FF000090BE00020C84608909E
:1069200001274FF0030904E00021089102274FF0EE
:1069300001084FEA491020182C30504908F038FC63
:106940004FEA481020182C304D4908F031FC7801EE
:1069500020182C304B4908F02BFC089A4A4950016A
:1069600020182C3008F024FC4849494808F020FC45
:106970004849494808F01CFC4849494808F018FCB7
:106980004849494808F014FC4849494808F010FCB7
:106990004849494808F00CFC09F102035B01E3187F
:1069A000187A4649400120182C3008F001FC08F103
:1069B00002035B01E318187A4149400120182C308A
:1069C00008F0F6FBBB1C5B01E318187A3D49400157
:1069D00020182C3008F0ECFBDDF820A03A490AF131
:1069E00002035B01E318187A4FF0000A40012018F7
:1069F0002C3008F0DDFB84F8E0A0344984F8DEA0F8
:106A0000334808F0D5FB84F800A1324984F8FEA091
:106A1000314808F0CDFB84F820A1304984F81EA14C
:106A20002F4808F0C5FB84F840A12E4884F83EA109
:106A30002D4908F0BDFB0523032E65D8DFE806F0DD
:106A400056020C5601228DF8493002238DF84A3047
:106A50008DF848209B1808E08DF8483001238DF808
:106A60004930DB188DF84A3001338DF84B30033B49
:106A700048E000BF901E0020E80C0020850B0100BC
:106A80008A0B01008F0B0100420B0100740A010008
:106A9000FC0E0020790A0100DC0E0020590B0100D9
:106AA0003C0F00205C0B0100BC0E0020950B010088
:106AB0005C0F00209A0B01007C0D0020A50B01004B
:106AC000AF0B0100B90B0100C40B0100D00B01009A
:106AD0009C0D0020DF0B0100BC0D0020EE0B01001F
:106AE000DC0D0020FC0D0020F90B010001238DF8C6
:106AF0004930DB188DF84A3001338DF84B308DF872
:106B000048A001338DF84C309DF848A04FF0180B89
:106B10000BFB0A4C0CF5026C0CF10C0C6046D249D4
:106B2000CDF814C008F044FB9DF84920CF490BFB79
:106B300002F0231803F502630C330B9018460792FA
:106B4000099308F035FB9DF84A10C94E0BFB01F381
:106B5000E01800F502600A910C30C6490C9308F069
:106B600027FB9DF84B00C4490BFB00F00D9020184B
:106B700000F502600C3008F01BFB9DF84C30BF495B
:106B80000BFB03FB04EB0B0000F502600C3008F07C
:106B90000FFB06F50A600430B94908F009FB062D21
:106BA00006F5A45306F5A65406F5A855079ADDF890
:106BB00014C057D1B81C4001012130188171DDF893
:106BC00030C006EB0C0080F83E18DDF82CC006EB58
:106BD0000C0080F83E18DDF834C006EB0C005E4473
:106BE00080F83E1886F83E18563183F8349084F8C1
:106BF00000A061705231A2704FF0FE0CE170FD26D2
:106C00004539002083F838C083F83C6083F83E00A3
:106C100083F83D10CE2384F8288084F834A084F8CB
:106C2000353084F8362084F837300A9B84F83830C1
:106C300084F8391084F82CC084F8306084F832006D
:106C400084F831102F7785F828A085F8291085F869
:106C50002A2085F82B1085F82C3085F82D1085F822
:106C600020C034E0604687490792069308F0A0FAF6
:106C70008549099808F09CFA069B64214FF0FE0CA8
:106C8000FD26002083F8349084F800A0617083F81A
:106C900038C083F83C6083F83E0083F83D1084F8E8
:106CA00028800A9B84F8343084F8351084F82CC08E
:106CB00084F8306084F8320084F831102F77079A16
:106CC00085F82820714A85F8291082F800C0704A9A
:106CD00085F8246085F8260085F8251017749DF83E
:106CE0004BC06421FE26082382F81CC0517716751C
:106CF0001376DA339376C43B537682F844709DF86A
:106D00004C70FD20002582F8507082F8511082F8F6
:106D1000486082F84C0082F84E5082F84D10DDF841
:106D200020A0042402F5546382F878A082F884C07D
:106D300082F885104FF0130C82F87C6082F8800096
:106D400082F8825082F8811082F8AC40013482F8D7
:106D5000B84082F8B91082F8B06082F8B40082F8C6
:106D6000B65082F8B51083F8347083F838C0ACF1AF
:106D70000C0C83F83CC00CF1210C83F83EC00CF1E4
:106D8000B00C83F83DC04FF00E084FF0140C82F8A1
:106D9000800D83F8425083F8411083F8447083F8E3
:106DA000488083F849C00CF1D80C83F84AC083F8B6
:106DB0004C40013483F84E5083F84D1083F8504016
:106DC000963483F8525083F8514083F8547083F816
:106DD000588083F859C083F85A4083F85C0083F8E0
:106DE0005E5083F85D1083F8600083F8625083F88A
:106DF00061409DF8481002F5446383F83410322155
:106E000083F8386083F83C0083F83E1083F83D1027
:106E100082F8800C83F8421083F841109DF84920D5
:106E200083F8442083F8486083F84C0083F84E10C0
:106E300083F84D1083F8500083F8521083F85110F6
:106E40009DF84A2083F8542083F8586083F85C004A
:106E500083F85E1083F85D1083F8600083F8621099
:106E600083F86110B0E100BF070C01000E0C0100B7
:106E7000D00C00208A0B0100420B0100D306010058
:106E80009A0B0100850B01008F0B0100F0210020FF
:106E9000102200200D2253F8251084F82820CC4819
:106EA00008F086F9CB49CC4808F082F9CB49CC48A8
:106EB00008F07EF9CB49CC4808F07AF9CB49CC48A8
:106EC00008F076F9CB49CC4808F072F99DF8488073
:106ED000182505FB084000F50260C8490C3008F091
:106EE00067F99DF84970C64905FB074000F5026047
:106EF0000C3008F05DF99DF84A60C24905FB064078
:106F000000F502600C3008F053F99DF84B90BE4933
:106F100005FB094404F502600C3008F049F9BB494F
:106F2000012381F834300B4603F8407F6422FD24AE
:106F30009C20E6354FF0000C5A709E70DA7083F892
:106F400004905A7181F8385081F83C4081F83EC075
:106F500081F83D2083F828C083F8348083F83520F9
:106F600083F82C5083F8304083F8320083F83120C6
:106F700081F89CC0032381F8A870122781F8A9200A
:106F800081F8AA6081F8AB0081F8A07081F8A44074
:106F900081F8A60081F8A52081F8D0309DF84C300A
:106FA00081F8DC3081F8DD2081F8D45081F8D840B8
:106FB00081F8DA0081F8D92006E1132284F828202C
:106FC000D96B834808F0F4F8002101200A463E29D5
:106FD00026DC342606FB0246642506F5A45300F1A0
:106FE000010C06F5A65683F8342083F8401083F888
:106FF000415083F8420083F8435086F804C000F102
:10700000020C757186F806C0F571FE2683F83860AB
:10701000013E83F83C60FD3E83F83E6083F83D50BE
:10702000013204300431402AC0B2D0D1CCE0132266
:1070300084F82820664853F8251008F0B9F800268F
:10704000770104EB070909F12C097149484608F05A
:10705000AFF8484608F00AF9C0190022711C201840
:107060002C3013464FF0010909B2E719CDF8009012
:10707000F9F73CFE002387F840303837102D5FFACF
:1070800086F803D104337B7287F80A90B8F10F0FAA
:1070900021D80C2303FB0643FF2003F58E5282F810
:1070A0003480FD2182F83800FF3882F83C1082F8E5
:1070B0003E002D3082F83D0003F594533222D1304A
:1070C00083F8348083F8380083F83C1083F83E203E
:1070D000921883F83D200136402EB1D1002334228E
:1070E00002FB034202F5A45282F83430642182F894
:1070F0004030FE25013382F84110FD2082F83850DF
:10710000FE3D402B82F83C0082F83E5082F83D1054
:10711000E5D118276F43E61906F502660C363D499E
:10712000304608F045F8304608F0A0F8C01920189D
:1071300001230022013500F5026000930C3029B2D2
:107140001346F9F7D3FD402DE3D13DE0052253F876
:10715000251084F828201E4808F02AF81D491E48EA
:1071600008F026F81D491E4808F022F81D491E485F
:1071700008F01EF81E48284908F01AF80D2D05D110
:107180001023FB73093B7B73073BBB730023342243
:1071900002FB0342FE2002F5A452FD2582F83430A2
:1071A00082F8380082F83C50613D82F83E50383D0C
:1071B00082F83D5082F84030013302F13001102B4B
:1071C00082F841500872E2D1012015B0BDE8F08F7D
:1071D000E80C0020150C0100FC0C00201D0C010027
:1071E0001C0D0020260C01003C0D00202A0C010083
:1071F0005C0D0020340C01003C0F00203D0C010010
:10720000430C01004A0C0100510C010050210020E8
:10721000580C0100610C0100680C01002DE9F041DF
:10722000344D86B06B780646FF2B2C4654D12A4647
:107230006B1C08461121FBF78FF82F4D2378294648
:107240000DF11702304600931123FBF791FD06F074
:1072500047FD2A4B804693F84A7006F03FFD0646EC
:1072600006F03EFDC7EB080701220346009200200E
:107270003246F9B20190029003900A2606F016F900
:107280002D7823E021783046C5EB010CDCF10001BC
:1072900041EB0C01FBF708F8102D13D8154B3046C5
:1072A0001A78174BC5EB020EDEF1000253F82510D9
:1072B00042EB0E02FAF7E6FD124B30465957FF2219
:1072C000FAF742FE0A360135F6B2EDB29DF81730F4
:1072D000AB42D7D8002009E0137010460121FAF71D
:1072E00019F9094B01201870FF236B7006B0BDE837
:1072F000F08100BFA9000020BD0300205031002014
:10730000F800002038090100900000202DE9F0412C
:107310002F4D86B06B780646FF2B2C464AD12A4665
:107320006B1C08460421FBF717F82A4D23782946E1
:107330000DF11702304600930423FBF719FD06F008
:10734000CFFC254B804693F84A7006F0C7FC0646F2
:1073500006F0C6FCC7EB0807012203460092002096
:107360003246F9B20190029003900A2606F09EF888
:107370002D7819E0217830464A1B514241EB020139
:10738000FAF792FF032D0BD8114B30461A78134BA6
:1073900053F82510531B5A4242EB0302FAF772FDD1
:1073A0000A360135F6B2EDB29DF81730AB42E1D89E
:1073B000002009E0137010460121FAF7ABF8084BE2
:1073C00001201870FF236B7006B0BDE8F08100BF8C
:1073D000320000207903002050310020AC00002052
:1073E000900000202DE9F041314D86B06B780646C3
:1073F000FF2B2C464ED12A466B1C08460421FAF777
:10740000ABFF2C4D237829460DF11702304600932F
:107410000423FBF7ADFC06F063FC274B804693F892
:107420004A7006F05BFC064606F05AFCC7EB0807FC
:1074300001220346009200203246F9B201900290E8
:1074400003900A2606F032F82D781DE021783046A8
:10745000C5EB010CDCF1000141EB0C01FAF724FF54
:10746000032D0DD8124B30461A78144BC5EB020E83
:10747000DEF1000253F8251042EB0E02FAF702FD8E
:107480000A360135F6B2EDB29DF81730AB42DDD8C1
:10749000002009E0137010460121FAF73BF8084B71
:1074A00001201870FF236B7006B0BDE8F08100BFAB
:1074B0003C010020AD0300205031002014000020CA
:1074C000900000202DE9F0412F4D86B06B780646E4
:1074D000FF2B2C464AD12A466B1C08460521FAF799
:1074E0003BFF2A4D237829460DF1170230460093C1
:1074F0000523FBF73DFC06F0F3FB254B804693F894
:107500004A7006F0EBFB064606F0EAFBC7EB0807FD
:1075100001220346009200203246F9B20190029007
:1075200003900A2605F0C2FF2D7819E02178304635
:107530004A1B514241EB0201FAF7B6FE042D0BD86B
:10754000114B30461A78134B53F82510531B5A42EF
:1075500042EB0302FAF796FC0A360135F6B2EDB2B9
:107560009DF81730AB42E1D8002009E013701046B7
:107570000121F9F7CFFF084B01201870FF236B7032
:1075800006B0BDE8F08100BF910000209B03002001
:107590005031002094000020900000202DE9F04F91
:1075A000814C89B094F859800546B8F1FF0F164612
:1075B00040F0C680084604F15802052104F1590341
:1075C000FAF7CAFE94F8583078490DF11F022846A0
:1075D00000930523FBF7CCFB06F082FB744F81463A
:1075E00097F84A5006F07AFB824606F079FBC5EB25
:1075F0000901002503464FF001092846C9B2524649
:10760000CDF8009001950295039505F04FFF97F88E
:107610004A30002B3FD006F063FB97F84A30834690
:10762000059306F05BFB824606F05AFB059B0AF1C8
:10763000FF32DB439B44431E5FFA8BF1D2B22846F4
:10764000DBB2CDF8009001950295039505F02EFF71
:10765000584D94F8583055F82300F9F7B5FF814696
:1076600006F03EFB544B97F84A201B7897F84A10D7
:10767000CDF80080CB1A03EBD373C2EB630194F80F
:1076800058304118CDF8048055F823204846C9B237
:10769000434606F0DBF9454B0A251F784BE094F88A
:1076A00058102846C7EB010CDCF1000141EB0C013E
:1076B000FAF7FAFD042F3AD83B4B284693F85820A6
:1076C0003E4BC7EB020EDEF1000253F8271042EBEF
:1076D0000E02FAF7D7FB7B1E032B28D8DFE803F056
:1076E000020B141D317894F85820354B284653F876
:1076F0002110012A16E0717894F85820314B284661
:1077000053F82110022A0DE0B17894F858202E4B3E
:10771000284653F82110032A04E094F858202B49F6
:107720002846042A14BF00220122FAF7CDFB0A35AD
:107730000137EDB2FFB29DF81F30BB42AFD82EE04B
:10774000B8F1040F2BD8DFE808F01A03091017006E
:107750001A4B5868FF23FFF7D9FD17E0174B01328A
:107760009868FF23FFF73EFE10E0144B0232D86802
:10777000FF23FFF753FD09E00846FEF7FDFC144B1D
:1077800001201870FF2384F8593009E0012806D140
:107790000F4B1870FF2384F85930013800E00020A7
:1077A00009B0BDE8F08F00BF420100207D0300203A
:1077B0005031002034000020F40000207C00002024
:1077C000AC00002014000020F8000020D10D0100C2
:1077D00090000020F0B585B09DF828C0C1EB030EE5
:1077E0001FFA8EFE0CFB0EFCDCB26FF063039CFBF9
:1077F000F3FCCEB2E6446533C7B2D5B206EB0E0158
:1078000000937F3301930293039338462A4623461D
:10781000C9B205F01FFF00230A93FF330B930C93AB
:107820000D93384631462A46234605B0BDE8F04060
:1078300005F010BF2DE9F04788B00E4606F04EFA6D
:10784000044606F04DFA0121A21F831F0091032078
:107850000139FF2402910391D2B20146DBB20194B7
:1078600005F0F8FE052001468E4A23460094019457
:1078700006F0ECF8012E05D18B4B1A78022A08D8B5
:10788000013205E0022E04D1874B1A780AB1013A81
:107890001A70864D2B78CBB91A4602F5926184484E
:1078A000013100EBC1010020C8804FF61000888034
:1078B0004FF4FE6008817F490020C8527E490132A2
:1078C000C8520233042AE8D1012358E0012B58D1D1
:1078D000FF247A48F9F778FE23460F21774A00946F
:1078E000019406F0B3F87648F9F76EFE23461921A5
:1078F000734A0094019406F0A9F87248F9F764FEFF
:10790000234623216F4A0094019406F09FF86E4F9E
:10791000FF3C204606F078FC0134E4B2042C27F842
:10792000020FF6D1604B634C1B78002234F9131020
:107930000123009305A81346F9F7D8F905A8F9F72C
:1079400043FEFF232D2105AA0093019306F07EF844
:10795000032E40F0A3805D49002303F59262544E4C
:107960002088013206EBC2020133D0800022042BB2
:1079700024F8022B21F8022FEFD12B7801332B7042
:107980008CE0022B40F08A80FF244C48F9F71CFE63
:1079900023460F21494A0094019406F057F84C48B9
:1079A000F9F712FE23461921494A0094019406F082
:1079B0004DF84448F9F708FE23462321414A009434
:1079C000019406F043F84348F9F7FEFD23462D21C4
:1079D000404A0094019406F039F8364F364C4FF087
:1079E0000008BA46A146404606F00EFC37F9023BB5
:1079F00008F10108984234F9023BB8BF27F8020C9D
:107A00005FFA88F89842C8BF24F8020CB8F1040F56
:107A1000E9D1254F00223B78FF243AF91310A8F151
:107A20000308134605A8CDF80080F9F75FF9372160
:107A30000A2005AA23460094019406F007F83B7833
:107A4000002239F9131005A81346CDF80080F9F784
:107A50004DF96420372105AA23460094019405F0CE
:107A6000F5FF032E1AD118481849002303F5926236
:107A70000F4C013204EBC202D48830F8026F01339C
:107A8000341B9480D48831F8026F042BC4EB0604B5
:107A90001481EBD1043B2B70012000E0002008B0E2
:107AA000BDE8F087831501008303002070030020E8
:107AB000D00C00208E030020B4030020710C0100C4
:107AC000780C01007F0C01008C030020B203002021
:107AD000860C01008B0C01002DE9F04F002387B0CC
:107AE00080460127924A590151183831097A924645
:107AF00009B90137FFB20133402BF3D1012F00F058
:107B000011818C4B5C781D46FF2C40F0D1801A46C9
:107B1000394601334046FAF71FFC2B78864E009316
:107B200086483B4686490DF11702FBF721F996F886
:107B30004A30002B35D006F0D3F896F84AB081468B
:107B400006F0CCF8804606F0CBF86FEA0B0B08F194
:107B5000FF32431E0121D9440020D2B2DBB2009192
:107B60005FFA89F101900290039005F09FFC75483F
:107B7000F9F72AFD804606F0B3F8734B96F84A20D1
:107B80001B7896F84A100094CB1A03EBD373C2EB20
:107B900063014118C9B240466A4A2346019405F080
:107BA00055FF674B0A261C787CE0297830460B1B72
:107BB000594241EB0301FAF777FBBC426ED254B94C
:107BC0005C4B30461A786149D2F1010238BF00227D
:107BD000FAF758F924E04FF00008C1464FEA48137D
:107BE0000AEB03023832127AA2B9621E4A450DD15D
:107BF0004F4A3046D3182A7803F12C01C4EB020C0B
:107C0000DCF1000242EB0C02FAF73CF909F1010940
:107C10005FFA89F908F10108B8F1400FDED14CB9DB
:107C20002A783046D2F10102494938BF0022FAF7DA
:107C30004BF933E04FF00008C1464FEA4813534474
:107C400038331A7A2ABB611E49451ED1597A012957
:107C500011D193F806E02B784FFA8EFE63319EFB2C
:107C6000F1F1C4EB030EDEF10003304643EB0E03EB
:107C7000FAF78CF909E02A789979131B5A423046B1
:107C800049B242EB0302FAF727FA09F101095FFA58
:107C900089F908F10108B8F1400FCED10A36013454
:107CA000F6B2E4B29DF81730A3423FF67EAF3BE058
:107CB0002CB9284A01201070FF225A7035E00024A8
:107CC0002646204662010AEB02033833197AF1B9DD
:107CD0006F78013FB74218D1587A01280DD19A79AF
:107CE00012B964329A7100E09971600150443E30DB
:107CF0000121F9F70FFC012007E00D4B16489A18F7
:107D000041463E32FF23FAF785FE0136F6B20134D2
:107D1000402CD7D1012807D10E4B1870FF236B7070
:107D2000013802E0384600E0002007B0BDE8F08FDF
:107D3000D00C00202800002050310020920C0100BF
:107D40007C0300205F0C0100F4000020E809010022
:107D5000D10D010090000020FA0A01002DE9F04346
:107D6000374C0025637887B0FF2B07468DF81750F6
:107D700055D1084622460621631CFAF7EDFA314E2A
:107D8000237831460DF11702384600930623FAF79F
:107D9000EFFF05F0A5FF2C4B814693F84A8005F0D4
:107DA0009DFF074605F09CFFC8EB0908012203462A
:107DB000009228465FFA88F13A46019502950395AC
:107DC00005F074FB35780A2623E021783046C5EBB0
:107DD000010CDCF1000141EB0C01FAF765FA052D0D
:107DE00013D8174B30461A78184BC5EB020EDEF14C
:107DF000000253F8251042EB0E02FAF743F8144B39
:107E000030465957FF22FAF79FF80A360135F6B285
:107E1000EDB29DF81730AB42D7D8002007E04BB148
:107E2000013B137010460121F9F774FB02E007B023
:107E3000BDE8F083074B01201870FF236370F6E75D
:107E400040010020B203002050310020B801002082
:107E5000E01D0100900000202DE9F0435A4E87B04C
:107E600074783546FF2C40F094803246731C4021D4
:107E7000FAF772FA3378554E009355484023554926
:107E80000DF11702FAF774FF96F84A30002B34D040
:107E900005F026FF96F84A90804605F01FFF07463A
:107EA00005F01EFF6FEA09097A1E431E0121C8442E
:107EB0000020D2B2DBB200915FFA88F1019002900B
:107EC000039005F0F3FA4448F9F77EFB074605F006
:107ED00007FF424B96F84A201B7896F84A10009408
:107EE000CB1A03EBD373C2EB63014118C9B2384616
:107EF000394A2346019405F0A9FD364B0A261C7821
:107F000042E029783046C4EB010CDCF1000141EB82
:107F10000C01FAF7C9F93F2C2B4F31D884B93A78C4
:107F20003046D2F1010238BF00222D49F9F7AAFFED
:107F30002A783046D2F101022A4938BF00221DE0DA
:107F40003A78DFF8B0806101C4EB020E41440C3195
:107F5000DEF1000242EB0E023046F9F793FF631C9C
:107F60005B0143449B793A78012BC4EB02030CBFBD
:107F70001D491E495A42304642EB0302F9F7A4FF5D
:107F80000A360134F6B2E4B29DF81730A342B8D8ED
:107F900016E0174D24B90120FF232870737010E0FC
:107FA000013414486401001983790121C3F10103EC
:107FB00000F8063FF9F7AEFA01232B70FE33737019
:107FC000002007B0BDE8F0832C00002050310020D5
:107FD000A10C0100B10300205F0C0100F40000209F
:107FE000E8090100D10D0100140F0100FC09010096
:107FF00090000020D00C00202DE9F043614E87B0A6
:1080000074783546FF2C40F09C803246731C40212A
:10801000FAF7A2F933785C4E00935C4840235C4940
:108020000DF11702FAF7A4FE96F84A30002B34D06F
:1080300005F056FE96F84A90804605F04FFE07463A
:1080400005F04EFE6FEA09097A1E431E0121C8445D
:108050000020D2B2DBB200915FFA88F10190029069
:10806000039005F023FA4B48F9F7AEFA074605F0FE
:1080700037FE494B96F84A201B7896F84A10009430
:10808000CB1A03EBD373C2EB63014118C9B2384674
:10809000404A2346019405F0D9FC3D4B0A261C7842
:1080A0004AE029783046C4EB010CDCF1000141EBD9
:1080B0000C01FAF7F9F83F2C324F39D884B93A78E5
:1080C0003046D2F1010238BF00223449F9F7DAFE16
:1080D0002A783046D2F10102314938BF002225E02A
:1080E000631E4FF0180808FB03F8DFF8C4903A78D5
:1080F00009EB0801C4EB020E01F502610C31DEF15F
:10810000000242EB0E023046C844F9F7BBFE08F508
:10811000026318339B793A78012BC4EB02030CBF3E
:10812000204921495A42304642EB0302F9F7CCFE7E
:108130000A360134F6B2E4B29DF81730A342B0D843
:108140001CE01A4D24B90120FF232870737016E03B
:108150001823013C5C4316480121031993F83E287B
:108160000019C2F1010200F5026083F83E281E30BA
:10817000F9F7D0F901232B70FE337370002007B09C
:10818000BDE8F0832400002050310020B00C010035
:108190009A0300205F0C0100F4000020E8090100B0
:1081A000D10D0100140F0100FC0901009000002016
:1081B000D00C00202DE9F047794C86B0667B07464D
:1081C000FF2E154640F0B580084604F10C02072149
:1081D00004F10D03FAF7C0F8237B3846714F009382
:1081E000714907230DF11702FAF7C2FD97F84A30DB
:1081F000002B3BD005F074FD97F84AA0814605F0AE
:108200006DFD804605F06CFD6FEA0A0AD14408F165
:10821000FF32431E01210020D2B20091DBB25FFA8F
:1082200089F1019002900390DFF8A48105F03EF9F6
:10823000237B58F82300F9F7C7F9814605F050FD74
:108240005A4B97F84A201B7897F84A100096CB1A99
:1082500003EBD373C2EB6301237B411858F823204F
:108260004846C9B23346019605F0F0FB4E4B0A264C
:108270001F7859E0217B3046C7EB010CDCF100018F
:1082800041EB0C01FAF710F8062FDFF8148147D8FC
:1082900098F80C20464BC7EB020EDEF1000242EBD1
:1082A0000E02304653F82710F9F7ECFD57B998F84D
:1082B00064203D21D2F10102304638BF0022F9F797
:1082C00043FE2DE0BB1E042B04D8DFE803F00E14A0
:1082D0001A202900227B3046A2F101035A42294686
:1082E00042EB0302F9F7F0FD1AE0227B3046B5F9C4
:1082F0001010022A0FE0227B3046B5F91210032A33
:1083000009E0227B3046B5F91410042A03E0227BF1
:10831000A97D3046052A14BF00220122F9F700FE8C
:108320000A360137F6B2FFB29DF81730BB42A1D82A
:1083300031E0062E2FD8DFE806F0040A0F12151BD5
:1083400021001C4B01201870FF23637324E0FF23DE
:108350001948F9F7C9FB16E01848103204E018482C
:10836000123201E017481432FF23F9F781FB0AE0CB
:108370001632FF231448F9F756F904E0134818326F
:10838000FF23FAF795FA012805D10A4B1870FF234D
:108390006373013800E0002006B0BDE8F08700BF3D
:1083A000420100205031002089030020F400002009
:1083B0005C1D01009000002011180100FA0A010064
:1083C000DB0B0100BA0F0100EE0E01008B0E010065
:1083D0006C0901002DE9FF479246394A0746D37BD5
:1083E0001446FF2B52D108460E32212104F10F030F
:1083F000F9F7B2FF334EA37B3146009305460DF1EA
:108400000F0238462123FAF7B3FC0A27367838E002
:10841000A17B3846C6EB010CDCF1000141EB0C01FD
:10842000DFF89C80F9F740FF4EB998F80E103846F7
:10843000D1F1010138BF0021F9F778FF1DE0202EAE
:108440001BD8731E4FF01C0909FB03A998F80E20D6
:108450003846C6EB020EDEF1000242EB0E02494640
:10846000F9F710FD98F80E203846931B5A42B9F9D7
:10847000101042EB0302F9F753FD0A370136FFB241
:10848000F6B29DF80F30B342C2D80EE02BB90E4BB6
:1084900001201870FF23D3730EE0013B1C2202FB66
:1084A00003A2DBB2FFF786FE0546012D03D1064B82
:1084B0001D70FF23E373002004B0BDE8F08700BF08
:1084C0004201002069030020900000202DE9F047C0
:1084D000854C86B0667E0746FF2E154640F0CB8061
:1084E000084604F11802072104F11903F9F734FFD3
:1084F000237E38467D4F00937D4907230DF11702F7
:10850000FAF736FC97F84A30002B3BD005F0E8FB31
:1085100097F84AA0814605F0E1FB804605F0E0FBB4
:108520006FEA0A0AD14408F1FF32431E01210020FC
:10853000D2B20091DBB25FFA89F101900290039010
:10854000DFF8DC8104F0B2FF237E58F82300F9F74E
:108550003BF8814605F0C4FB664B97F84A201B7830
:1085600097F84A100096CB1A03EBD373C2EB630162
:10857000237E411858F823204846C9B23346019655
:1085800005F064FA5A4B0A261F786FE0217E3046C8
:10859000CA1B514241EB0201F9F786FE062FDFF8B4
:1085A00048815FD898F81820534B304653F827106D
:1085B000D31B5A4242EB0302F9F764FC57B998F80F
:1085C00064203D21D2F10102304638BF0022F9F784
:1085D000BBFC47E0BB1E042B04D8DFE803F0081DFA
:1085E00027333900227E30462978012A18E069783D
:1085F0003F2903D9227E3046404904E0404B4901DF
:10860000227E3046C918A2F1020CDCF1000242EBD6
:108610000C02F9F759FC25E0227EA9783046032A9E
:1086200014BF00220122F9F77BFC1BE0227E291DEA
:10863000A2F1040EDEF10002304642EB0E02F9F721
:10864000C5FD0FE0227E304605F10801052A04E051
:10865000227E304605F10C01062A14BF00220122B9
:10866000F9F774FD0A360137F6B2FFB29DF81730FC
:10867000BB428BD834E0062E32D8DFE806F0040A7D
:108680000F151B2124001F4B01201870FF23637658
:1086900027E0FF231C48F8F7C6FF19E00132FF234B
:1086A0001A48FCF781FE13E00232FF231848FAF75C
:1086B0004FF90DE00432FF231648FDF7EFF807E00D
:1086C0001548083201E015480C32FF23FCF794FFEF
:1086D000012805D10B4B1870FF236376013800E0A9
:1086E000002006B0BDE8F087420100205031002094
:1086F00084030020F40000203C080100120B01005C
:10870000FC0C002090000020EE0E0100280E01005D
:10871000D90C0100E90C0100F20C01002F0A010044
:10872000081E01002DE9F04790465E4A1F46D37EA1
:1087300086B0FF2B0546164640F08C8008461A325C
:10874000112106F11B03F9F707FE574CB37E2146B2
:10875000009381460DF1170228461123FAF708FB12
:108760000A25247871E0B17E28460A1B514241EB6C
:108770000201F9F799FD4CB94A4B2846997ED1F18F
:10878000010138BF0021F9F7D1FD5AE0102C58D86B
:10879000631E4FF0140A0AFB038A9AF80130BB42A9
:1087A00015D105F09BFA414B6FF003021B780021B5
:1087B000D21A821805F109030091FF31019102914B
:1087C000039102202946D2B2DBB204F06FFE9AF880
:1087D00001103F2914D9B27E2846131B5A4242EB9E
:1087E00003023349F9F74EFBB27E2846C4EB020C74
:1087F000DCF100022F4942EB0C02F9F765FB20E0A7
:10880000B27E2D4BC4EB020E4901DEF1000242EBB9
:108810000E02C9182846F9F735FB05F05FFA234B1D
:108820006FF003021B78611ED21A82180A206B1C9B
:10883000009003380190D2B2C8B2DBB2FF21FBF73F
:108840007DFB0A350134EDB2E4B29DF81730A34246
:1088500089D81AE02BB9194B01201870FF23D37661
:108860001CE0FF2F07D01422013B02FB03835A7840
:10887000FF2A08BF5F70F37E1422013B02FB0382D4
:108880002846DBB2FFF722FE8146B9F1010F04D181
:108890000A4B83F80090FF23F376002006B0BDE872
:1088A000F08700BF42010020850300203000002037
:1088B000120B0100F50C0100FC0C002090000020C0
:1088C0002DE9F0477B4C86B0667F0746FF2E1546A4
:1088D00040F0C080084604F11C02052104F11D038C
:1088E000F9F73AFD237F3846734F00937349052308
:1088F0000DF11702FAF73CFA97F84A30002B3BD0FB
:1089000005F0EEF997F84AA0814605F0E7F98046B0
:1089100005F0E6F96FEA0A0AD14408F1FF32431E76
:1089200001210020D2B20091DBB25FFA89F10190FF
:1089300002900390DFF8AC8104F0B8FD237F58F873
:108940002300F8F741FE814605F0CAF95C4B97F821
:108950004A201B7897F84A100096CB1A03EBD37382
:10896000C2EB6301237F411858F823204846C9B25F
:108970003346019605F06AF8504B0A271E7864E0EA
:10898000217F38468B1B594241EB0301F9F78CFCE0
:10899000042EDFF8208154D898F81C20494BC6EBF0
:1089A000020CDCF1000242EB0C02384653F82610B0
:1089B000F9F768FA56B998F864203D21D2F101021E
:1089C000384638BF0022F9F7BFFA3AE0032E98F88C
:1089D0001C2020D0042E29D0022E12D029783F2925
:1089E00002D93846384903E0384B49013846C9189E
:1089F000A2F1010EDEF1000242EB0E02F9F764FA79
:108A00001FE0A2F102035A423846697842EB0302A2
:108A1000F9F786FA15E0A2F1030C291DDCF100023A
:108A2000384642EB0C02F9F7D1FB0AE0A2F1040E42
:108A3000DEF10002384605F1080142EB0E02F9F7BB
:108A400085FB0A370136FFB2F6B29DF81730B34204
:108A500096D82AE0042E28D8DFE806F003090E1481
:108A60001A001B4B01201870FF2363771EE0FF23C1
:108A70001848FCF799FC10E00132FF231648F8F77C
:108A8000D2FD0AE00432FF231448FCF707FF04E09C
:108A900013480832FF23FCF7AFFD012805D10C4B2A
:108AA0001870FF236377013800E0002006B0BDE8AE
:108AB000F08700BF4201002050310020A2030020B7
:108AC000F4000020381C0100120B0100FC0C0020F7
:108AD00090000020280E0100EE0E0100E90C0100BC
:108AE000FC0C0100280801002DE9F04717465E4AFA
:108AF0009846D37F86B0FF2B0546164640F08C8003
:108B000008461E32112106F11F03F9F725FC574CC8
:108B1000B37F2146009381460DF1170228461123A9
:108B2000FAF726F90A25247871E0B17F28460A1B56
:108B3000514241EB0201F9F7B7FB4CB94A4B2846C9
:108B4000997FD1F1010138BF0021F9F7EFFB5AE01D
:108B5000102C58D8631E4FF00C0A0AFB03FA17F8C2
:108B60000A30434515D105F0B9F8414B6FF00302C7
:108B70001B780021D21A821805F109030091FF31F8
:108B800001910291039102202946D2B2DBB204F096
:108B90008DFC17F80A103F2914D9B27F2846131B01
:108BA0005A4242EB03023349F9F76CF9B27F284687
:108BB000C4EB020CDCF100022F4942EB0C02F9F786
:108BC00083F920E0B27F2D4BC4EB020E4901DEF1A8
:108BD000000242EB0E02C9182846F9F753F905F0D6
:108BE0007DF8234B6FF003021B78611ED21A8218A6
:108BF0000A206B1C009003380190D2B2C8B2DBB2DD
:108C0000FF21FBF7FFF80A350134EDB2E4B29DF81D
:108C10001730A34289D81BE02BB9194B01201870DB
:108C2000FF23D3771DE0B8F1FF0F07D00C22013BE3
:108C30005343FA5CFF2A08BF07F80380F37F0C2236
:108C4000013B02FB03722846DBB2FFF739FE814687
:108C5000B9F1010F04D10A4B83F80090FF23F37799
:108C6000002006B0BDE8F0874201002098030020F4
:108C700030000020120B0100050D0100FC0C00204B
:108C8000900000202DE9F047754C86B094F82160E3
:108C90000746FF2E154640F0B980084604F1200231
:108CA000042104F12103F9F757FB94F820303846EA
:108CB0006C4F00936C4904230DF11702FAF758F832
:108CC00097F84A30002B3DD005F00AF897F84AA0F3
:108CD000814605F003F8804605F002F86FEA0A0ABB
:108CE000D14408F1FF32431E01210020D2B200918D
:108CF000DBB25FFA89F1019002900390DFF88C817A
:108D000004F0D4FB94F8203058F82300F8F75CFC0A
:108D1000814604F0E5FF554B97F84A201B7897F8F9
:108D20004A100096CB1A03EBD373C2EB630194F89D
:108D30002030411858F823204846C9B233460196DE
:108D400004F084FE484B0A271E785AE094F820105D
:108D50003846C6EB010CDCF1000141EB0C01F9F7E0
:108D6000A3FA032EDFF8F88047D898F82020404B6C
:108D7000C6EB020EDEF1000242EB0E02384653F85B
:108D80002610F9F77FF856B998F864203D21D2F102
:108D90000102384638BF0022F9F7D6F82DE0022E3E
:108DA00098F8202013D0032E1CD029783F2902D90F
:108DB0003846304903E0304B49013846C918A2F122
:108DC00001035A4242EB0302F9F77EF815E0A2F1E3
:108DD000020C291DDCF10002384642EB0C02F9F7C7
:108DE000F5F90AE0A2F1030EDEF10002384605F1C2
:108DF000080142EB0E02F9F7A9F90A370136FFB272
:108E0000F6B29DF81730B342A0D825E0032E23D840
:108E1000DFE806F002090E14184B01201870FF233A
:108E200084F8213019E0FF231548FCF7BDFA0AE069
:108E30000432FF231348FCF731FD04E012480832E6
:108E4000FF23FCF7D9FB012806D10C4B1870FF2338
:108E500084F82130013800E0002006B0BDE8F0873A
:108E60004201002050310020A8030020F40000201F
:108E7000E0070100120B0100FC0C00209000002014
:108E8000280E0100E90C01000A0D0100E4080100B0
:108E90002DE9F0471746634A984692F8233086B08A
:108EA000FF2B0546164640F09280084622321121DB
:108EB00006F12303F9F750FA5B4C96F8223021466D
:108EC000009381460DF1170228461123F9F750FF50
:108ED0000A25247876E096F8221028460B1B594282
:108EE00041EB0301F9F7E0F954B94E4B284693F8EA
:108EF0002210D1F1010138BF0021F9F717FA5DE026
:108F0000102C5BD8631E4FF00C0A0AFB03FA17F80B
:108F10000A30434515D104F0E1FE444B6FF00302E3
:108F20001B780021D21A821805F109030091FF3144
:108F300001910291039102202946D2B2DBB204F0E2
:108F4000B5FA17F80A103F2918D996F822202846B2
:108F5000C4EB020CDCF1000242EB0C023449F8F7DE
:108F600091FF96F822202846C4EB020EDEF10002A3
:108F7000304942EB0E02F8F7A7FF1FE096F82220D7
:108F80002D4B4901C918131B5A4242EB03022846D4
:108F9000F8F778FF04F0A2FE244B6FF003021B7871
:108FA000611ED21A82180A206B1C009003380190AF
:108FB000D2B2C8B2DBB2FF21FAF77EFE0A35013425
:108FC000EDB2E4B29DF81730A34284D81DE033B966
:108FD0001A4B01201870FF2382F823301FE0B8F1EC
:108FE000FF0F07D00C22013B5343FA5CFF2A08BF56
:108FF00007F8038096F823300C22013B02FB037232
:109000002846DBB2FFF73EFE8146B9F1010F05D1DC
:109010000A4B83F80090FF2386F82330002006B027
:10902000BDE8F087420100207B03002030000020D3
:10903000120B0100100D0100FC0C0020900000201C
:109040002DE9F047A34C86B094F825600746FF2E23
:10905000154640F02C81084604F124020D2104F14C
:109060002503F9F779F994F8243038469A4F00939C
:109070009A490D230DF11702F9F77AFE97F84A3055
:10908000002B3DD004F02CFE97F84AA0814604F056
:1090900025FE804604F024FE6FEA0A0AD14408F156
:1090A000FF32431E01210020D2B20091DBB25FFAF1
:1090B00089F1019002900390DFF83C8204F0F6F908
:1090C00094F8243058F82300F8F77EFA814604F02B
:1090D00007FE834B97F84A201B7897F84A100096B2
:1090E000CB1A03EBD373C2EB630194F8243041181D
:1090F00058F823204846C9B23346019604F0A6FC2E
:10910000764B0A261F78CCE094F824103046CA1B10
:10911000514241EB0201F9F7C7F80C2FDFF8B48197
:1091200000F2BB8098F824206E4B304653F827108D
:10913000D31B5A4242EB0302F8F7A4FE57B998F842
:1091400064203D21D2F10102304638BF0022F8F7F9
:10915000FBFEA2E0BB1E0A2B07D8DFE803F01B28AA
:1091600036484F61687A81939E0029783F2904D957
:1091700094F8242030465C4905E05C4B490194F8A2
:1091800024203046C918012A14BF00220122F8F712
:109190009BFE82E094F82420291DA2F1020CDCF150
:1091A0000002304642EB0C02F9F710F875E094F833
:1091B00024203046A2F1030EDEF1000205F1080181
:1091C00042EB0E02F8F7C2FF67E02B7B3F2B04D97E
:1091D00094F824203046444907E0454A182101FB11
:1091E000032194F8242030460431042ACCE794F873
:1091F0002420304695F90D10052A49E0AB7B3F2B22
:1092000004D994F824203046374907E0384A182119
:1092100001FB032194F8242030460431062AB3E7E9
:1092200094F82420304695F90F10072A30E02B7C63
:109230003F2B04D994F8242030462B4907E02C4AD0
:10924000182101FB032194F8242030460431082A18
:109250009AE794F82420304695F91110092A17E06E
:10926000AB7C3F2B04D994F8242030461E4907E0FC
:109270001F4A182101FB032194F8242030460431B1
:109280000A2A81E794F8242095F9131030460B2A16
:1092900014BF00220122F8F743FE0A360137F6B266
:1092A000FFB29DF81730BB423FF62EAF60E00C2EA8
:1092B0005ED8DFE806F00723252B3134373A3D40EE
:1092C00043494F000B4B01201870FF2384F82530D1
:1092D0004FE000BF4201002050310020AB030020CE
:1092E000F4000020AC070100120B0100FC0C002070
:1092F000F814002090000020081D01001E481FE007
:109300000432FF231D48FCF7C9FA28E00832FF2386
:109310001B48FCF771F922E01A480C3210E01A4899
:109320000D3213E019480E320AE019480F320DE0F1
:109330001848103204E01848113207E0174812327A
:10934000FF23F9F705FB0AE015481332FF23F9F76D
:1093500061FB04E013481432FF23FBF73FFE0128B2
:1093600006D1114B1870FF2384F82530013800E036
:10937000002006B0BDE8F087190D0100E90C0100DE
:10938000240D01002C0D0100390D0100480D0100D4
:10939000550D0100640D0100710D0100800D0100EB
:1093A0008D0D01009C0D0100900000202DE9F04F73
:1093B0001746654A984692F8273087B0FF2B054636
:1093C000164640F0958008462632412106F12703D3
:1093D000F8F7C2FF5D4C96F826302146009381468F
:1093E0000DF1170228464123F9F7C2FC0A2524781B
:1093F00079E096F8261028460B1B594241EB0301F1
:10940000DFF844B1F8F750FF4CB99BF82610284616
:10941000D1F1010138BF0021F8F788FF5FE0402C4F
:109420005DD8631E4FF0340A0AFB03FA17F80A10DE
:109430009BF82620FF2902D1284645490DE0FE2948
:1094400002D12846434908E03F2904D8424B49014C
:109450002846C91801E041492846C4EB020CDCF15A
:10946000000242EB0C02F8F70DFD04F037FCDFF8C8
:10947000F4B06FF001019BF80020631E891A4118B7
:109480000720009096F826006A1CC4EB000EDEF15F
:10949000000040EB0E000190C9B2D8B2D2B20A234C
:1094A000FAF79EF8B8F1FF0F19D017F80A304345C4
:1094B00015D104F013FC9BF800306FF00102D21AB2
:1094C0000021821805F109030091FF3101910291F9
:1094D000039102202946D2B2DBB203F0E7FF0A353E
:1094E0000134EDB2E4B29DF81730A34281D81DE0FB
:1094F00033B91B4B01201870FF2382F827301FE07F
:10950000B8F1FF0F07D03422013B5343FA5CFF2A26
:1095100008BF07F8038096F827303422013B02FB8E
:1095200003722846DBB2FFF78BFD8146B9F1010FCC
:1095300005D10B4B83F80090FF2386F827300020DD
:1095400007B0BDE8F08F00BF420100208203002079
:10955000D50A0100E40A0100FC0C0020120B0100F6
:1095600090000020300000202DE9F04FA24C87B081
:10957000667C8046FF2E15461F4640F02781084630
:1095800004F110020E2104F11103F8F7E5FE237C2B
:109590004046DFF88082009398490E230DF11702B0
:1095A000F9F7E6FB98F84A30002B3BD004F098FB23
:1095B00098F84AB0824604F091FB814604F090FB93
:1095C0006FEA0B0BDA4409F1FF32431E0121002040
:1095D000D2B20091DBB25FFA8AF10190029003905F
:1095E000DFF8349203F062FF237C59F82300F7F789
:1095F000EBFF824604F074FB814B98F84A201B78FD
:1096000098F84A100096CB1A03EBD373C2EB6301B0
:10961000237C411859F823205046C9B2334601969D
:1096200004F014FA754B4FF00B081E78C4E0217C4F
:1096300048468A1B514241EB0201F8F735FE0D2ED8
:10964000DFF8B4A100F2B2809AF810206D4B4846C2
:1096500053F82610931B5A4242EB0302F8F712FC10
:109660004EB99AF864203D21D2F10102484638BF34
:109670000022F8F769FC04F031FB634B6FF0030242
:109680001B78D21A8218731ED2B20C2B00F28E8075
:10969000DFE803F0071319262D39444B525F697335
:1096A0007D00227C4846A2F10109D9F10002294639
:1096B00042EB0902F8F708FC78E0227C484695F96D
:1096C0001210022A24E0227C4846A2F1030CDCF1AD
:1096D000000295F9131042EB0C02F8F735FC65E037
:1096E000237C0222484695F91410042B05E0237CC4
:1096F00095F9151003224846052B14BF00230123BA
:10970000F8F744FC52E0227C95F916104846062AE8
:1097100014BF00220122F8F703FC47E0237C01225A
:10972000484695F91A10072BE7E7237C052248469F
:1097300095F91B10082BE0E7227C4846A2F1090EA0
:10974000DEF1000205F11C0142EB0E02F8F7FEFC0F
:109750002CE00A230093033B0193FF203946434644
:10976000FAF7AAFA22E00A230093033B0193FF20B1
:1097700039464346FAF746FB18E00A230093033BB9
:109780000193FF2039464346FAF7D8FB0EE0072342
:109790000093237C3846A3F10D014B4243EB0103B8
:1097A000019311460A234246F9F7ACFE013608F14F
:1097B0000A08F6B25FFA88F89DF8173008F1FF3909
:1097C000B3425FFA89F93FF632AF6DE00D2E6BD8E8
:1097D000DFE806F0070D24272D30363C42454B517B
:1097E000575D0A4B01201870FF2363745DE0FF236F
:1097F0000748F8F779F94FE042010020970300206D
:10980000F40000206C0701003000002090000020D0
:109810001118010050310020D01C010024481232E0
:1098200010E01332FF232348F8F75EFE34E02248AD
:1098300014320DE01532FF232048FEF78FFA2BE09B
:109840001F481632FF23F9F7E5F825E01D481A32C4
:10985000FF23F7F7E8FE1FE01B481B32F8E71C3236
:10986000FF231A48FBF7C8FE16E0194A3B46194881
:10987000FFF70EFB10E0184A3B461848FFF734F993
:109880000AE0174A3B461748FEF74CFF04E016482B
:10989000164A3B46FFF78AFD012805D1144B187084
:1098A000FF236374013800E0002007B0BDE8F08FAB
:1098B000FA0A010039130100D90D0100EE0E010072
:1098C000E40D0100140F0100EC0D0100F80D010082
:1098D000841F0020790A0100C41E0020740A0100C0
:1098E00044200020820A0100CF0A010084210020C8
:1098F000900000202DE9F04F8DB00992704A054686
:10990000D37C9346FF2B40F0C080084612324121A1
:109910000BF11303F8F720FD6A4C9BF81230079007
:109920000093214628460DF12F024123F9F720FA32
:109930004FF00A082478A2E09BF812104046C4EBCE
:10994000010EDEF1000141EB0E01F8F7ADFC4CB960
:109950005B4A4046917CD1F1010138BF0021F8F704
:10996000E5FC86E0402C00F28480099A04F1FF397E
:109970004FEA4913D3180893514B08999A7C4046F3
:10998000151B6A4242EB0502F8F77CFA04F0A6F9CF
:10999000DFF83CC107279CF80030494A00976FF078
:1099A0000305ED1A937C4519181B434208F1010683
:1099B00043EB00035FFA89F9F6B2EDB22946019351
:1099C00032460A234846CDF818C0F9F79BFD2D1AF8
:1099D000EDB24FF00A0A2A46FF2049463346CDF839
:1099E00000A00197FAF768F92D1AEDB22A46FF2078
:1099F00049463346CDF800A00197FAF703FA2D1A2D
:109A0000EDB22A46FF2049463346CDF800A0019723
:109A1000FAF794FA2A4A0097937C2D1A191B4B42A5
:109A200043EB0103EDB229463246019348465346C3
:109A3000FAF75EFC2D1A04F051F9DDF818C06FF04A
:109A400003039CF80020EDB29B1A1B189D4210D115
:109A5000089A0A3D92F9123064210093EDB21A4837
:109A60000A46002301950296CDF80CA00497F9F759
:109A70005FFF08F10A0801345FFA88F8E4B29DF844
:109A80002F30A3423FF658AF0EE02BB90F4B012009
:109A90001870FF23D37410E0013B099C5A01A218EF
:109AA000DBB2FFF761FD0790079A012A04D1074B4B
:109AB0001A70FF238BF8133000200DB0BDE8F08F33
:109AC000420100207A030020FF0D010090000020D9
:109AD000300000202DE9F0477B4C86B094F82960D7
:109AE0000746FF2E154640F0C080084604F12802C4
:109AF000052104F12903F8F72FFC94F828303846A3
:109B0000724F0093724905230DF11702F9F730F9EE
:109B100097F84A30002B3DD004F0E2F897F84AA0BD
:109B2000814604F0DBF8804604F0DAF86FEA0A0AAE
:109B3000D14408F1FF32431E01210020D2B200912E
:109B4000DBB25FFA89F1019002900390DFF8A881FF
:109B500003F0ACFC94F8283058F82300F7F734FDF4
:109B6000814604F0BDF85B4B97F84A201B7897F8C4
:109B70004A100096CB1A03EBD373C2EB630194F83F
:109B80002830411858F823204846C9B23346019678
:109B900003F05CFF4E4B0A271E7861E094F8281012
:109BA0003846C6EB010CDCF1000141EB0C01F8F783
:109BB0007BFB042EDFF810814ED898F82820464B06
:109BC000C6EB020EDEF1000242EB0E02384653F8FD
:109BD0002610F8F757F956B998F864203D21D2F1CC
:109BE0000102384638BF0022F8F7AEF934E0032E00
:109BF00098F8282022D0042E25D0022E13D02B78BE
:109C00003F2B02D93846354905E03549182000FB7D
:109C1000031138460431A2F101035A4242EB030218
:109C2000F8F752F918E0A2F1020C291DDCF100024C
:109C3000384642EB0C02F8F7C9FA0DE0384605F158
:109C40000801032A03E0384605F10C01042A14BF79
:109C500000220122F8F77AFA0A370136FFB2F6B28B
:109C60009DF81730B34299D829E0042E27D8DFE8B1
:109C700006F0030A0F1518001A4B01201870FF2375
:109C800084F829301CE0FF231748FBF73FFC0DE068
:109C90000432FF231548FBF701FE07E014480832A1
:109CA00001E014480C32FF23FBF7A6FC012806D183
:109CB0000C4B1870FF2384F82930013800E0002095
:109CC00006B0BDE8F08700BF4201002050310020FF
:109CD000BC030020F400002098090100120B0100D1
:109CE000F814002090000020280E0100E90C01006B
:109CF000F20C01002F0A0100140801002DE9F047C1
:109D00001746634A984692F82B3086B0FF2B0546DB
:109D1000164640F0938008462A32112106F12B03A3
:109D2000F8F71AFB5B4C96F82A30214600938146DF
:109D30000DF1170228461123F9F71AF80A2524789D
:109D400077E096F82A1028460B1B594241EB030195
:109D5000F8F7AAFA54B94E4B284693F82A10D1F1D5
:109D6000010138BF0021F8F7E1FA5EE0102C5CD861
:109D700004F1FF3A4FEA0A1A17F80A30434515D1A1
:109D800003F0ACFF444B6FF003021B780021D21AA2
:109D9000821805F109030091FF31019102910391AD
:109DA00002202946D2B2DBB203F080FB17F80A305A
:109DB0003F2B18D996F82A202846C4EB020CDCF178
:109DC000000242EB0C023549F8F75CF896F82A20BD
:109DD0002846C4EB020EDEF10002314942EB0E02CE
:109DE000F8F772F821E02F4A182101FB032196F8B9
:109DF0002A200431131B5A4242EB03022846F8F78B
:109E000041F803F06BFF244B6FF003021B78611ED7
:109E1000D21A82180A206B1C009003380190D2B22B
:109E2000C8B2DBB2FF21FAF72FF90A350134EDB2DF
:109E3000E4B29DF81730A34283D81BE033B91A4B24
:109E400001201870FF2382F82B301DE0B8F1FF0FBE
:109E500006D0013B1B01FA5CFF2A08BF07F803800C
:109E600096F82B302846013B07EB0312DBB2FFF7D5
:109E700031FE8146B9F1010F05D10B4B83F80090FB
:109E8000FF2386F82B30002006B0BDE8F08700BF26
:109E9000420100206B03002030000020120B010063
:109EA000050E0100F8140020900000202DE9F04775
:109EB000794C86B094F82D600746FF2E154640F089
:109EC000BD80084604F12C02052104F12D03F8F7AA
:109ED00043FA94F82C303846704F009370490523AC
:109EE0000DF11702F8F744FF97F84A30002B3DD0E8
:109EF00003F0F6FE97F84AA0814603F0EFFE804695
:109F000003F0EEFE6FEA0A0AD14408F1FF32431E65
:109F100001210020D2B20091DBB25FFA89F10190F9
:109F200002900390DFF8A08103F0C0FA94F82C307F
:109F300058F82300F7F748FB814603F0D1FE594B50
:109F400097F84A201B7897F84A100096CB1A03EB33
:109F5000D373C2EB630194F82C30411858F82320D6
:109F60004846C9B23346019603F070FD4C4B0A27B0
:109F70001E785EE094F82C1038468A1B514241EB63
:109F80000201F8F791F9042EDFF80C814DD898F80A
:109F90002C20454B384653F82610931B5A4242EB6F
:109FA0000302F7F76FFF56B998F864203D21D2F10C
:109FB0000102384638BF0022F7F7C6FF35E0032E0E
:109FC00098F82C2023D0042E26D0022E14D02B78E3
:109FD0003F2B02D93846354905E03549182000FBAA
:109FE000031138460431A2F1010CDCF1000242EB0E
:109FF0000C02F7F769FF18E0A2F1020E291DDEF14D
:10A000000002384642EB0E02F8F7E0F80DE0384661
:10A0100005F10801032A03E0384605F10C01042A82
:10A0200014BF00220122F8F791F80A370136FFB277
:10A03000F6B29DF81730B3429CD829E0042E27D8F9
:10A04000DFE806F0030A0F1518001A4B01201870FC
:10A05000FF2384F82D301CE0FF231748FBF756FA46
:10A060000DE00432FF231548FBF718FC07E0144805
:10A07000083201E013480C32FF23FBF7BDFA012838
:10A0800006D10C4B1870FF2384F82D30013800E006
:10A09000002006B0BDE8F0874201002050310020CA
:10A0A0009D030020F4000020CC1D0100120B0100D4
:10A0B000F814002090000020280E0100E90C010097
:10A0C000F20C01002F0A0100AC0901002DE9F04754
:10A0D0001746634A984692F82F3086B0FF2B054604
:10A0E000164640F0938008462E32112106F12F03C8
:10A0F000F8F732F95B4C96F82E30214600938146F2
:10A100000DF1170228461123F8F732FE0A252478AC
:10A1100077E096F82E1028460A1B514241EB0201C7
:10A12000F8F7C2F854B94E4B284693F82E10D1F1E7
:10A13000010138BF0021F8F7F9F85EE0102C5CD877
:10A1400004F1FF3A4FEA0A1A17F80A30434515D1CD
:10A1500003F0C4FD444B6FF003021B780021D21AB8
:10A16000821805F109030091FF31019102910391D9
:10A1700002202946D2B2DBB203F098F917F80A3070
:10A180003F2B16D996F82E202846131B5A4242EB35
:10A1900003023649F7F776FE96F82E202846C4EBE0
:10A1A000020CDCF10002324942EB0C02F7F78CFEA4
:10A1B00023E0304A182101FB032196F82E200431B8
:10A1C000C4EB020EDEF1000242EB0E022846F7F766
:10A1D00059FE03F083FD244B6FF003021B78611ED0
:10A1E000D21A82180A206B1C009003380190D2B258
:10A1F000C8B2DBB2FF21F9F7E1FF0A350134EDB255
:10A20000E4B29DF81730A34283D81BE033B91A4B50
:10A2100001201870FF2382F82F301DE0B8F1FF0FE6
:10A2200006D0013B1B01FA5CFF2A08BF07F8038038
:10A2300096F82F302846013B07EB0312DBB2FFF7FD
:10A2400035FE8146B9F1010F05D10B4B83F8009023
:10A25000FF2386F82F30002006B0BDE8F08700BF4E
:10A26000420100207603002030000020120B010084
:10A27000090E0100F8140020900000202DE9F04F95
:10A280009C4C87B094F831600746FF2E15469846DF
:10A2900040F0EE80084604F13002082104F1310359
:10A2A000F8F75AF894F830303846934F00939349B2
:10A2B00008230DF11702F8F75BFD97F84A30002BE1
:10A2C0003DD003F00DFD97F84AB0824603F006FD3D
:10A2D000814603F005FD6FEA0B0BDA4409F1FF320A
:10A2E000431E01210020D2B20091DBB25FFA8AF155
:10A2F000019002900390DFF83C9203F0D7F894F8B5
:10A30000303059F82300F7F75FF9824603F0E8FC94
:10A310007B4B97F84A201B7897F84A100096CB1A87
:10A3200003EBD373C2EB630194F83030411859F852
:10A3300023205046C9B23346019603F087FB6F4B8A
:10A340000B271E788AE094F8301048468A1B514249
:10A3500041EB0201F7F7A8FF072EDFF898A179D8A3
:10A360009AF83020674B484653F82610931B5A4200
:10A3700042EB0302F7F786FD4EB99AF864203D21BF
:10A38000D2F10102484638BF0022F7F7DDFD03F0A5
:10A39000A5FC5D4B6FF003021B78D21A8218731E66
:10A3A000D2B2062B56D8DFE803F004111F2734423F
:10A3B0004C0094F830204846A2F10109D9F100027E
:10A3C000294642EB0902F7F77FFD43E094F830207D
:10A3D0004846A2F1020CDCF10002B5F9101042EB84
:10A3E0000C02F7F79DFD35E094F830300122484625
:10A3F00095F91210032B06E094F8303095F91310FC
:10A4000005224846042B14BF00230123F7F7BEFDA5
:10A4100020E094F830204846A2F1050EDEF100025B
:10A4200005F1140142EB0E02F7F790FE12E00A2349
:10A430000093033B0193FF2041463B46F9F724FE7E
:10A4400008E00A230093033B0193FF2041463B466B
:10A45000F9F7B4FE01360A37F6B2FFB29DF81730AD
:10A4600007F1FF39B3425FFA89F93FF66CAF3CE080
:10A47000072E3AD8DFE806F0040B1016191F252B1B
:10A48000224B01201870FF2384F831302EE0FF2387
:10A490001F48F7F729FB1FE01032FF231D48F7F78D
:10A4A000E7FA19E01C48123201E01C481332FF237E
:10A4B000F7F7B9F810E01432FF231948FBF79CF8BE
:10A4C0000AE0184A43461848FFF718FC04E017480A
:10A4D000174A4346FFF7FAFD012806D10B4B1870C7
:10A4E000FF2384F83130013800E0002007B0BDE8D8
:10A4F000F08F00BF4201002050310020AF03002048
:10A50000F4000020F41B0100300000209000002027
:10A5100011180100FA0A0100140F0100EC0D0100EE
:10A52000F80D0100842E0020890A01008D0A010027
:10A53000842F0020580801002DE9F04F8DB00992BA
:10A54000694A054692F833301646FF2B40F0AF803B
:10A5500008463232412106F13303F7F7FDFE634C22
:10A5600096F8323007900093284621460DF12F02CD
:10A570004123F8F7FDFB0A25247892E096F8321083
:10A580002846C4EB010EDEF1000141EB0E01DFF8BD
:10A5900058B1F7F789FE4CB99BF832102846D1F133
:10A5A000010138BF0021F7F7C1FE76E0402C74D8D6
:10A5B000099A04F1FF38182303FB08239BF8322083
:10A5C0001946171B7A4242EB070228460893F7F711
:10A5D00059FC03F083FB464A6FF0030713785FFAD8
:10A5E00088FCFF1AC71905F101085FFA88F8FFB265
:10A5F0004FF00A094FF0070A61463A46FF204346EA
:10A60000CDF818C0CDF80090CDF804A0F9F73CFDC6
:10A61000DDF818C03F1AFFB261463A46FF204346B4
:10A62000CDF80090CDF804A0F9F7C8FD9BF83230C2
:10A63000DDF818C0191B4B42C0EB070743EB0103C1
:10A64000FFB239464246019360464B46CDF800A022
:10A65000F8F7A8FF3F1A03F041FB254BFFB21A7829
:10A660006FF003039B1A1B189F4216D1089B0A3FE9
:10A67000B3F91020142392FBF3F35BB2642100932F
:10A68000FFB21C480A4600230197CDF80880CDF898
:10A690000C90CDF810A0F9F74BF90A350134EDB262
:10A6A000E4B29DF82F30A3423FF668AF10E033B913
:10A6B000114B01201870FF2382F8333011E0099C00
:10A6C000013B182202FB0342DBB2FFF7D7FD0790E4
:10A6D000079A012A04D1084B1A70FF2386F83330F9
:10A6E00000200DB0BDE8F08F42010020860300205D
:10A6F00030000020110E0100900000202DE9F047ED
:10A700006C4C86B094F839600746FF2E154640F031
:10A71000A580084604F13802052104F13903F7F752
:10A720001BFE94F838303846634F00936349052385
:10A730000DF11702F8F71CFB97F84A30002B3DD0BB
:10A7400003F0CEFA97F84AA0814603F0C7FA804694
:10A7500003F0C6FA6FEA0A0AD14408F1FF32431E39
:10A7600001210020D2B20091DBB25FFA89F10190A1
:10A7700002900390DFF8648102F098FE94F838307C
:10A7800058F82300F6F720FF814603F0A9FA4C4B56
:10A7900097F84A201B7897F84A100096CB1A03EBDB
:10A7A000D373C2EB630194F83830411858F8232072
:10A7B0004846C9B23346019603F048F93F4B0A2791
:10A7C0001E7846E094F8381038468B1B594241EB0E
:10A7D0000301F7F769FD042EDFF8D88035D898F823
:10A7E0003820384BC6EB020CDCF1000242EB0C02C5
:10A7F000384653F82610F7F745FB56B998F8642009
:10A800003D21D2F10102384638BF0022F7F79CFB08
:10A810001BE0032E98F838200BD0042E0DD0022E0A
:10A8200003D038462978012A0AE038466978022A96
:10A8300006E03846A978032A02E0E9783846042A77
:10A8400014BF00220122F7F76BFB0A370136FFB273
:10A85000F6B29DF81730B342B4D826E0042E24D8BF
:10A86000DFE806F0030A0C0F1500174B01201870E3
:10A87000FF2384F8393019E014480AE01448013203
:10A8800007E00232FF231348F6F7CDFE04E012483A
:10A890000332FF23F8F75CF8012806D10A4B187041
:10A8A000FF2384F83930013800E0002006B0BDE80D
:10A8B000F08700BF4201002050310020A603002095
:10A8C000F4000020F408010090000020180E0100A0
:10A8D000240E0100EE0E0100300E0100B81D010033
:10A8E0002DE9FF41384E074696F83B303446FF2BA2
:10A8F0004FD106F13A0206F13B0308460321F7F770
:10A900002BFD324E94F83A303146009305460DF156
:10A910000F0238460323F8F72BFA0A27367833E07C
:10A9200094F83A1038468B1B594241EB0301DFF88B
:10A930009880F7F7B9FC4EB998F83A103846D1F13B
:10A94000010138BF0021F7F7F1FC19E0022E17D8FA
:10A9500098F83A203846C6EB020CDCF1000242EBD4
:10A960000C021B49F7F78EFA98F83A20711EC6EBD5
:10A97000020EDEF10002384642EB0E02F7F7D0FA83
:10A980000A370136FFB2F6B29DF80F30B342C7D88E
:10A990000FE033B90F4B01201870FF2386F83B30CE
:10A9A0000FE0013B242505FB0322DBB2FFF7A6FEE7
:10A9B0000546012D04D1074B1D70FF2384F83B3061
:10A9C000002004B0BDE8F08142010020A90300206E
:10A9D000700F0100900000202DE9F047954C86B0E3
:10A9E00094F835600746FF2E154640F0DF80084694
:10A9F00004F134020A2104F13503F7F7ADFC94F8B1
:10AA0000343038468C4F00938C490A230DF11702DD
:10AA1000F8F7AEF997F84A30002B3DD003F060F913
:10AA200097F84AA0814603F059F9804603F058F997
:10AA30006FEA0A0AD14408F1FF32431E01210020C7
:10AA4000D2B20091DBB25FFA89F1019002900390DB
:10AA5000DFF8248202F02AFD94F8343058F82300FD
:10AA6000F6F7B2FD814603F03BF9754B97F84A20A3
:10AA70001B7897F84A100096CB1A03EBD373C2EBFE
:10AA8000630194F83430411858F823204846C9B27D
:10AA90003346019602F0DAFF684B0A261F787FE002
:10AAA00094F834103046CB1B594241EB0301F7F7C1
:10AAB000FBFB092FDFF87C816ED898F83420614BBE
:10AAC000C7EB020CDCF1000242EB0C02304653F8FB
:10AAD0002710F7F7D7F957B998F864203D21D2F13C
:10AAE0000102304638BF0022F7F72EFA54E0BB1EB1
:10AAF000072B05D8DFE803F00A121F2732383E443F
:10AB000094F8342030462978012A21E094F8343032
:10AB10000422304695F90110022B06E094F83430F7
:10AB200095F9021000223046032B14BF00230123A5
:10AB3000F7F72CFA30E094F834300022304695F9DB
:10AB40000310042BF1E794F83420A9883046052A35
:10AB500014BF00220122F7F7E3F91DE094F8342036
:10AB60003046E988062AF3E794F8342030462989EC
:10AB7000072AEDE794F8342030466989082AE7E788
:10AB800094F834203046A2F1090EDEF100022E497D
:10AB900042EB0E02F7F798F90A360137F6B2FFB228
:10ABA0009DF81730BB423FF67BAF3FE0092E3DD802
:10ABB000DFE806F0050C1215181E2124282F234B60
:10ABC00001201870FF2384F8353030E02A46FF2337
:10ABD0001F48F7F7BDFE20E01E486A1C04E01E482F
:10ABE000AA1C01E01D48EA1CFF23F6F71CFD14E037
:10ABF0001B482A1D09E01B48AA1D06E01A4805F15A
:10AC0000080202E0194805F10A02FF23F6F70BFFDC
:10AC100003E01748174AFFF763FE012806D10B4BE4
:10AC20001870FF2384F83530013800E0002006B0AA
:10AC3000BDE8F08742010020503100208A03002047
:10AC4000F4000020BC080100D10D0100900000209C
:10AC5000300E0100390E0100400E0100460E0100C9
:10AC6000510E01004C0E0100260A0100570E010092
:10AC70005D0E0100DC3000204C1C01002DE9FF417D
:10AC8000384E074696F837303446FF2B4FD106F141
:10AC9000360206F1370308460321F7F75DFB324E13
:10ACA00094F836303146009305460DF10F023846D0
:10ACB0000323F8F75DF80A27367833E094F8361066
:10ACC00038468B1B594241EB0301DFF89880F7F7B8
:10ACD000EBFA4EB998F836103846D1F1010138BF79
:10ACE0000021F7F723FB19E0022E17D898F8362039
:10ACF0003846C6EB020CDCF1000242EB0C021B49A9
:10AD0000F7F7C0F898F83620711EC6EB020EDEF198
:10AD10000002384642EB0E02F7F702F90A37013615
:10AD2000FFB2F6B29DF80F30B342C7D80FE033B987
:10AD30000F4B01201870FF2386F837300FE0013BDE
:10AD40002C2505FB0322DBB2FFF746FE0546012D4D
:10AD500004D1074B1D70FF2384F83730002004B066
:10AD6000BDE8F0814201002074030020660E01005E
:10AD7000900000202DE9F047944D86B095F8416091
:10AD80000746FF2E144640F0EE80084605F14002CB
:10AD90000D2105F14103F7F7DFFA95F84030384609
:10ADA0008B4F00938B490D230DF11702F7F7E0FF4E
:10ADB00097F84A30002B3DD002F092FF97F84AA056
:10ADC000814602F08BFF804602F08AFF6FEA0A0A92
:10ADD000D14408F1FF32431E01210020D2B200917C
:10ADE000DBB25FFA89F1019002900390DFF81882DC
:10ADF00002F05CFB95F8403058F82300F6F7E4FBCE
:10AE0000814602F06DFF744B97F84A201B7897F843
:10AE10004A100096CB1A03EBD373C2EB630195F88B
:10AE20004030411858F823204846C9B233460196AD
:10AE300002F00CFE674B0A261F788EE095F8401052
:10AE40003046C7EB010CDCF1000141EB0C01F7F7D8
:10AE50002BFA0C2FDFF874817BD898F840205F4BD9
:10AE6000C7EB020EDEF1000242EB0E02304653F851
:10AE70002710F7F707F857B998F864203D21D2F169
:10AE80000102304638BF0022F7F75EF861E0BB1ED2
:10AE90000A2B07D8DFE803F00C1319262C32383EB2
:10AEA000444B520095F840203046217D012A4BE06A
:10AEB00095F84020304694F91510022A44E095F8A0
:10AEC00040203046A17D032A3EE095F840203046E0
:10AED000A2F104035A4204F1180142EB0302F7F70E
:10AEE00035F936E095F840203046217F052A2BE0E1
:10AEF00095F840203046617F062A25E095F84020ED
:10AF00003046A17F072A1FE095F840203046218C6B
:10AF1000082A19E095F840203046618C092A13E090
:10AF200095F84020304694F825100A2A0CE095F850
:10AF30004020304694F826100B2A05E095F8402072
:10AF400094F8271030460C2A14BF00220122F6F78D
:10AF5000E7FF0A360137F6B2FFB29DF81730BB4261
:10AF60003FF66CAF5FE00C2E5DD8DFE806F0070E11
:10AF700011171A2023265656292C4F00184B012052
:10AF80001870FF2385F841304EE0164814323FE038
:10AF90001532FF231448F7F73DFD3CE01348163205
:10AFA00036E01832FF231248FAF726FB33E0114847
:10AFB0001C322DE010481D322AE010481E3227E0D6
:10AFC0000F48253224E00F48263221E042010020BC
:10AFD0005031002080030020F40000208808010088
:10AFE00090000020860E0100910E01009D0E0100D0
:10AFF000AA0E0100B40E0100C10E0100CD0E010029
:10B00000D90E0100E60E0100481E01000848273253
:10B01000FF23F7F79DFC012805D1064B01221A708A
:10B02000FF2385F84130002006B0BDE8F08700BF5F
:10B03000F30E0100900000202DE9F047754B86B01B
:10B0400093F845600746FF2E15461C4640F0CB801E
:10B0500003F14402084645330821F7F77DF994F8D7
:10B06000443038466C4F00936C4908230DF11702A9
:10B07000F7F77EFE97F84A30002B3DD002F030FE05
:10B0800097F84AA0814602F029FE804602F028FE89
:10B090006FEA0A0AD14408F1FF32431E0121002061
:10B0A000D2B20091DBB25FFA89F101900290039075
:10B0B000DFF8788102F0FAF994F8443058F8230068
:10B0C000F6F782FA814602F00BFE554B97F84A20BC
:10B0D0001B7897F84A10CB1A03EBD373C2EB6301CA
:10B0E00094F84430411858F823204846C9B23346F2
:10B0F0000096019602F0AAFC484B0A261F786DE0E4
:10B1000094F844103046C7EB010CDCF1000141EB30
:10B110000C01F7F7C9F8072FDFF8F8805AD898F82C
:10B120004420404BC7EB020EDEF1000242EB0E0260
:10B13000304653F82710F6F7A5FE57B998F8642063
:10B140003D21D2F10102304638BF0022F6F7FCFE65
:10B1500040E0BB1E052B04D8DFE803F00F151C23CD
:10B160002A3194F844203046A2F101035A4229685A
:10B1700042EB0302F6F7D4FE2CE094F84420291D9C
:10B180003046022A21E094F84420304605F11401AB
:10B19000032A1AE094F84420304605F12401042AD9
:10B1A00013E094F84420304605F13401052A0CE000
:10B1B00094F84420304605F14401062A05E094F84D
:10B1C0004420304605F5A271072A14BF002201224F
:10B1D000F6F77AFE0A360137F6B2FFB29DF817305D
:10B1E000BB428DD80AE016B1072E07D80AE00E4AF6
:10B1F00001201070FF2283F8452000E0002006B0F7
:10B20000BDE8F087084A01211170FF2283F845202C
:10B21000F4E700BF42010020503100209F030020CE
:10B22000F4000020781D010090000020C0090100FA
:10B230002DE9F0435B4F064697F84D4087B0FF2C51
:10B2400008463D4640F09180022107F14C0207F18B
:10B250004D03F7F781F897F84C303046524E009383
:10B26000524902230DF11702F7F782FD96F84A3092
:10B27000002B3BD002F034FD96F84A90804602F055
:10B280002DFD074602F02CFD6FEA0909C8447A1E1D
:10B29000431E01210020D2B20091DBB25FFA88F197
:10B2A000019002900390424F02F000F995F84C3063
:10B2B00057F82300F6F788F9804602F011FD3D4B60
:10B2C00096F84A201B7896F84A10CB1A03EBD373F2
:10B2D000C2EB630195F84C30411857F823204046E3
:10B2E000C9B223460094019402F0B0FB2F4B0A260A
:10B2F0001C7835E095F84C1030460B1B594241EB59
:10B300000301F6F7D1FF012C264F25D897F84C20E2
:10B31000294BC4EB020CDCF1000242EB0C0230467C
:10B3200053F82410F6F7AEFD54B997F864203D2188
:10B33000D2F10102304638BF0022F6F705FE0BE0DD
:10B3400097F84C203046A2F1010EDEF100021B49B5
:10B3500042EB0E02F6F7B8FD0A360134F6B2E4B25B
:10B360009DF81730A342C5D817E014B1012C14D1B1
:10B3700006E0134B01201870FF2387F84D300DE0D5
:10B380001048114AFCF756FA012806D10C4B1870E8
:10B39000FF2387F84D30013800E0002007B0BDE8FA
:10B3A000F08300BF42010020503100206E030020D6
:10B3B000A4070100F4000020741C0100D10D01005D
:10B3C00090000020020F01005C3100202DE9F047C1
:10B3D0009C4C86B094F851600746FF2E154640F00D
:10B3E000FB80084604F15002092104F15103F6F7ED
:10B3F000B3FF94F850303846934F00939349092394
:10B400000DF11702F7F7B4FC97F84A30002B3DD046
:10B4100002F066FC97F84AA0814602F05FFC804685
:10B4200002F05EFC6FEA0A0AD14408F1FF32431EC3
:10B4300001210020D2B20091DBB25FFA89F10190C4
:10B4400002900390DFF83C8202F030F894F850301C
:10B4500058F82300F6F7B8F8814602F041FC7C4B1F
:10B4600097F84A201B7897F84A100096CB1A03EBFE
:10B47000D373C2EB630194F85030411858F823207D
:10B480004846C9B23346019602F0E0FA6F4B0A26ED
:10B490001F789BE094F850103046C7EB010CDCF1AC
:10B4A000000141EB0C01F6F7FFFE082FDFF8948155
:10B4B00000F2888098F85020664BC7EB020EDEF150
:10B4C000000242EB0E02304653F82710F6F7DAFC82
:10B4D00057B998F864203D21D2F10102304638BFB7
:10B4E0000022F6F731FD6DE0BB1E062B05D8DFE824
:10B4F00003F0141B2B3242495E0029783F2904D9FE
:10B5000094F850203046544905E0544B490194F8D2
:10B5100050203046C918012A43E094F850203046A4
:10B5200095F90110022A48E0A9783F2904D994F836
:10B5300050203046484905E0484B490194F85020D6
:10B540003046C918032A2CE094F85020304695F96B
:10B550000310042A31E029793F2904D994F85020B6
:10B5600030463D4905E03D4B490194F850203046B6
:10B57000C918052A15E094F85020304695F90510B1
:10B58000062A1AE0A9793F2904D994F850203046B8
:10B59000314905E0314B490194F850203046C91833
:10B5A000072A14BF00220122F6F78EFC0AE094F865
:10B5B000502095F907103046082A14BF00220122B6
:10B5C000F6F7AEFC0A360137F6B2FFB29DF8173037
:10B5D000BB423FF65FAF57E0082E55D8DFE806F0D4
:10B5E000050C0E1114171A1D23001D4B0120187095
:10B5F000FF2384F8513048E01A4810E01A4801321D
:10B6000013E01A4802320AE0194803320DE01948E3
:10B61000043204E01848053207E018480632FF23D8
:10B62000F7F796F904E016480732FF23F7F7F2F927
:10B63000012829D10A4B1870FF2384F851300138B2
:10B6400023E000BF420100205031002066030020AB
:10B65000F4000020141C0100120B0100FC0C00205F
:10B6600090000020060F01000D0F01001C0F0100CB
:10B67000230F0100320F0100390F0100480F0100B4
:10B680004F0F0100241E0100002006B0BDE8F08726
:10B690002DE9F047874D86B095F855600746FF2E97
:10B6A000144640F09C80084605F154020C2105F137
:10B6B0005503F6F751FE95F8543038467E4F009307
:10B6C0007E490C230DF11702F7F752FB97F84A3029
:10B6D000002B3DD002F004FB97F84AA0814602F00F
:10B6E000FDFA804602F0FCFA6FEA0A0AD14408F13A
:10B6F000FF32431E01210020D2B20091DBB25FFA7B
:10B7000089F1019002900390DFF8EC8101F0CEFE08
:10B7100095F8543058F82300F5F756FF814602F0AB
:10B72000DFFA674B97F84A201B7897F84A10009683
:10B73000CB1A03EBD373C2EB630195F85430411875
:10B7400058F823204846C9B23346019602F07EF9E4
:10B750005A4B0A271E783DE095F8541038468A1B4C
:10B76000514241EB0201F6F79FFD0B2EDFF84481B9
:10B770002CD898F85420534B384653F82610931B76
:10B780005A4242EB0302F6F77DFB56B998F8642063
:10B790003D21D2F10102384638BF0022F6F7D4FB32
:10B7A00014E0022E08D001D30B2E0FD995F85420A7
:10B7B00038462168012A04E098F854202179384657
:10B7C000022A14BF00220122F6F7AAFB0A3701362B
:10B7D000FFB2F6B29DF81730B342BDD865E00B2E2C
:10B7E00063D8DFE806F0060D12181E252C333B4304
:10B7F0004B52354B01201870FF2385F8553055E02A
:10B80000FF233248F6F7F0F846E00432FF233048D1
:10B81000F7F79EF840E04832FF232E48FDF764F921
:10B820003AE002F58472FF232B48FDF731FB33E049
:10B8300002F5E472FF232948FCF774FF2CE002F5BF
:10B840004272FF232648FDF7B1FD25E002F5805244
:10B850000832FF232348FEF751FA1DE002F5885213
:10B860000832FF232048FEF731FC15E002F5905224
:10B870000832FF231D48FFF701FA0DE002F593524D
:10B88000FF231B48FFF72CF806E002F594521948F5
:10B890002832FF23FFF79AFD012806D10A4B1870C2
:10B8A000FF2385F85530013800E0002006B0BDE8E0
:10B8B000F08700BF42010020503100209E0300208D
:10B8C000F40000207C1C0100900000205E0F0100AD
:10B8D000640F0100740A0100790A0100820A010064
:10B8E000CF0A0100890A01008D0A01006E0F0100D4
:10B8F0005D0E0100790F0100080901002DE9F047F4
:10B90000A44D88B095F861600746FF2E144640F0BC
:10B910000D81084605F16002082105F16103F6F783
:10B920001BFD95F8603038469B4F00939B490823D8
:10B930000DF11F02F7F71CFA97F84A30002B3DD0A3
:10B9400002F0CEF997F84AA0814602F0C7F9804686
:10B9500002F0C6F96FEA0A0AD14408F1FF32431E29
:10B9600001210020D2B20091DBB25FFA89F101908F
:10B9700002900390DFF8508201F098FD95F8603056
:10B9800058F82300F5F720FE814602F0A9F9844B10
:10B9900097F84A201B7897F84A100096CB1A03EBC9
:10B9A000D373C2EB630195F86030411858F8232037
:10B9B0004846C9B23346019602F048F8774B0A264A
:10B9C0001F78ADE095F860103046CB1B594241EB33
:10B9D0000301F6F769FC072FDFF8B88100F29C80BD
:10B9E00098F860206F4BC7EB020CDCF1000242EBD1
:10B9F0000C02304653F82710F6F744FA57B998F876
:10BA000064203D21D2F10102304638BF0022F6F712
:10BA10009BFA81E0BB1E052B04D8DFE803F04853F6
:10BA2000595F657021684EF66023B1FBF3F1022285
:10BA300000234FF0010909B205A8CDF80090F5F7F1
:10BA400055F9594905A803F08FFB05A803F00EFC32
:10BA500022684FF47A78B2FBF8F23C23B2FBF3F1A0
:10BA600003FB112305AA19B2101800230222CDF8F6
:10BA70000090F5F73BF94C4905A803F075FB05A8C4
:10BA800003F0F4FB2368CDF80090B3FBF8F208FB59
:10BA9000123805AB032218180FFA88F10023F5F7C6
:10BAA00025F995F86020304605A94A4504E095F847
:10BAB00060203E493046022A14BF00220122F6F7D8
:10BAC00003FA29E095F860203046A188032A10E0A7
:10BAD00095F860203046E188042A0AE095F8602055
:10BAE0003046217A052A04E095F86020617A3046D4
:10BAF000062A14BF00220122F6F712FA0CE095F88C
:10BB000060203046A2F1070EDEF1000204F10C01C4
:10BB100042EB0E02F6F75AFB0A360137F6B2FFB2D5
:10BB20009DF81F30BB423FF64DAF5DE0072E5BD85E
:10BB3000DFE806F0040B111C1F25294C1C4B0120CB
:10BB40001870FF2385F861304FE02246FF23194823
:10BB5000F5F74AFF40E0637A33B1012B0CBFA288AE
:10BB6000E2884FF47A735343236037E01248221D72
:10BB700001E01248A21DFF23F5F755FF2CE0104805
:10BB800004F1080202E00F4804F10902FF23F6F76E
:10BB9000DFFE21E04201002050310020710300202F
:10BBA000F4000020E81D0100E6090100D10D0100AC
:10BBB000900000200C150100BE0F0100C50F010010
:10BBC000CC0F0100060701003C1D0100084804F1EC
:10BBD0000C02FF23F9F762FE012805D1054B012273
:10BBE0001A70FF2385F86130002008B0BDE8F087A7
:10BBF00026140100900000202DE9FF41384E074631
:10BC000096F863303446FF2B4FD106F1620206F1FD
:10BC1000630308460321F6F79FFB324E94F8623027
:10BC20003146009305460DF10F0238460323F7F71E
:10BC30009FF80A27367833E094F8621038468B1B59
:10BC4000594241EB0301DFF89880F6F72DFB4EB91E
:10BC500098F862103846D1F1010138BF0021F6F79B
:10BC600065FB19E0022E17D898F862203846C6EB1B
:10BC7000020CDCF1000242EB0C021B49F6F702F960
:10BC800098F86220711EC6EB020EDEF10002384603
:10BC900042EB0E02F6F744F90A370136FFB2F6B26C
:10BCA0009DF80F30B342C7D80EE033B90F4B0120D7
:10BCB0001870FF2386F863300EE0013B02EB03129D
:10BCC000DBB2FFF71BFE0546012D04D1074B1D70AB
:10BCD000FF2384F86330002004B0BDE8F08100BF8A
:10BCE0004201002099030020581501009000002017
:10BCF0002DE9F0477D4C86B094F865600746FF2E2D
:10BD0000154640F0A580084604F16402082104F1BC
:10BD10006503F6F721FB94F864303846744F0093BE
:10BD2000744908230DF11702F7F722F897F84A3003
:10BD3000002B3DD001F0D4FF97F84AA0814601F0D6
:10BD4000CDFF804601F0CCFF6FEA0A0AD14408F12A
:10BD5000FF32431E01210020D2B20091DBB25FFA14
:10BD600089F1019002900390DFF8B48101F09EFB0D
:10BD700094F8643058F82300F5F726FC814601F06A
:10BD8000AFFF5D4B97F84A201B7897F84A10009652
:10BD9000CB1A03EBD373C2EB630194F86430411800
:10BDA00058F823204846C9B23346019601F04EFEAA
:10BDB000504B0A271E7846E094F8641038468A1BD8
:10BDC000514241EB0201F6F76FFA072EDFF81C81B2
:10BDD00035D898F86420494B384653F82610931B01
:10BDE0005A4242EB0302F6F74DF846B998F8642040
:10BDF0003D21D2F10102384638BF00221DE0022E5B
:10BE000010D001D3072E1AD994F864203846A2F135
:10BE1000010CDCF1000205F1180142EB0C02F6F70F
:10BE200053F80CE098F8642095F92810A2F1020E5E
:10BE3000DEF10002384642EB0E02F6F785F80A37CB
:10BE40000136FFB2F6B29DF81730B342B4D848E0DD
:10BE5000072E46D8DFE806F0040B11171D252D35F7
:10BE6000274B01201870FF2384F865303AE0183220
:10BE7000FF232448F5F738FE2AE02832FF23224822
:10BE8000F6F732FB24E02C32FF232048FDF732FD89
:10BE90001EE002F502620C32FF231D48FEF74CFB48
:10BEA00016E002F562620C32FF231A48FCF792FAA0
:10BEB0000EE002F58C522C32FF231748FFF7E8FB07
:10BEC00006E002F5105215485C32FF23FFF794FE9E
:10BED000012806D10A4B1870FF2384F86530013819
:10BEE00000E0002006B0BDE8F08700BF420100205E
:10BEF000503100208D030020F4000020981D010027
:10BF0000900000201118010039130100FF0D0100FD
:10BF1000110E0100ED130100D10F01000C150100FD
:10BF20004C0901002DE9F0437B4C87B094F86D502B
:10BF30000646FF2D40F0AF80084604F16C0209214F
:10BF400004F16D03F6F708FA94F86C303046734E3E
:10BF50000093734909230DF11702F6F709FF96F8CC
:10BF60004A30002B3BD001F0BBFE96F84A90804649
:10BF700001F0B4FE074601F0B3FE6FEA0909C844B8
:10BF80007A1E431E01210020D2B20091DBB25FFA7B
:10BF900088F1019002900390624F01F087FA94F8C3
:10BFA0006C3057F82300F5F70FFB804601F098FE40
:10BFB0005D4B96F84A201B7896F84A100095CB1AEC
:10BFC00003EBD373C2EB630194F86C30411857F85C
:10BFD00023204046C9B22B46019501F037FD504B56
:10BFE0000A251E7852E094F86C1028468A1B5142AC
:10BFF00041EB0201F6F758F9082E474F42D897F85F
:10C000006C204A4B284653F82610931B5A4242EBA9
:10C010000302F5F737FF56B997F864203D21D2F1B6
:10C020000102284638BF0022F5F78EFF2AE0B31E32
:10C03000062B05D8DFE803F00A10161C262626007A
:10C0400094F86C2028463A49012A16E094F86C20AE
:10C0500028463749022A10E094F86C2028463449D3
:10C06000032A0AE094F86C2028463149042A04E0A7
:10C0700094F86C202E492846052A14BF002201227C
:10C08000F5F722FF0A350136EDB2F6B29DF817300A
:10C09000B342A8D83CE0082D3AD8DFE805F0050CFB
:10C0A0001014181C20252B00224B01201870FF2390
:10C0B00084F86D302DE00846F9F758FD1FE008467A
:10C0C000F9F7CEFE1BE00846FBF706FD17E0084631
:10C0D000FBF7C2FE13E00846FBF78EFF0FE0FF23DD
:10C0E0001548FFF7A5F80AE02032FF231348FEF7B2
:10C0F00041FE04E012484832FF23FEF79DFF01286D
:10C1000006D10C4B1870FF2384F86D30013800E025
:10C11000002007B0BDE8F08342010020503100202C
:10C12000AA030020F0070100F4000020AC1C01006D
:10C13000D10D01009000002083150100D80F0100EF
:10C14000E00F01002DE9F0435E4C87B094F8715088
:10C150000646FF2D40F08780084604F17002042156
:10C1600004F17103F6F7F8F894F870303046564E43
:10C170000093564904230DF11702F6F7F9FD96F8DE
:10C180004A30002B3BD001F0ABFD96F84A90804638
:10C1900001F0A4FD074601F0A3FD6FEA0909C844B8
:10C1A0007A1E431E01210020D2B20091DBB25FFA59
:10C1B00088F1019002900390454F01F077F994F8CF
:10C1C000703057F82300F5F7FFF9804601F088FD3D
:10C1D000404B96F84A201B7896F84A100095CB1AE7
:10C1E00003EBD373C2EB630194F87030411857F836
:10C1F00023204046C9B22B46019501F027FC334B62
:10C200000A261D782AE094F870103046C5EB010C20
:10C21000DCF1000141EB0C01F6F746F8032D294F44
:10C2200018D897F870202C4BC5EB020EDEF10002F7
:10C2300042EB0E02304653F82510F5F723FE4DB9B8
:10C2400097F864203D21D2F10102304638BF002228
:10C25000F5F77AFE0A360135F6B2EDB29DF81730E1
:10C26000AB42D0D829E0032D27D8DFE805F002093A
:10C270000E161A4B01201870FF2384F871301DE050
:10C28000FF231748FFF734FD0EE002F51252083283
:10C29000FF231448FBF782F906E002F51252124818
:10C2A0000C32FF23FFF73EFE012806D10B4B18701E
:10C2B000FF2384F87130013800E0002007B0BDE8AA
:10C2C000F08300BF42010020503100208B0300208A
:10C2D00088090100F4000020780801009000002087
:10C2E000AF110100E80F0100EF0F01000000000096
:10C2F0002DE9F04FB64C91B023780646FF2B40F065
:10C300009C87042804D00F21B24A2346F6F724F86C
:10C31000B04B1D78012D40F04F83AF48F6F7DEF8A3
:10C3200001F0DCFC044601F0DBFCDFF8BC82621E9D
:10C33000431E002420460A21D2B2DBB200950194AC
:10C340000294039401F0B2F8B8F838102B46224654
:10C3500009B20BA80095F4F7C9FCA0490BA802F09C
:10C3600003FF0BA802F082FFB8F854100BAA2B466B
:10C3700009B210182246FF270095F4F7B7FC0BA866
:10C38000F5F734F93B460C210BAA0097019701F011
:10C390003DFB01F0A3FC4008C5B201F0A1FC06463C
:10C3A00001F09EFC0A3800EBD0700A3E4FEA600AAA
:10C3B00006EBD676AAF10F0A76101FFA8AFA0A3629
:10C3C000F6B25FFA8AFB3B46284631465A4600974A
:10C3D000019701F0FAFB2746384603F013FF0F37A9
:10C3E000FF2403460090314628465A46BFB20194C6
:10C3F0000294039401F071FCB7F5B47FECD14FF0D7
:10C400000009ABF10502ABF10407DFF8E081284633
:10C410003146FFB2D2B24B46CDF80090CDF8049031
:10C4200001F04BFB314628463A464B46CDF800908A
:10C43000CDF8049001F041FB08F58653188FABF15D
:10C4400002021B8FD2B200B20692059303F0DEFE09
:10C45000634903F0E3FF634903F024FE059B844630
:10C4600018B2CDF814C003F0D1FE5D4903F0D6FF39
:10C470005C4903F017FEDDF814C0314663460090B6
:10C48000069A284601940294039401F026FC08F5CC
:10C490008852908A938A00B2059303F0B7FE504900
:10C4A00003F0BCFF4F4903F0FDFD4FF07E5103F058
:10C4B000F7FD059B844618B2CDF814C003F0A6FE24
:10C4C000474903F0ABFF474903F0ECFD4FF07E51C5
:10C4D00003F0E8FDDDF814C03A46ABF10707634608
:10C4E0003146FFB20090284601940294039401F073
:10C4F000F4FB284631463A464B46CDF80090CDF83D
:10C50000049001F0DAFA284631463A4623460327DA
:10C510000094019401F059FBBAFBF7F3B8F8381F07
:10C52000DFB2B8F8383F09B21BB2A1F50071A3F52C
:10C53000007301FB0AF103FB0AF34FEA5A0B5FFA9F
:10C540008BFB91FBF4F193FBF4F3CBEB0500EA1BBF
:10C550007118F318C0B2C9B2D2B2DBB20094019420
:10C56000029401F030F9B8F8381FB8F8383F09B232
:10C570001BB2A1F50071A3F5007301FB0AF103FBE7
:10C580000AF391FBF4F193FBF4F30BEB05007A193A
:10C590007118F318D2B2DBB2C9B2C0B200940194E0
:10C5A000029401F010F9B8F838CFB8F81C0F0FFA60
:10C5B0008CFCACF5007C0CFB0AFC9CFBF4FCB4444A
:10C5C00000B25FFA8CFCA0F50070B8F81CBF0FE059
:10C5D000B6010020B0030020ED130100F60F0100AA
:10C5E000000020410000B442901D0020D00C00202B
:10C5F000CDF814C003F00AFE03F0C8F900224FF092
:10C600007E5303F017FA70A3D3E9002303F012FA64
:10C6100003F0F2FC07900FFA8BF0A0F5007003F026
:10C62000F5FD03F0B3F900224FF07E53053F03F010
:10C6300001FA65A3D3E9002303F0FCF903F0DCFC65
:10C64000DDF814C0FFB261463A460090079B2846C9
:10C6500001940294039401F040FBB8F8383FB8F815
:10C660001C0F1BB200B2A3F50073A0F5007003FB12
:10C670000AFA03F0CBFD03F089F900224FF07E5354
:10C6800003F0D8F950A3D3E9002303F0D3F950A362
:10C69000D3E9002303F01CF803F0AEFCB8F81CBF8C
:10C6A0009AFBF4FA564482460FFA8BF0A0F500701C
:10C6B00003F0ACFD03F06AF900224FF07E5303F063
:10C6C000B9F941A3D3E9002303F0B4F940A3D3E9B6
:10C6D000002302F0FDFF03F08FFCF6B253460090FA
:10C6E000314628463A4601940294039401F0F5FA43
:10C6F00001F0F6FAB8F8005FA0F10E0AADB21FFA29
:10C700008AFA44468DB934490BA802F051FD334BE7
:10C710000DF12F0019880A2389B2B1FBF3F1093B0F
:10C72000009309B22A46013312E02D490BA802F00A
:10C730003FFDB4F8001F4FF47A7309B2890291FBF0
:10C74000F3F1012300930DF12F0009B24A46DB18E3
:10C75000F4F7CCFA23490BA802F006FD0BA8F4F776
:10C7600045FF054601F0BCFAA0F10A01FF23284667
:10C77000C9B20BAA4FEA5A0600930193023E01F098
:10C7800045F90C2700251BE06B01E31893F83E20C8
:10C79000394652B2002AB8BF0F321211FF230A32B3
:10C7A0000093019302930A203B46D2B2013502372F
:10C7B00001F009F8402DFFB202D10C27002539E025
:10C7C000B542E1DBF9E700BF000000000080464011
:10C7D0000000000000806640F80F0100D203002036
:10C7E000FC0F0100B215010001F078FA804601F05B
:10C7F00075FA182303FB054303F5026318339B887E
:10C80000A8F10A081BB2002BB8BFFF331B120A3B6A
:10C81000C2185FFA88F8FF23009301930293394608
:10C820003B464046D2B20135023700F0CCFF402DE6
:10C83000FFB201D0B542D7DBB4F8742E642112B236
:10C8400003254A4348BF1F32BAFBF5F55211594F31
:10C85000192605F1080BD2B20FFA8BF300924FF0B4
:10C86000320814200C213246CDF80480029603973A
:10C87000FAF7B0FF05F10C0307932B1D5B0008933B
:10C88000B4F8583E4FF064091BB209FB03F3FF22D2
:10C8900093FBF2F3079A029611B23246089EDBB27E
:10C8A0000093142033B2CDF804800397FAF792FF77
:10C8B000B4F8902E063512B248466D0050438146BA
:10C8C00048BF00F11F094FEA69195FFA89F2009227
:10C8D0006FF018020AF1080A0192921829B20FFAB1
:10C8E0008AF3029214204B3209950397FAF772FFEC
:10C8F00001F0F4F9054601F0F1F9B4F8AC6EA0F1DD
:10C90000140236B26420193D464348BF1F367611E3
:10C9100029B2F6B20FFA8BF312B219250096084627
:10C9200032260C21019602950397FAF753FF01F086
:10C93000D5F9804601F0D2F9B4F8E41EA8F1190344
:10C9400009B24FF0640808FB01F1A0F11402FF20C6
:10C95000029591FBF0F1089D18B2079BC9B212B283
:10C96000009119B22BB201960397FAF733FF01F049
:10C97000B5F9054601F0B2F9B4F8C84EA0F11402B9
:10C9800024B24046193D4443099E48BF1F346FF00E
:10C9900018002DB2641101900018E4B2029031B277
:10C9A00012B20FFA8AF3284600940397FAF712FF9F
:10C9B00000F04DBCEE290100042EBF4C20D194F8AC
:10C9C00065305BB194F86530012B14BFB4F8622078
:10C9D000B4F860204FF47A7392B25343E36594F84D
:10C9E0007520B54B5AB193F87520012A0CBFB3F8E6
:10C9F0007010B3F872104FF47A7289B24A43DA6653
:10CA0000AE48F5F76BFD01F069F9054601F068F9EC
:10CA10006A1E431E00254FF001080A212846D2B2A3
:10CA2000DBB2CDF8008001950295039500F03EFD44
:10CA300001F054F9A24F8008143897F828300E21DD
:10CA40000222C0B2CDF80080019500F073FD01F024
:10CA500045F9064607F1180000F092FFB608053EBA
:10CA6000A6EB5000FF2607F1180233462021C0B282
:10CA70000096019600F0CAFF92490BA802F098FBBD
:10CA8000914B2A4619880A2389B2B1FBF3F109B206
:10CA9000083B0CA8CDF80080F4F728F98B490BA8C7
:10CAA00002F062FB01F01CF9A0F1120133460BAA5F
:10CAB0000220C9B20096019600F0A8FF84490BA895
:10CAC00002F076FBB7F8541F4FF47A7309B289026B
:10CAD00091FBF3F12A46022309B20CA8CDF800809D
:10CAE000F4F704F97B490BA802F03EFB01F0F8F8DB
:10CAF000B0F10C0148BFA0F10901891001EB41011F
:10CB0000FF270D313B460220C9B20BAA00970197BF
:10CB100000F09CFFE16D4EF66029B1FBF9F10125B3
:10CB20000222002309B20BA80095F4F7DFF86A4946
:10CB30000BA802F019FB0BA802F098FBE36D4FF471
:10CB40007A764FF03C08B3FBF6F3B3FBF8F208FB40
:10CB500012330BAA19B21018002302220095F4F721
:10CB6000C5F85D490BA802F0FFFA0BA802F07EFBA6
:10CB7000E36D4FF00A0AB3FBF6F106FB1133B3FB8A
:10CB8000FAF10BAB022209B2181800230095F4F752
:10CB9000ADF801F0A3F883460BA800F0F1FEABF16D
:10CBA000020BC0EB0B000D213B460BAAC0B2009755
:10CBB000019700F02BFFE36E0222B3FBF9F90FFAA5
:10CBC00089F100230BA80095F4F790F842490BA8CF
:10CBD00002F0CAFA0BA802F049FBE36E0095B3FB22
:10CBE000F6F3B3FBF8F208FB12380BAA00230FFA96
:10CBF00088F110180222F4F779F837490BA802F0EF
:10CC0000B3FA0BA802F032FBE36E0095B3FBF6F229
:10CC100006FB12360BABB6FBFAFA02220FFA8AF1C8
:10CC200018180023F4F762F801F058F806460BA82C
:10CC300000F0A6FE054601F053F80346023EB3F1AC
:10CC40000C0148BFA3F10901751B8910234EE8B2FE
:10CC50000D31FF25C9B20BAA2B460095019500F0B6
:10CC6000D5FE716D4EF66023B1FBF3F10222002375
:10CC70004FF0010809B20BA8CDF80080F4F736F8A0
:10CC800015490BA802F070FA0BA802F0EFFA726DCA
:10CC90004FF47A77B2FBF7F23C23B2FBF3F103FBDC
:10CCA00011230BAA19B2101800230222CDF800801C
:10CCB000F4F71CF814E000BFD03000200010010091
:10CCC000D00C002009100100D2030020B215010091
:10CCD0000E10010013100100E60901005031002080
:10CCE000A2490BA802F040FA0BA802F0BFFA736D3C
:10CCF0000A22B3FBF7F107FB11370BABB7FBF2F1DD
:10CD000009B2083A18180023CDF80080F3F7EEFFB7
:10CD100000F0E4FF80460BA800F032FE074600F06A
:10CD2000DFFFA8F10208A0F11201C7EB0807C9B2A2
:10CD30000BAA2B46F8B20095019500F067FE301F54
:10CD4000F3F75CFD01281BD100F0C8FF06468848B8
:10CD500000F0C2FD054600F0C3FF0346023EB3F1FA
:10CD60000C0148BFA3F10901891001EB4101FF2328
:10CD7000751B0D31E8B200930193C9B27C4A1AE0E9
:10CD800000F0ACFF06467B4800F0A6FD054600F02B
:10CD9000A7FF0346023EB3F10C0148BFA3F109010E
:10CDA000891001EB4101FF23751B0D31714AE8B277
:10CDB00000930193C9B200F049FE00F08FFF4508CF
:10CDC00000F08EFF94F85410EDB26B4A0E3D11380E
:10CDD0003F29ADB286B202F5105300F2A48093F859
:10CDE00054100231490151188979012912D193F85F
:10CDF00054104901521892F83E1093F8552049B248
:10CE00002BB203EBD3794B4352B293FBF2F3C3EB58
:10CE1000690913E093F854104901521892F83E90B2
:10CE200093F855204FFA89F92BB209FB03F952B256
:10CE300099FBF2F903EBD37309EB63092BB20FFAF9
:10CE400089F99945D4BF29EAE979A94600F046FF56
:10CE5000059000F045FF834600F040FF074600F0D4
:10CE60003FFF5FFA85FA6FF00308059BCAEB0808DD
:10CE70005FFA88F803EB080EABF10A013A1F031FB3
:10CE80000020FF27C9B2D2B2DBB200905FFA8EF069
:10CE900001970297039700F0DDFB00F01FFF05905C
:10CEA00000F01EFF069000F019FF834600F018FF07
:10CEB000059B069943445FFA89F9D84409EB030EB0
:10CEC0000B39C144C31E5FFA89F2C9B25FFA8EF012
:10CED000DBB200970197029700F075FC00F0FEFEB0
:10CEE0002BB203EBD373CAEB630A834600F0F8FE60
:10CEF000814600F0F3FE804600F0F2FEAAF1040A3B
:10CF00005FFA8AFA8022D344831FA9F10801C24440
:10CF1000019202925FFA8BF0C9B25FFA8AF2DBB239
:10CF2000009700F050FC94F85610134A3F2902F580
:10CF3000105300F28B8093F85610023149015118BA
:10CF4000897901291AD193F856104901521892F89B
:10CF50003E1093F8572049B233B203EBD3784B43DA
:10CF600052B293FBF2F3C3EB68081BE0E609010041
:10CF70001810010020100100D00C002093F856106A
:10CF80004901521892F83E8093F857204FFA88F8DA
:10CF900033B208FB03F852B298FBF2F803EBD373F9
:10CFA00008EB63080FFA88F833B29845DABF28EA2D
:10CFB000E8781FFA88F8B04600F090FE074600F0C7
:10CFC0008DFE7F084208B91C0020083206F10D03CF
:10CFD000FF27D2B2DBB20090C8B20D2101970297B1
:10CFE000039700F037FB00F079FE814600F076FEF3
:10CFF00008F10D0842084FEA59095FFA88F109F172
:10D00000010909320B46D2B25FFA89F00097019705
:10D01000029700F0D8FB00F061FE804600F05EFE53
:10D0200033B203EBD373591042080D314FEA58085D
:10D030008023C9B208F104080632019302935FFA13
:10D0400088F0D2B20B46009700F0BDFB94F8581060
:10D05000814A3F2902F5105300F2848093F858105A
:10D060000231490151188979012912D193F85810D8
:10D070004901521892F83E1093F8592049B233B240
:10D0800003EBD3784B4352B293FBF2F3C3EB680844
:10D0900013E093F858104901521892F83E8093F823
:10D0A00059204FFA88F833B208FB03F852B298FBC4
:10D0B000F2F803EBD37308EB63080FFA88F833B286
:10D0C0009845D6BF28EAE878B0461FFA88F800F0FD
:10D0D00005FE074600F002FE7F084208A7F109019D
:10D0E00006F10D030020033AFF27D2B2DBB2009015
:10D0F000C8B20D2101970297039700F0ABFA00F038
:10D10000EDFD814600F0EAFD08F10D0842084FEA06
:10D1100059095FFA88F1A9F10A09023A0B46D2B21D
:10D120005FFA89F000970197029700F04CFB00F03E
:10D13000D5FD804600F0D2FD36B206EBD6767110F2
:10D1400042080D314FEA58088023C9B2A8F10708F8
:10D15000053A019302935FFA88F0D2B20B4600972A
:10D1600000F031FB94F85A103B4A3F2902F5105366
:10D170005FD893F85A10023149015118897993F810
:10D180005A104901521892F83E6093F85B2076B22B
:10D190002BB25E4352B296FBF2F603EBD37306EB6F
:10D1A000630636B22BB29E42D6BF26EAE6762E46FC
:10D1B000B6B200F095FD044600F092FDA4F10A011C
:10D1C000EA1C031F0020FF24C9B2D2B2DBB20090D8
:10D1D000033001940294039400F03CFA00F080FDC7
:10D1E000074600F07DFD0336F6B2C31EA7F10B0122
:10D1F0003246C9B2DBB2304600940194029400F08A
:10D20000E2FA00F06DFD064600F06AFD2DB205EB76
:10D21000D5756D1003358022EDB2831FA6F108018C
:10D22000019202922846C9B22A46DBB2009400F06D
:10D23000CAFA0A4D00232B7009E000230848314642
:10D24000054AFEF77FFF012801D1FF23237000204C
:10D2500011B0BDE8F08F00BFD00C0020B00300205B
:10D2600029100100AFF3008010F0800F10B532D10B
:10D270005F2930D8CB08DC0100196FF0070404FBEC
:10D280000311022AC9B20AD0032A11D0012A22D1DD
:10D2900012FA01F1104B1A5C42EA010106E0012288
:10D2A00012FA01F10C4B1A5C22EA0101195410BD6B
:10D2B000094B1A5C52FA01F414F0010F4FF001040B
:10D2C00005D014FA01F122EA01021A5410BD14FA31
:10D2D00001F10A431A5410BD780500202DE9F04FE2
:10D2E000772885B082460091934603939DF8385085
:10D2F0003EDC13019B1A002401930646A14621E05F
:10D30000224B019A9B181B5D3B4113F0010F07D084
:10D3100030464146039AFFF7A7FFDDF8089005E085
:10D3200025B1304641462A46FFF79EFF013708F1F6
:10D330000108082F5FFA88F8E2D1013401360F2C7A
:10D34000F6B205D0E3B20293DDF800800027D7E7FC
:10D3500085B10024009A0AF10F00A1180134C0B26F
:10D36000C9B22A46E4B2FFF77FFF082CF2D101E0F0
:10D370004FF00009BBF1560F86BF09F101095FFAB2
:10D3800089F00F2005B0BDE8F08F00BF2E2401000A
:10D390002DE9F04F85B0009040480191039301784A
:10D3A0003F4B1F2A5C5C9DF83860C4F10804E4B26E
:10D3B0000294824604D97E2A34BF15467E2500E0B9
:10D3C0002025384B5A5C009952187F2A53DC203DA7
:10D3D000EDB24FF0000B0F465C46A9462BE03149F9
:10D3E000CA5C314951F82330029902FB0932125DBF
:10D3F0006B1852FA03F313F0010F06D0384641467A
:10D40000039AFFF731FFA34605E026B138464146AF
:10D410003246FFF729FF013508F10108EDB25FFA46
:10D4200088F89AF800301E49CA5CAA42D7D801345D
:10D430000137E4B2FFB29AF800301A4AD35CA34233
:10D4400003D9DDF804800025EBE74D46AEB1002797
:10D450000AE0019A009BB918E018C0B2C9B232467E
:10D46000FFF702FF0137FFB29AF800300C49CB5C9E
:10D47000BB42EED801E04FF0000B103DEDB2092D9C
:10D4800004D89AF80030074AD05C03E00BF1010B96
:10D490005FFA8BF005B0BDE8F08F00BFE00100201F
:10D4A000612001002B240100D40100202DE9F84364
:10D4B00098469DF924709DF82030002FACBF0227BC
:10D4C0000127012B04460D4616460ED089461EE064
:10D4D000484629463A46FFF7C7FE09F101095FFAB7
:10D4E00089F9B145F4D90135EDB2454520D8A146B9
:10D4F000F7E7494620463A46FFF7B6FE494630462A
:10D500003A46FFF7B1FE09F101095FFA89F9C14511
:10D51000EFD90BE0204629463A46FFF7A5FE204604
:10D5200041463A46FFF7A0FE0134E4B2B442F1D9D5
:10D53000BDE8F8832DE9F04F8BB00F469DF85410ED
:10D54000772814460593069174DC059A1B0100F1B7
:10D55000FF399B1AA144002508935FFA89F9824696
:10D560000990AB4638E03A4B08995B185A5D42FA8D
:10D5700008F212F0010210D0049A504693190122C9
:10D580000092FE3201920292039231464A46DBB289
:10D59000FFF78CFFDDF81CB00EE0069B63B1049929
:10D5A00001928B190121009102920392504631465B
:10D5B0004A46DBB2FFF77AFF08F101083619B8F1E5
:10D5C000080FF6B2CFD10135A244A1440F2D5FFA66
:10D5D0008AFA5FFA89F908D0631EEAB2DBB20792D1
:10D5E00004933E464FF00008BDE7069BDC46DDF89D
:10D5F00024B00BB305FB04B50499EDB24E19F6B295
:10D60000E146049A08F1FF38D31901220092013A49
:10D61000019202920392394628463246DBB23F1904
:10D620005FFA88F8FFF742FFFFB2B8F1000FE8D1C8
:10D63000CC4601E04FF0000C059B562B86BF0CF149
:10D64000010C5FFA8CF00F200BB0BDE8F08F00BF2B
:10D650002E2401002DE9F14F98469DF92C709DF87C
:10D660002830002FACBF02270127012B04460D46AE
:10D6700016465DD101F1010B5FFA8BFBDA4611E032
:10D6800004F1010906E0484651463A46FFF7ECFD31
:10D6900009F101095FFA89F94E45F4DC0AF1010A42
:10D6A0005FFA8AFAD045EBDC05F102090BE0494646
:10D6B00020463A46FFF7D8FD494630463A46FFF73E
:10D6C000D3FD09F101095FFA89F908F1FF334B45F0
:10D6D000EDDC04F102090BE0484629463A46FFF723
:10D6E000C3FD484641463A46FFF7BEFD09F1010930
:10D6F0005FFA89F906F1FF3ACA45EDDC0134E4B27C
:10D7000008F1FF38204659463A465FFA8AFA5FFA2E
:10D7100088F8FFF7A9FD504641463A46FFF7A4FDB9
:10D72000204641463A46FFF79FFD5046594644E0A1
:10D7300001F102090BE0494620463A46FFF794FD05
:10D74000494630463A46FFF78FFD09F101095FFA75
:10D7500089F908F1FF334B45EDDC04F102090BE0D8
:10D76000484629463A46FFF77FFD484641463A4635
:10D77000FFF77AFD09F101095FFA89F906F1FF3A2D
:10D78000CA45EDDC01340135E4B2EDB208F1FF38F1
:10D79000204629463A465FFA8AFA5FFA88F8FFF788
:10D7A00063FD504641463A46FFF75EFD204641463E
:10D7B0003A46FFF759FD504629463A4601B0BDE8C2
:10D7C000F04FFFF751BD2DE9F04F87B005939DF95C
:10D7D000403005460492121A0598002BACBF022374
:10D7E000012392B20393431A9BB297B250000C46A6
:10D7F000590017F4004F9EB280B289B204D180B2B2
:10D8000001904FF0010806E04042574280B2BFB29B
:10D8100001904FF6FF7816F4004F04D189B20291BF
:10D820004FF0010B06E049425E4289B2B6B2029166
:10D830004FF6FF7B28462146039AFFF715FD0FB9E7
:10D84000002E46D032B23BB29A42AA46A14620DC14
:10D850001FFA88F84544ADB20024029A2E46A41857
:10D86000A3B29CB221B23AB2914205DD0199D944EA
:10D870005C1A1FFA89F9A4B2E8B2039A5FFA89F137
:10D88000FFF7F2FC049A36B245449642ADB2E4D1B9
:10D890001FE01FFA8BFB5C44A4B20025019B32B24F
:10D8A000ED18ABB29DB229B29142274605DD029830
:10D8B000C2441D1A1FFA8AFAADB2E1B25FFA8AF0C9
:10D8C000039AFFF7D1FC05993FB25C448F42A4B2A2
:10D8D000E4D107B0BDE8F08F2DE9F047244B0646B0
:10D8E0001B7800203DE0234911F803C0A2F130016C
:10D8F000C9B2CCF1080809295FFA88F81E4901D895
:10D90000C95C2BE01F2A03D95E2A28BF5E2200E0F3
:10D910002022CF5C203AD2B200217A430C4617E095
:10D92000DFF8589059F8239019F802A005EB080980
:10D930004AFA09F909F00109B9F1000F18BF2146A7
:10D9400001355FFA85F9E145EAD30134E4B20132E9
:10D95000BC4201D00025F4E70131C9B201314018C1
:10D96000C0B216F8012B002ABDD1BDE8F08700BF78
:10D97000E0010020612001002B240100D4010020DF
:10D980002DE9F0411F4B204C0022197824681A70B1
:10D990009C462EE0A5F13003DBB2092B25D91F2DC3
:10D9A00003D95E2D28BF5E2500E02025203DEDB285
:10D9B00005EB4505631900252F4611E093F800801B
:10D9C00048FA06F8013608F00108B8F1000F18BF50
:10D9D0002F46082EF2D10135EDB20133032D01D0CF
:10D9E0000226EBE70137FFB200E003270137D21927
:10D9F000D2B210F8015B002DCCD18CF8001010468B
:10DA0000BDE8F081E0010020D40100202DE9F341C0
:10DA10000D4B0F4600211E78044619701546984696
:10DA200009E000230093204639460333FFF7B0FC9A
:10DA300001302418E4B215F8012B002AF1D188F83E
:10DA400000602046BDE8FC81E00100200B4B73B56F
:10DA50000E46012104461970154609E00023009383
:10DA6000204631460333FFF793FC01302418E4B21B
:10DA700015F8012B002AF1D120467CBDE0010020E1
:10DA80002DE9F0410C4686B0984611B201230022E0
:10DA900005469DF830709DF83460009302A8134647
:10DAA000F3F724F92846214602AA43460097019637
:10DAB000FFF7CCFF06B0BDE8F0812DE9F04F8BB049
:10DAC0009DF850B09A469DF85430C2F101064FF0CF
:10DAD000010C00245F468046894608931546B6B27D
:10DAE0000794E34604EB08035FFA85FCDBB2069378
:10DAF0000CEB0901089AC4EB0803DBB2C9B2099325
:10DB0000029206981A460B46CDF814C0CDF800A034
:10DB10000197FFF758FEDDF814C0089BCCEB090114
:10DB2000C9B2029306980B46099ACDF800A0019756
:10DB3000FFF749FEDDF814C0089ACCEB0803C4EBEC
:10DB40000901C4445FFA8CFCDBB2C9B218460693E3
:10DB500002920B466246CDF814C0CDF800A00197A2
:10DB6000FFF731FE089BDDF814C004EB0901C9B2D0
:10DB70000293069862460B46CDF800A00197FFF786
:10DB800022FE16F4004F06D0079A033606EB420633
:10DB9000B6B25B4609E0079A2BB2D31A053606EBFC
:10DBA0004306013DB6B25B46ADB2079A1BB20132E5
:10DBB00007922AB2013C0BF1010B9342E4B21FFA27
:10DBC0008BFB8FDD0BB0BDE8F08F2DE9F04F5BB222
:10DBD00089B0C2F101074FF0010800258346039187
:10DBE000002BACBF022401241646BFB2AA46C14690
:10DBF000039AC5EB0B035FFA86F8DBB2069308EBDA
:10DC00000203DBB21946069822460193FFF72CFB6C
:10DC100008EB0B02D2B20492039A0498C5EB020CF3
:10DC20005FFA8CFC61462246CDF808C0FFF71CFB6A
:10DC3000019B05EB0B02D2B2104619460792224611
:10DC4000FFF712FBDDF808C0C8EB0B03DBB261463F
:10DC5000184622460593FFF707FB039A0498AB1872
:10DC6000DBB2194622460193FFF7FEFA039A0698A3
:10DC7000C8EB02085FFA88F841462246FFF7F4FA3B
:10DC8000079841462246FFF7EFFA019B059819468F
:10DC90002246FFF7E9FA17F4004F05D0033707EBE8
:10DCA0004A07BFB24B4609E033B2C3EB0A0305375C
:10DCB00007EB4307013EBFB24B46B6B21BB232B2CE
:10DCC000013D09F1010993420AF1010AEDB21FFA7F
:10DCD00089F98DDD09B0BDE8F08F7047802070476D
:10DCE00060207047024800214FF4C06201F0E2B9A1
:10DCF00078050020014800F0B1B800BF7805002089
:10DD000008B500F01DF9002008BD7047F8B51C4E9D
:10DD10000D4626F07F4206F0704322F4700243F075
:10DD20000071520111430968074641B343F0007383
:10DD300043F0040343EA02021368F3B1114800F010
:10DD40009DFF04460028F9D10F488021224600F0AB
:10DD500093FE06F0704343F0007326F07F4643F0D5
:10DD6000040326F4700643EA4616346005E00548CD
:10DD700017F8011B00F07CFF013D002DF7D1F8BD25
:10DD8000C8030020008000400060004038B51C4DF2
:10DD9000044625F07F4205F0704322F4700243F000
:10DDA000007152011143096849B343F0007343F015
:10DDB000040343EA02021368BBB9124800F05EFF95
:10DDC0000028FAD1802110480A4600F055FE05F0DF
:10DDD000704343F0007325F07F4543F0040325F4BE
:10DDE000700543EA451501232B60084D05E0054801
:10DDF00015F8011B00F03CFF013C002CF7D138BDA9
:10DE0000C80300200080004000600040BE030020E6
:10DE100038B50E4B00221A605A600D480321FFF7F7
:10DE200075FF0C480321FFF771FF0B480221FFF734
:10DE30006DFF602406E00820FFF7A8FF013DFAD13E
:10DE4000013C01D00825F6E738BD00BFBE03002025
:10DE5000A12901004F2901004D2901002DE9F347B7
:10DE6000334B03211A889B78ADF804208DF80630D7
:10DE7000304B80461A889B7801A8ADF800208DF8B9
:10DE80000230FFF743FF68460321FFF73FFF2A48B0
:10DE90000221FFF73BFF012000F0C7F900243EE01C
:10DEA0007B0803218DF8053001A801338DF8063079
:10DEB000FFF72CFF214B00221A60494619F8012B6D
:10DEC0001AEA020218BF80221A6049781AEA010F82
:10DED00014BF42F0080222F00802013701201A6044
:10DEE000BFB2FFF753FF802FDAD10135082D10D0D4
:10DEF0008DF801600136F6B2684603214FF0010A41
:10DF00008DF802600AFA05FAFFF700FFC146002704
:10DF1000C6E70834E4B2602C08F1800802D0264637
:10DF20000025E5E7012000F07FF9BDE8FC8700BF90
:10DF3000472901004A2901004D290100BE030020A4
:10DF4000F7B5314800F09EFE304800F09BFE3048A7
:10DF500000F098FE4FF040202C2100F0BAFD042282
:10DF60000A234FF040202C2100F01FFD2948C0213A
:10DF700000F093FD08232748C021042200F015FD7E
:10DF8000254EC0210A46234800F076FD06F0704376
:10DF900026F07F4643F0007726F47006760147F0BE
:10DFA0000403334301251D601C4800F05CFE00F0B3
:10DFB00029FF1B4B08240146032200931748002326
:10DFC000019400F026FE21464FF0402000F081FD34
:10DFD000214604220A234FF0402000F0E6FC47EAE5
:10DFE00006060E4800F03AFE3560FFF711FF083CC8
:10DFF0000C4B601C1D5D1818691E01356419FFF774
:10E0000085FE4E2CF4D9FEBD10000010010000204A
:10E010000400002000600040C80300200080004091
:10E0200040420F005229010008B5054800F03EFEAD
:10E0300000F0D8F800F0F6F800F01AF8002008BD5B
:10E04000803B800710B500F0EEF8BDE8104000F00E
:10E05000D5B80000034B044A188005234B431380B6
:10E06000704700BFCE030020CC03002070470000A3
:10E0700010B54FF0101000F005FE1C4800F002FE35
:10E0800002211B4800F017FD1A4800F0FBFD01219A
:10E09000194800F010FD00F0B5FE4FF4DC74B0FB41
:10E0A000F4F440210222154800F06CFD4021224684
:10E0B000124800F081FDA2084021104804EB4404FE
:10E0C00000F08EFD4121A2080C4800F089FD0321DB
:10E0D00001220A4800F095FD4021084800F076FD35
:10E0E00006484021BDE8104000F075BD0800002042
:10E0F00000700040200000200050024000800240DC
:10E1000008B500F07BFFB0F57A7FFAD800F076FF13
:10E11000B0F57A7FFAD308BD10B50E4800F0B2FD15
:10E120000D4800F0AFFD0F210C4800F0A8FC0122C3
:10E130000A230F21094800F038FC0221084800F0AA
:10E140009EFC0748022101220A23BDE8104000F08E
:10E150002CBC00BF10000020200000200040024026
:10E16000005002407047000008B51248012100F03D
:10E1700080FCB8B10F48022100F07BFCA0B10D4833
:10E18000042100F076FC88B10A48082100F071FCF7
:10E1900070B10948022100F06CFC00280CBF04207B
:10E1A000002008BD042008BD012008BD032008BDD3
:10E1B000022008BD004002400050024008B5FFF7B1
:10E1C000D3FF022808D0032808D0012808D004284B
:10E1D0000CBF4420002008BD432008BD412008BDDD
:10E1E000422008BD10B500F00DFE0A23B0FBF3F08D
:10E1F00000F0FEFEBDE8104000F0F2BE7047704730
:10E2000000207047FFF7FBBF032808B507D840B2CE
:10E21000FFF7F6FF8000A0F5FE600F3800E0002059
:10E2200000B208BD704770477047704770470000E4
:10E2300010B50F4800F026FD0E4800F023FD00F059
:10E2400064FC03214FF0402000F051FC00F0DAFDA7
:10E250004FF4E13201466023074800F0EFFE15203D
:10E2600000F058FC04485021BDE8104000F016BFF3
:10E27000010000100100002000C00040024B0022FD
:10E2800023F81020704700BFA80C002038B50846BE
:10E290000D4600F0EBFF044604E0044815F8011BAE
:10E2A00000F0F3FE013CF8D238BD00BF00C00040D2
:10E2B00010B5012386B000220446009302A813463D
:10E2C000F2F714FD204602A9FFF7E0FF06B010BDEB
:10E2D000024B33F8101009B2FFF7EABFA80C002078
:10E2E0005F4B70B55A6D00240A325A6504F51076FA
:10E2F0005C4D063605EB061606F10800F2F77EFACD
:10E3000001286AD13379ABB105EB041303F510533F
:10E31000DA6D583372B15A6833794FF47A714B43DE
:10E32000B2FBF3F103FB112323B94FF448700A2128
:10E33000FFF790FE04F51072063205EB02125279D7
:10E34000484923012ABBCB1803F51053DA6D0A3272
:10E35000DA65B3F86020D96D4FF47A7392B2B1FBED
:10E36000F3F39A4204D14FF448702821FFF772FE6C
:10E3700005EB041303F51053B3F86220D96D4FF485
:10E380007A7392B2B1FBF3F39A4216D14FF46170F3
:10E3900010E0CB1803F5105358335A680A2A03D9F2
:10E3A0005A680A3A5A6008E05A6832B100225A6044
:10E3B0004FF47A702821FFF74DFE04F510760636EB
:10E3C00005EB0613DB7923B94FF448700521FFF7FD
:10E3D00041FE05EB0615012331E07379012B08D1CD
:10E3E00005EB041303F51053DA6D58330AB91A8993
:10E3F00010E004F51073063305EB03135B79022B71
:10E400000DD1184B03EB041303F51053DA6D583399
:10E410002AB95A8992B24FF47A714A435A6004F584
:10E420001076063605EB0613DB79012B04D14FF489
:10E430002F700521FFF70EFE05EB061500230134B2
:10E44000022CEB717FF452AF074B1B78012B05D1E7
:10E45000064C237813B9FFF7B1FE207070BD00BFE2
:10E4600050310020D00C0020D7030020D103002021
:10E470007FB52648F2F726F9F2F73CFAFFF7D4FD0C
:10E48000FFF7F4FD0020FFF7D3FE00202049FFF73F
:10E49000FDFE00201F49FFF7F9FE00220123009333
:10E4A00003A8134642F21871F2F720FC002003A9DA
:10E4B000FFF7ECFE00201849FFF7E8FE002017499F
:10E4C000FFF7E4FEFFF71CFC00201549FFF7DEFE16
:10E4D000F4F702F900201349FFF7D8FE1248F4F7C9
:10E4E00001FB00201149FFF7D1FEFFF703FC0020DC
:10E4F0000F49FFF7CBFEFFF785FEFFF70DFE00206B
:10E500000C49FFF7C3FE07B000BD00BFD00C0020D0
:10E51000A4290100B5290100E20A0100C029010077
:10E52000C9290100CD290100D1290100DD290100FF
:10E53000E1290100E729010010B5FFF7D3FBF4F74B
:10E54000CBF81248F4F7CEFAFFF7D4FBF2F7E0FF6E
:10E55000F4F7C2F80E48F4F7C5FAFFF7CBFB4FF417
:10E560007A70FFF7CDFDFFF7BDFBFFF7C3FBFFF7A9
:10E57000CCFB6420FFF7C4FDFFF7F4FD0020FFF79C
:10E5800055FEBDE81040FFF75DBD00BFEF2901005B
:10E59000FE29010070B5494B494C00250122257028
:10E5A00028461A704749FFF771FE474B1D76803B9E
:10E5B00093F85320012A04D128464449FFF766FE08
:10E5C0006BE093F85330022B67D128464049FFF7A0
:10E5D0005DFE5CE0FFF784FE2B78002B39D02B78B2
:10E5E0002B78412B02D02B78482B02D14FF4487066
:10E5F00027E02B78422B02D02B78502B02D14FF4FE
:10E6000061701EE02B78432B05D02B780A2B02D0AB
:10E610002B780D2B02D14FF47A7012E02B78442B1B
:10E6200002D140F24C400CE02278254B712A32D0C6
:10E630001A78952A08D91A78C72A05D81B784FF472
:10E64000FA700A21FFF706FD0A20FFF759FD0023A3
:10E650002370F4F741F8FFF741FB1E4D29782A7823
:10E66000401A15F8023C0021C0B2F3F7ADFEFFF7E7
:10E6700035FB0246002015F8023C0146F4F76CF821
:10E68000FFF738FB144BFF221A70FFF7EFFC2378DB
:10E690000B4D712B9ED10023237010490020FFF7F2
:10E6A000F5FDF2F76BFB0E48F2F776FBF2F766FB2F
:10E6B0000B48BDE87040F2F76FBB00BFD7030020E6
:10E6C000D10300200A2A0100D0310020112A0100C4
:10E6D0001C2A01009B310020E2010020E7290100F3
:10E6E000FC0C00202DE9F347FFF7C2FEFFF752FFB5
:10E6F0007C487D497D4AFF237D4E03700B7013706B
:10E70000FF3B33707B4B01241C7081468846924648
:10E71000DDE0FFF7E5FDF2F731FBF2F797F82B7834
:10E72000002B52D0744CB4F9003003B92B703278FE
:10E7300032786F4B412A02D01A78482A05D16F4BA4
:10E7400002221A704FF4487034E01A78422A02D03C
:10E750001A78502A05D1694B01221A704FF4617062
:10E7600028E01A78432A05D01A780A2A02D01A78A3
:10E770000D2A05D1614B03221A704FF47A7019E00B
:10E780001A78442A05D15D4B403A1A7040F24C4049
:10E7900010E01A78712A00F09F801B78952B0CD915
:10E7A0003378C72B09D8524B4FF4FA701A78534B71
:10E7B000323A1A700A21FFF74DFC0A20FFF7A0FC3D
:10E7C0000023337042F2107323804D4B1B7863B1EA
:10E7D0009AF80020454B3F2A07D81A780A2188F872
:10E7E0000020484A1170FF221A70F3F775FFFFF7F7
:10E7F00075FA454C414F21782278401A14F8023CB2
:10E800000021C0B2F3F7E0FDFFF768FA14F8023C0C
:10E8100002463E4C00200146F3F79EFF23781BB9C9
:10E820003878FDF765FD18E0022B4FF0000513D096
:10E83000032B11D0042B0FD002AAFF2302F8015D95
:10E8400033483978F8F73EFE012806D19DF80730A5
:10E85000042B01D125703FE0257000233B70294B2C
:10E860001A7852B1013A98F800001A70294B420107
:10E87000D318997949B2F4F76DF9274C237853B13D
:10E8800026482146F4F722FA254B1A78013A1A70E5
:10E890001B7803B92370234B1A8840F6736392B236
:10E8A0009A420DD82048F3F719FEF3F715FFFFF74A
:10E8B000DDFB114B1A8811B20A2901DD0A3A1A80D0
:10E8C000FFF718FAFF2389F80030FFF7CFFB337802
:10E8D000074D712B7FF41DAFFFF72EFE0020BDE822
:10E8E000FC8700BFE2010020E1010020E3010020DD
:10E8F000D1030020D7030020E4010020D003002032
:10E90000A1310020D50300209B310020D40300203A
:10E91000400E0100080D0020AC0C0020292A010047
:10E92000D6030020D2030020322A0100FEE7FEE7D2
:10E93000FEE700000A4A0B4B03E052F8041B43F8C1
:10E94000041B09498B42F8D3084809494FF00002DB
:10E950008842B8BF40F8042BFADBFFF7C3BE00BF04
:10E96000B42B010000000020E0020020E0020020A3
:10E97000E8330020EFF3108062B67047D0F800341F
:10E9800012F0010F14BF0B438B4310B500F58064E8
:10E99000236012F0020FD0F8202400F5846314BF26
:10E9A000114322EA0101196010BD30B5D0F80045CD
:10E9B00012F0010F14BF0C438C4300F5A0652C60CE
:10E9C000D0F8045512F0020F00F5A06414BF0D43F7
:10E9D0008D4304342560D0F8084512F0040F14BFAD
:10E9E0000C438C4300F5A1652C6012F0080FD0F8A1
:10E9F000182500F5A36414BF0A438A432260D0F8A7
:10EA00000C4513F0010F00F5A06214BF0C438C43BA
:10EA10000C321460D0F8102513F0020F14BF0A4313
:10EA20008A4300F5A2642260D0F8144513F0040F65
:10EA300000F5A26214BF0C438C4304321460D0F87A
:10EA40001C4513F0080F00F5A26202F10C0214BF7E
:10EA50000C438C43146000F5A56223B9D0F8283527
:10EA600043EA010103E0D0F8283523EA01011160EF
:10EA700030BD50F82100704740F82120704770B534
:10EA8000002205460C46FFF779FF28462146012261
:10EA90000823BDE87040FFF788BF70B50122054626
:10EAA0000C46FFF76BFF2846214601220823BDE8EC
:10EAB0007040FFF77ABF70B5022205460C46FFF79B
:10EAC0005DFF2846214601220823BDE87040FFF77C
:10EAD0006CBF70B5022205460C46FFF74FFF284673
:10EAE000214601220823BDE87040FFF75EBF70B5E4
:10EAF000022205460C46FFF741FF28462146012227
:10EB00000823BDE87040FFF750BF08B5FFF732FF9C
:10EB1000C0B208BD042804D1164B1A6842F48032F2
:10EB200005E0052805D1134B1A6842F400321A603B
:10EB30007047062804D10F4B1A6842F48022F6E78A
:10EB40000F2804D10C4B1A6842F00202EFE7A0F143
:10EB500010031F2B05D8012212FA03F3074A136092
:10EB600070472F2805D90123303813FA00F0044BE1
:10EB70001860704724ED00E010E000E000E100E0E4
:10EB800004E100E030B50D580A4C12F0020F05EA1E
:10EB9000040444EA020401EB00030C5004D0B02248
:10EBA0001A624FF4306203E08C221A6240F60C02C3
:10EBB0005A6230BD0100F8FF0B18095811F0020F1E
:10EBC00001D0520800E0013A1A6170470B5843F037
:10EBD00001030B5070470B5823F001030B50704793
:10EBE00010B521F03F042318205810F0020F1869C7
:10EBF00018BF5208821A11F0010F14BFDA619A612E
:10EC000010BD8368012A0CBF194323EA010181600A
:10EC10007047022B10B502D023B1002300E0082377
:10EC2000042400E01C4623434360029BB1FBF3F144
:10EC300000230233B1FBF3F4013CFF2CF9D803614C
:10EC4000930103F0FF0302F0300243EA0202039B48
:10EC5000013B1A4342EA0424046010BD436843F0B8
:10EC6000020343607047436823F002034360704728
:10EC7000C36813F0020FFBD081607047C068C0F317
:10EC800000107047020F81B200F4F810000C11FA66
:10EC900000F0034B53F822301A6810431860704795
:10ECA000A02A01000138FDD1704700004B4B70B520
:10ECB0001A68044612F0E04F06D01A68484B02EA80
:10ECC0000303B3F1805F02D1002CC0F28680454976
:10ECD000454A0B68166843F4006323F4800546F444
:10ECE000006613F0020F0D60166002D014F0020FE0
:10ECF00005D015F0010F1AD014F0010F17D164F0F0
:10ED000003031D40374B002E1D6005DA06F070032B
:10ED1000302B05D0702B02E005F03003302B02D1F0
:10ED20004FF4805001E04FF40020FFF7BBFF25F4C3
:10ED30005E5543F2F07304EA030325F070051D43AA
:10ED40002A4B2B4A06EA03032A4E402104EA060610
:10ED50001E4304F0080356EAC306234B116002F178
:10ED600008024BBF1E60156015601E601020FFF783
:10ED700099FF214B25F0F86504EA030325F003050C
:10ED80001D4326F0FC5604F0FC5314F0804F46EA75
:10ED9000030608D0194B26F4800604EA030345F461
:10EDA00080051E4301E026F0804614F4006F0CD16C
:10EDB0004FF40043124A126812F0400F01D1013B98
:10EDC000F8D125F4006526F40066064B10201D607E
:10EDD0001E61BDE87040FFF765BF70BD00E00F40E9
:10EDE0000000FF7060E00F4070E00F408FDFFF7F9A
:10EDF00058E00F40302000800300C0070000404072
:10EE000050E00F40694B70B51A6810331B68002B37
:10EE1000B4BF03F0700102F0300120293AD004D8C9
:10EE200069B1102940F0C08010E060295DD07029E0
:10EE300058D0302940F0B88047F2305063E002F4F7
:10EE4000F8605B49800951F820005CE05949086886
:10EE500010F0E04F4CD00C68574804EA0000B0F1C5
:10EE6000805F45D00C68544804EA0000534CA0422F
:10EE700003D1096889B202293CD04E484E49046842
:10EE800004EA01014E4CA14236D100684D4980B2DE
:10EE90004D4C22E04749086810F0E04F2ED00C6836
:10EEA000454804EA0000B0F1805F27D00C68424872
:10EEB00004EA0000414CA04203D1096889B202294A
:10EEC0001ED03C483C49046804EA01013C4CA14284
:10EED00018D100683D493E4C80B200280CBF204646
:10EEE000084610E04FF400400DE04FF480000AE0C7
:10EEF000384808E0344806E0324804E0364802E08A
:10EF0000334800E03148002B02DA13F4006F01E0CF
:10EF100012F4006F2AD13149264D09682C6814F08B
:10EF2000E04F43F6E07401EA040406D02E68224D57
:10EF300006EA0505B5F1805F06D16409023401F0E7
:10EF40001F056043023505E06409604301F01F05B9
:10EF500001356D00B0FBF5F011F4804F18BF40088B
:10EF600011F4004F18BF800842F4800212F4800FA1
:10EF70001BD0002B11DA13F0804F07D013F4006F71
:10EF800004D103F0FE5340009B0D02E003F0FC535C
:10EF9000DB0D0133B0FBF3F070BD02F0F062D20D77
:10EFA0000132B0FBF2F070BD002070BD60E00F4098
:10EFB000442A010000E00F400000FF700000011033
:10EFC000000003100024F400001BB70000093D00FE
:10EFD000C0C62D00C0E1E4007038390064E00F4085
:10EFE000024B1A6842F005021A60704710E000E018
:10EFF000014B01381860704714E000E0014B1868BD
:10F00000704700BF18E000E0C36A43F01003C3621A
:10F01000036B43F4407343F0010303637047836958
:10F0200013F0080FFBD1C36A23F01003C362036B14
:10F0300023F4407323F00103036370472DE9F0418B
:10F040000D46164604461F46FFF7E9FFB5EB061FBF
:10F0500005D2236B760843F02003236303E0236B80
:10F0600023F020032363ED00B5FBF6F601367308A9
:10F0700003F03F03F60966622046A3620023E762BD
:10F08000A361BDE8F041FFF7BFBF836913F0200F14
:10F0900002D101600120704700207047836B0B4351
:10F0A0008363704700210A2200F0C2B900220A23BC
:10F0B00000F00CB9032AC9B270B408D82AB10346CB
:10F0C000121803F8011B9342FBD170BC70478218E1
:10F0D000044601E004F8011B14F0030FFAD14FF0CD
:10F0E000013303FB01F31FE044F8403C44F83C3C8F
:10F0F00044F8383C44F8343C44F8303C44F82C3C68
:10F1000044F8283C44F8243C44F8203C44F81C3C97
:10F1100044F8183C44F8143C44F8103C44F80C3CC7
:10F1200044F8083C44F8043C161B254640343F2E66
:10F13000DADC2C4607E044F8103C44F80C3C44F878
:10F14000083C44F8043C161B254610340F2EF2DC14
:10F1500001E045F8043B541B032CFADC01E005F800
:10F16000011B9542FBD3B0E710F0030F38B50446FE
:10F1700012D10368A3F1013222EA030313F0803FA6
:10F180000AD1031D184653F8042BA2F1013525EAD4
:10F19000020212F0803FF5D003782BB1431C1846D1
:10F1A00013F8012B002AFAD100F002F8204638BDEE
:10F1B00080EA0102844612F0030F4FD111F0030FD1
:10F1C00032D14DF8044D11F0040F51F8043B0BD02F
:10F1D000A3F101329A4312F0803F04BF4CF8043B84
:10F1E00051F8043B16D100BF51F8044BA3F1013292
:10F1F0009A4312F0803FA4F101320BD14CF8043B4A
:10F20000A24312F0803F04BF51F8043B4CF8044B7A
:10F21000EAD023460CF8013B13F0FF0F4FEA3323EB
:10F22000F8D15DF8044B704711F0010F06D011F8CA
:10F23000012B0CF8012B002A08BF704711F0020FB8
:10F24000BFD031F8022B12F0FF0F16BF2CF8022BA3
:10F250008CF8002012F47F4FB3D1704711F8012BC6
:10F260000CF8012B002AF9D1704700BF20F00301F0
:10F2700010F00300C0F1000051F8043B00F1040C51
:10F280004FEACC0C6FF000021CBF22FA0CF21343C1
:10F290004FF0010C4CEA0C2C4CEA0C4CA3EB0C028A
:10F2A00022EA030212EACC1204BF51F8043B0430F4
:10F2B000F4D013F0FF0F1FBF013013F47F4F013064
:10F2C00013F47F0F18BF0130704700BF2DE9F04FD6
:10F2D00040F2E814C2F2000485B01F468C4626684E
:10F2E0000B460390029213F8014B32191D4692F817
:10F2F00001B01BF0080BF6D12D2C73D02B2C08BFBE
:10F3000015F8014BD7F1010338BF0023102F14BFAC
:10F310001A4643F0010232B1302C73D01BB1302CAD
:10F3200000F083800A27B946BBF1000F49460CBFA5
:10F330006FF0004A4FF0004ACDF804C0504600F08C
:10F34000B1F950468846494600F07EF8331900224C
:10F35000DDF804C05B78114613F0040F1ED0303C7A
:10F36000A74225DD814294BF0023012353EAD272D4
:10F370002ED10A1A534243EB02034445D4BF002363
:10F3800003F00103002B23D109FB014115F8014BC8
:10F39000012233195B7813F0040FE0D113F003035B
:10F3A00006D0012B14BF57233723E41AA742D9DC18
:10F3B000B2F1FF3F1BD00846BBF1000F10D1029BFA
:10F3C0001BB152B90299C1F800C005B0BDE8F08F79
:10F3D0004FF0FF3215F8014BDBE705F1FF3CF1E799
:10F3E0004842ECE715F8014B4FF0010B8AE703990F
:10F3F000BBF1000F0CBF6FF000404FF00040222324
:10F400000B60DCE72A78A2F17800414241EB000171
:10F41000582A14BF0A4641F00102002A3FF47EAF89
:10F4200010276C78B94602357EE70827B9467BE796
:10F4300030B440F2EC14C2F200040D46134601460B
:10F440002A46206830BC41E74A1E08BF7047C0F01A
:10F450002481884240F21681114200F01781B0FAEF
:10F4600080F3B1FA81F2A2EB0303C3F11F0304A2FC
:10F4700002EB03134FF000029F4600BFAFF3008082
:10F48000B0EBC17F00BF42EB020228BFA0EBC1700E
:10F49000B0EB817F00BF42EB020228BFA0EB81707E
:10F4A000B0EB417F00BF42EB020228BFA0EB4170EE
:10F4B000B0EB017F00BF42EB020228BFA0EB01705E
:10F4C000B0EBC16F00BF42EB020228BFA0EBC160EE
:10F4D000B0EB816F00BF42EB020228BFA0EB81605E
:10F4E000B0EB416F00BF42EB020228BFA0EB4160CE
:10F4F000B0EB016F00BF42EB020228BFA0EB01603E
:10F50000B0EBC15F00BF42EB020228BFA0EBC150CD
:10F51000B0EB815F00BF42EB020228BFA0EB81503D
:10F52000B0EB415F00BF42EB020228BFA0EB4150AD
:10F53000B0EB015F00BF42EB020228BFA0EB01501D
:10F54000B0EBC14F00BF42EB020228BFA0EBC140AD
:10F55000B0EB814F00BF42EB020228BFA0EB81401D
:10F56000B0EB414F00BF42EB020228BFA0EB41408D
:10F57000B0EB014F00BF42EB020228BFA0EB0140FD
:10F58000B0EBC13F00BF42EB020228BFA0EBC1308D
:10F59000B0EB813F00BF42EB020228BFA0EB8130FD
:10F5A000B0EB413F00BF42EB020228BFA0EB41306D
:10F5B000B0EB013F00BF42EB020228BFA0EB0130DD
:10F5C000B0EBC12F00BF42EB020228BFA0EBC1206D
:10F5D000B0EB812F00BF42EB020228BFA0EB8120DD
:10F5E000B0EB412F00BF42EB020228BFA0EB41204D
:10F5F000B0EB012F00BF42EB020228BFA0EB0120BD
:10F60000B0EBC11F00BF42EB020228BFA0EBC1104C
:10F61000B0EB811F00BF42EB020228BFA0EB8110BC
:10F62000B0EB411F00BF42EB020228BFA0EB41102C
:10F63000B0EB011F00BF42EB020228BFA0EB01109C
:10F64000B0EBC10F00BF42EB020228BFA0EBC1002C
:10F65000B0EB810F00BF42EB020228BFA0EB81009C
:10F66000B0EB410F00BF42EB020228BFA0EB41000C
:10F67000B0EB010F00BF42EB020228BFA0EB01007C
:10F68000104670470CBF012000207047B1FA81F28C
:10F69000C2F11F0220FA02F0704708B14FF0FF30AC
:10F6A00000F00EB80029F8D02DE90340FFF7CCFE9A
:10F6B000BDE8064002FB00F3A1EB0301704700BF69
:10F6C000704700BF81F0004102E000BF83F00043BB
:10F6D00030B54FEA41044FEA430594EA050F08BFED
:10F6E00090EA020F1FBF54EA000C55EA020C7FEAB1
:10F6F000645C7FEA655C00F0E2804FEA5454D4EB2E
:10F700005555B8BF6D420CDD2C4480EA020281EAF7
:10F71000030382EA000083EA010180EA020281EA2F
:10F720000303362D88BF30BD11F0004F4FEA013181
:10F730004FF4801C4CEA113102D0404261EB410190
:10F7400013F0004F4FEA03334CEA133302D0524216
:10F7500063EB430394EA050F00F0A780A4F10104D2
:10F76000D5F1200E0DDB02FA0EFC22FA05F280180C
:10F7700041F1000103FA0EF2801843FA05F35941F2
:10F780000EE0A5F120050EF1200E012A03FA0EFC71
:10F7900028BF4CF0020C43FA05F3C01851EBE3719B
:10F7A00001F0004507D54FF0000EDCF1000C7EEBB8
:10F7B00000006EEB0101B1F5801F1BD3B1F5001FF6
:10F7C0000CD349085FEA30004FEA3C0C04F1010415
:10F7D0004FEA445212F5800F80F09A80BCF1004F3E
:10F7E00008BF5FEA500C50F1000041EB045141EAC0
:10F7F000050130BD5FEA4C0C404141EB010111F4C1
:10F80000801FA4F10104E9D191F0000F04BF01466B
:10F810000020B1FA81F308BF2033A3F10B03B3F149
:10F8200020020CDA0C3208DD02F1140CC2F10C02D9
:10F8300001FA0CF021FA02F10CE002F11402D8BF37
:10F84000C2F1200C01FA02F120FA0CFCDCBF41EA03
:10F850000C019040E41AA2BF01EB0451294330BDD2
:10F860006FEA04041F3C1CDA0C340EDC04F11404AF
:10F87000C4F1200220FA04F001FA02F340EA030086
:10F8800021FA04F345EA030130BDC4F10C04C4F1CC
:10F89000200220FA02F001FA04F340EA03002946AC
:10F8A00030BD21FA04F0294630BD94F0000F83F4F6
:10F8B000801306BF81F480110134013D4EE77FEAD9
:10F8C000645C18BF7FEA655C29D094EA050F08BF25
:10F8D00090EA020F05D054EA000C04BF1946104606
:10F8E00030BD91EA030F1EBF0021002030BD5FEA4A
:10F8F000545C05D14000494128BF41F0004130BD72
:10F9000014F580043CBF01F5801130BD01F00045C5
:10F9100045F0FE4141F470014FF0000030BD7FEA38
:10F92000645C1ABF194610467FEA655C1CBF0B4633
:10F93000024650EA013406BF52EA033591EA030F4A
:10F9400041F4002130BD00BF90F0000F04BF002142
:10F95000704730B54FF4806404F132044FF0000575
:10F960004FF0000150E700BF90F0000F04BF0021EE
:10F97000704730B54FF4806404F1320410F0004554
:10F9800048BF40424FF000013EE700BF42004FEA4F
:10F99000E2014FEA31014FEA02701FBF12F07F43CC
:10F9A00093F07F4F81F06051704792F0000F14BFC9
:10F9B00093F07F4F704730B54FF4607401F000450D
:10F9C00021F0004120E700BF50EA010208BF704764
:10F9D00030B54FF000050AE050EA010208BF704759
:10F9E00030B511F0004502D5404261EB41014FF4C2
:10F9F000806404F132045FEA915C3FF4DCAE4FF0C6
:10FA000003025FEADC0C18BF03325FEADC0C18BFAC
:10FA1000033202EBDC02C2F1200300FA03FC20FAFD
:10FA200002F001FA03FE40EA0E0021FA02F114444A
:10FA3000C1E600BF70B54FF0FF0C4CF4E06C1CEA5F
:10FA400011541DBF1CEA135594EA0C0F95EA0C0FD4
:10FA500000F0DEF82C4481EA030621EA4C5123EA47
:10FA60004C5350EA013518BF52EA033541F4801176
:10FA700043F4801338D0A0FB02CE4FF00005E1FB29
:10FA800002E506F00042E0FB03E54FF00006E1FB73
:10FA900003569CF0000F18BF4EF0010EA4F1FF04B6
:10FAA000B6F5007F64F5407404D25FEA4E0E6D41F6
:10FAB00046EB060642EAC62141EA55514FEAC52007
:10FAC00040EA5E504FEACE2EB4F1FD0C88BFBCF583
:10FAD000E06F1ED8BEF1004F08BF5FEA500E50F134
:10FAE000000041EB045170BD06F0004646EA0101FA
:10FAF00040EA020081EA0301B4EB5C04C2BFD4EB2C
:10FB00000C0541EA045170BD41F480114FF0000E24
:10FB1000013C00F3AB8014F1360FDEBF002001F092
:10FB2000004170BDC4F10004203C35DA0C341BDC0C
:10FB300004F11404C4F1200500FA05F320FA04F0DE
:10FB400001FA05F240EA020001F0004221F0004112
:10FB500010EBD37021FA04F642EB06015EEA430E85
:10FB600008BF20EAD37070BDC4F10C04C4F12005B5
:10FB700000FA04F320FA05F001FA04F240EA020068
:10FB800001F0004110EBD37041F100015EEA430E39
:10FB900008BF20EAD37070BDC4F1200500FA05F259
:10FBA0004EEA020E20FA04F301FA05F243EA0203D8
:10FBB00021FA04F001F0004121FA04F220EA0200E7
:10FBC00000EBD3705EEA430E08BF20EAD37070BD2D
:10FBD00094F0000F0FD101F00046400041EB01010D
:10FBE00011F4801F08BF013CF7D041EA060195F0EF
:10FBF000000F18BF704703F00046520043EB0303A9
:10FC000013F4801F08BF013DF7D043EA0603704795
:10FC100094EA0C0F0CEA135518BF95EA0C0F0CD0A0
:10FC200050EA410618BF52EA4306D1D181EA0301E6
:10FC300001F000414FF0000070BD50EA410606BFE0
:10FC40001046194652EA430619D094EA0C0F02D125
:10FC500050EA013613D195EA0C0F05D152EA03366A
:10FC60001CBF104619460AD181EA030101F0004188
:10FC700041F0FE4141F470014FF0000070BD41F0D1
:10FC8000FE4141F4780170BD70B54FF0FF0C4CF4AB
:10FC9000E06C1CEA11541DBF1CEA135594EA0C0FCA
:10FCA00095EA0C0F00F0A7F8A4EB050481EA030E17
:10FCB00052EA03354FEA013100F088804FEA0333FE
:10FCC0004FF0805545EA131343EA12634FEA0222CC
:10FCD00045EA111545EA10654FEA00260EF000418D
:10FCE0009D4208BF964244F1FD0404F5407402D2DF
:10FCF0005B084FEA3202B61A65EB03055B084FEA70
:10FD000032024FF480104FF4002CB6EB020E75EB6C
:10FD1000030E22BFB61A754640EA0C005B084FEA94
:10FD20003202B6EB020E75EB030E22BFB61A754611
:10FD300040EA5C005B084FEA3202B6EB020E75EB5C
:10FD4000030E22BFB61A754640EA9C005B084FEAD4
:10FD50003202B6EB020E75EB030E22BFB61A7546E1
:10FD600040EADC0055EA060E18D04FEA051545EAD0
:10FD700016754FEA06164FEAC30343EA52734FEA79
:10FD8000C2025FEA1C1CC0D111F4801F0BD141EAF2
:10FD900000014FF000004FF0004CB6E711F4801F57
:10FDA00004BF01430020B4F1FD0C88BFBCF5E06F37
:10FDB0003FF6AFAEB5EB030C04BFB6EB020C5FEA47
:10FDC000500C50F1000041EB045170BD0EF0004E9C
:10FDD0004EEA113114EB5C04C2BFD4EB0C0541EACE
:10FDE000045170BD41F480114FF0000E013C90E6CB
:10FDF00045EA060E8DE60CEA135594EA0C0F08BF8F
:10FE000095EA0C0F3FF43BAF94EA0C0F0AD150EA8D
:10FE100001347FF434AF95EA0C0F7FF425AF104620
:10FE200019462CE795EA0C0F06D152EA03353FF448
:10FE3000FDAE1046194622E750EA410618BF52EAC5
:10FE400043067FF4C5AE50EA41047FF40DAF52EA99
:10FE500043057FF4EBAE12E74FF0FF3C06E000BF36
:10FE60004FF0010C02E000BF4FF0010C4DF804CD43
:10FE70004FEA410C7FEA6C5C4FEA430C18BF7FEA03
:10FE80006C5C1BD001B050EA410C0CBF52EA430C31
:10FE900091EA030F02BF90EA020F0020704710F1B1
:10FEA000000F91EA030F58BF994208BF90422CBF40
:10FEB000D8176FEAE37040F0010070474FEA410C39
:10FEC0007FEA6C5C02D150EA013C07D14FEA430C57
:10FED0007FEA6C5CD6D152EA033CD3D05DF8040BC8
:10FEE000704700BF8446104662468C4619466346FA
:10FEF00000E000BF01B5FFF7B7FF002848BF10F1D1
:10FF0000000F01BD4DF808EDFFF7F4FF0CBF012015
:10FF100000205DF808FB00BF4DF808EDFFF7EAFF91
:10FF200034BF012000205DF808FB00BF4DF808ED4C
:10FF3000FFF7E0FF94BF012000205DF808FB00BF41
:10FF40004DF808EDFFF7CEFF94BF012000205DF8CB
:10FF500008FB00BF4DF808EDFFF7C4FF34BF0120D8
:10FF600000205DF808FB00BF4FEA410212F50012C5
:10FF700015D211D56FF47873B3EB625212D94FEAF0
:10FF8000C12343F0004343EA505311F0004F23FADA
:10FF900002F018BF404270474FF00000704750EA2F
:10FFA000013005D111F0004008BF6FF000407047EC
:10FFB0004FF00000704700BF4A0011D212F5001246
:10FFC00011D20DD56FF47873B3EB62520ED44FEAB1
:10FFD000C12343F0004343EA505323FA02F0704731
:10FFE0004FF00000704750EA013002D14FF0FF306F
:10FFF00070474FF0000070474FEA4102B2F1E04312
:020000021000EC
:1000000024BFB3F5001CDCF1FE5C0DD901F0004CFF
:100010004FEAC0024CEA5070B2F1004F40EB83004F
:1000200008BF20F00100704711F0804F21D113F17B
:100030003872BCBF01F00040704741F480114FEAB4
:100040005252C2F11802C2F1200C10FA0CF320FA3D
:1000500002F018BF40F001004FEAC1234FEAD3235A
:1000600003FA0CFC40EA0C0023FA02F34FEA4303C4
:10007000CCE77FEA625307D150EA01331EBF4FF04D
:10008000FE4040F44000704701F0004040F0FE4068
:1000900040F40000704700BF80F0004002E000BF65
:1000A00081F0004142001FBF5FEA410392EA030F63
:1000B0007FEA226C7FEA236C6AD04FEA1262D2EBAD
:1000C0001363C1BFD218414048404140B8BF5B42B2
:1000D000192B88BF704710F0004F40F4000020F04B
:1000E0007F4018BF404211F0004F41F4000121F061
:1000F0007F4118BF494292EA030F3FD0A2F10102AB
:1001000041FA03FC10EB0C00C3F1200301FA03F1E8
:1001100000F0004302D5494260EB4000B0F5000F0B
:1001200013D3B0F1807F06D340084FEA310102F1CA
:100130000102FE2A51D2B1F1004F40EBC25008BF7C
:1001400020F0010040EA03007047490040EB000046
:1001500010F4000FA2F10102EDD1B0FA80FCACF175
:10016000080CB2EB0C0200FA0CF0AABF00EBC25074
:1001700052421843BCBFD0401843704792F0000F62
:1001800081F4000106BF80F400000132013BB5E7B5
:100190004FEA41037FEA226C18BF7FEA236C21D02B
:1001A00092EA030F04D092F0000F08BF0846704790
:1001B00090EA010F1CBF0020704712F07F4F04D15E
:1001C000400028BF40F00040704712F100723CBF71
:1001D00000F50000704700F0004343F0FE4040F49B
:1001E000000070477FEA226216BF08467FEA236359
:1001F0000146420206BF5FEA412390EA010F40F444
:10020000800070474FF0000304E000BF10F000438F
:1002100048BF40425FEA000C08BF704743F0964376
:1002200001464FF000001CE050EA010208BF704791
:100230004FF000030AE000BF50EA010208BF704718
:1002400011F0004302D5404261EB41015FEA010C2D
:1002500002BF84460146002043F0B64308BFA3F125
:100260008053A3F50003BCFA8CF2083AA3EBC25307
:1002700010DB01FA02FC634400FA02FCC2F1200226
:10028000BCF1004F20FA02F243EB020008BF20F05D
:100290000100704702F1200201FA02FCC2F12002C3
:1002A00050EA4C0021FA02F243EB020008BF20EAB8
:1002B000DC7070474FF0FF0C1CEAD0521EBF1CEAE6
:1002C000D15392EA0C0F93EA0C0F6FD01A4480EAD4
:1002D000010C400218BF5FEA41211ED04FF00063BD
:1002E00043EA501043EA5111A0FB01310CF00040E9
:1002F000B1F5000F3EBF490041EAD3715B0040EA0F
:10030000010062F17F02FD2A1DD8B3F1004F40EBDE
:10031000C25008BF20F00100704790F0000F0CF0B1
:10032000004C08BF49024CEA502040EA51207F3A75
:10033000C2BFD2F1FF0340EAC250704740F4000050
:100340004FF00003013A5DDC12F1190FDCBF00F041
:1003500000407047C2F10002410021FA02F1C2F1EF
:10036000200200FA02FC5FEA310040F1000053EA8B
:100370004C0308BF20EADC70704792F0000F00F0D9
:10038000004C02BF400010F4000F013AF9D040EADF
:100390000C0093F0000F01F0004C02BF490011F473
:1003A000000F013BF9D041EA0C018FE70CEAD15371
:1003B00092EA0C0F18BF93EA0C0F0AD030F0004CF1
:1003C00018BF31F0004CD8D180EA010000F00040A5
:1003D000704790F0000F17BF90F0004F084691F063
:1003E000000F91F0004F14D092EA0C0F01D142029D
:1003F0000FD193EA0C0F03D14B0218BF084608D166
:1004000080EA010000F0004040F0FE4040F40000AF
:10041000704740F0FE4040F4400070474FF0FF0C42
:100420001CEAD0521EBF1CEAD15392EA0C0F93EA89
:100430000C0F69D0A2EB030280EA010C49024FEADB
:10044000402037D04FF0805343EA111143EA101394
:100450000CF000408B4238BF5B0042F17D024FF44C
:10046000000C8B4224BF5B1A40EA0C00B3EB510F27
:1004700024BFA3EB510340EA5C00B3EB910F24BF10
:10048000A3EB910340EA9C00B3EBD10F24BFA3EB95
:10049000D10340EADC001B0118BF5FEA1C1CE0D15D
:1004A000FD2A3FF650AF8B4240EBC25008BF20F010
:1004B000010070470CF0004C4CEA50207F32C2BF64
:1004C000D2F1FF0340EAC250704740F400004FF001
:1004D0000003013A37E792F0000F00F0004C02BF32
:1004E000400010F4000F013AF9D040EA0C0093F0FC
:1004F000000F01F0004C02BF490011F4000F013B56
:10050000F9D041EA0C0195E70CEAD15392EA0C0FBD
:1005100008D142027FF47DAF93EA0C0F7FF470AFF5
:10052000084676E793EA0C0F04D14B023FF44CAF38
:1005300008466EE730F0004C18BF31F0004CCAD1CD
:1005400030F000427FF45CAF31F000437FF43CAF09
:100550005FE700BF4FF0FF3C06E000BF4FF0010C2B
:1005600002E000BF4FF0010C4DF804CD4FEA40020D
:100570004FEA41037FEA226C18BF7FEA236C11D057
:1005800001B052EA530C18BF90EA010F58BFB2EB0A
:10059000030088BFC81738BF6FEAE17018BF40F08A
:1005A000010070477FEA226C02D15FEA402C05D13E
:1005B0007FEA236CE4D15FEA412CE1D05DF8040BC3
:1005C000704700BF844608466146FFE70FB5FFF756
:1005D000C9FF002848BF10F1000F0FBD4DF808ED0E
:1005E000FFF7F4FF0CBF012000205DF808FB00BFFF
:1005F0004DF808EDFFF7EAFF34BF012000205DF859
:1006000008FB00BF4DF808EDFFF7E0FF94BF0120A5
:1006100000205DF808FB00BF4DF808EDFFF7D2FFA2
:1006200094BF012000205DF808FB00BF4DF808EDE5
:10063000FFF7C8FF34BF012000205DF808FB00BFB2
:100640004FEA4002B2F1FE4F0FD34FF09E03B3EBDF
:1006500012620DD94FEA002343F0004310F0004F1F
:1006600023FA02F018BF404270474FF00000704775
:1006700012F1610F01D1420205D110F0004008BF14
:100680006FF0004070474FF00000704774656C6574
:100690006D65747269652000696E70757420006FF5
:1006A00075747075742000737973696E666F2000BD
:1006B0006D6F64656C2000417263757300517565E0
:1006C00072727564657200486F6568656E727564F4
:1006D00065720044726F7373656C0053656974656D
:1006E0006E727564657200466C6170730042757459
:1006F000746572666C79004153573100415357322B
:1007000000446966662D4D6F64650044535732009E
:100710004453573300445357340051756572727512
:100720006465722D52005175657272756465722D23
:100730004C00466C61702D5200466C61702D4C006F
:1007400072636F732D6D6F64656C2D302E392E378B
:100750000072434F530053414D3700556E6E616D2B
:10076000656400535344313332390000E809010015
:1007700011180100FA0A010039130100D90D010016
:10078000EE0E0100E40D0100140F0100EC0D01005C
:10079000F80D0100790A0100740A0100820A0100C3
:1007A000CF0A0100E8090100990E0100E8090100E3
:1007B000190D0100E90C0100240D01002C0D0100B0
:1007C000390D0100480D0100550D0100640D0100B7
:1007D000710D0100800D01008D0D01009C0D0100C7
:1007E000E8090100280E0100E90C01000A0D0100D2
:1007F000E809010094120100A3120100B3120100E4
:10080000C2120100D1120100E1120100EE1201003A
:10081000FC120100E80901007A180100A318010088
:10082000CA180100EA180100E80901007A1801005D
:100830001B1A0100A3180100401A0100E809010079
:10084000EE0E0100280E0100D90C0100E90C010098
:10085000F20C01002F0A0100E80901000B18010049
:10086000161801002E1801003C1801005318010051
:100870005C18010069180100E8090100AF110100CE
:10088000E80F0100EF0F0100E8090100860E0100EA
:10089000910E01009D0E0100AA0E0100B40E010090
:1008A000C10E0100CD0E0100741601008116010079
:1008B000D90E0100E60E0100F30E0100E809010067
:1008C000300E0100390E0100400E0100460E0100FD
:1008D000510E01004C0E0100260A0100570E0100C6
:1008E0005D0E0100E80901007A180100A31801005B
:1008F000091A0100E8090100180E0100240E010088
:10090000EE0E0100300E0100E8090100F8130100AD
:100910000614010011140100391401001F14010014
:10092000CF0A01002E140100481401005D140100DB
:100930006F14010081140100010100000002040491
:1009400004050D0D0D13131313000000E809010039
:1009500026130100321301003E1301004A13010067
:10096000561301006713010073130100E809010029
:10097000111801007B1001007310010066100100C6
:100980000D140100E71B0100E80901005C120100E1
:100990007112010082120100E8090100280E010015
:1009A000E90C0100F20C01002F0A0100E809010026
:1009B0007A180100A3180100CA180100EA18010002
:1009C000E809010005150100121501001B150100C1
:1009D00035150100D80F0100241501003E15010056
:1009E0000A0D424D4F443A006261636B00416464FA
:1009F0000045646974005B454E445D004E6F726D46
:100A0000616C005669727475616C004C696E656149
:100A100072004E6F004F766572616C6C00526561BA
:100A20006C00596573004D6964646C6500557044D1
:100A30006F776E004D656D6F7279004175746F0050
:100A40004669786564200046697865642030250031
:100A500020284F6E290020284F66662900466978B5
:100A60006564204F6E004669786564204F666600B5
:100A70002C0028004578706F004475616C726174B9
:100A800065004D6F74696F6E00417476004C696D3E
:100A90006974657200254D49582D3E002545585012
:100AA0002D3E002544522D3E00254D542D3E00255F
:100AB0004154562D3E004C4D2D3E00254C494D2DA8
:100AC0003E00592000636F70792066726F6D204D73
:100AD000697865720046697865642D4F66662028DE
:100AE0003025290046697865642D4F6E2028313005
:100AF0003025290046697865642D56616C7565005E
:100B0000696E707574004E4F4E45006F7574707548
:100B10007400556E7573656400496E7075742D4F61
:100B200076657276696577004F75747075742D4FB0
:100B300076657276696577005175657200486F68F1
:100B400065005365697465004B6C617070656E007B
:100B50005374616E6467617300334400456E676966
:100B60006E6500536D6F6B6500517565722D4C009D
:100B7000486F68652D4C00517565722D5200486FA5
:100B800068652D5200526F6C6C004E69636B0050AB
:100B90006974636800486F6C64004779726F2D5305
:100BA000656E736500526F6C6C2D5472696D004EEA
:100BB00069636B2D5472696D0050697463682D54BC
:100BC00072696D005275646465722D5472696D00AE
:100BD00049646C652D53706565642F4D696E0049DD
:100BE000646C652D53706565642F4D617800486FA6
:100BF0006C642D53706565640050697463682D3EA4
:100C000052756464657200526F6C6C2D4C00526FAB
:100C10006C6C2D52004C656E6B756E6700556E6284
:100C2000656C656774004761730042756773747221
:100C300061686C005475726E4D6F64650052756426
:100C40006572004D6F746F7231004D6F746F723248
:100C5000004D6F746F7233004368616E6E656C2D6A
:100C600000536572766F2D00476574726965626521
:100C700000506C656173650063656E746572005346
:100C80007469636B73006D6F76650061726F756E6A
:100C900064005669727475616C2D496E7075747359
:100CA00000526576657273652D496E7075747300B8
:100CB000526576657273652D4F7574707574730027
:100CC0005461726765740054657374006C6F676972
:100CD00063636F6E74726F6C00536F6674737461CC
:100CE00072742D5370656564005263737769746321
:100CF00068005570006D6F74696F6E0047726164B3
:100D000069656E74006578706F004C696D69740078
:100D10006475616C72617465004368616E6E656CC8
:100D20002D496E0050657263656E74004368616E94
:100D30006E656C2D4F7574310050657263656E740D
:100D40002D56616C756531004368616E6E656C2D62
:100D50004F7574320050657263656E742D56616C08
:100D6000756532004368616E6E656C2D4F75743326
:100D70000050657263656E742D56616C7565330045
:100D80004368616E6E656C2D4F75743400506572EA
:100D900063656E742D56616C7565340043757276AB
:100DA00065002D3E50504D31002D3E50504D3200CB
:100DB0002D3E6D456E6331002D3E6D456E633200F4
:100DC0006F757400464958004F4646004F4E002547
:100DD0002D3E003A3130302500496E7075742D4D2E
:100DE0006F6465004F7074696F6E310043656E7497
:100DF00065722D4D6F64650043656E7465720049C0
:100E00006E70757400617476006C696D69746572DA
:100E1000004F75747075740050706D2D456E636F62
:100E20006465720050706D2D4368616E6E656C0074
:100E30004368616E6E656C7300496E76657274000E
:100E4000506F776572004672616D652D53796E63E0
:100E50000053686966740052616E6765004D656E87
:100E6000636F6465720070706D656E636F64657248
:100E70000052656400477265656E00426C756500DE
:100E8000416C70686100426174742D5363616C65DC
:100E900000426174742D4F6666736574004261741C
:100EA000742D5761726E696E67004261636B6C6985
:100EB00067687400456E7472792D48656967687457
:100EC00000486561642D48656967687400466F6F06
:100ED000742D48656967687400496E7075742D508B
:100EE0006F7075707300456E636F6465722D547911
:100EF0007065004175746F6C6F6164007374696331
:100F00006B00536574005472696D6D3100547269E1
:100F10006D6D312D52657665727365005472696D21
:100F20006D32005472696D6D322D52657665727343
:100F300065005472696D6D33005472696D6D332DA7
:100F400052657665727365005472696D6D34005434
:100F500072696D6D342D52657665727365005472D9
:100F6000786964004D6F64656C74797065005070C9
:100F70006D656E636F646572005472696D6D76693C
:100F80006577004C6F676E756D004C6F67706F739F
:100F900000496E74657276616C00496E7075742DCF
:100FA0004D6178004F75747075742D4D61780054E3
:100FB000656C656D65747269652D4D617800416C75
:100FC00061726D3100416C61726D32005469636B06
:100FD0000045787065727400446973706C617900C3
:100FE000537973696E666F0057697A617264005352
:100FF000797374656D002F005458200052582000FA
:101000004D61696E766965770054583A20005258F0
:101010003A2000566F6C74004C6F672E204F6E00A4
:101020004C6F672E204F6666004D61696E6D656E70
:1010300075005900582D416368736500592D41634F
:1010400068736500332D506F696E740048616C667B
:1010500000436F7079004D6178696D616C004D6976
:101060006E696D616C004D6178696D616C2D5765BD
:101070007274004D696E696D616C2D5765727400F4
:101080004669782D57657274005570706572004C12
:101090006F776572004F6265726572204772656E88
:1010A0007A7765727400556E746572657220477246
:1010B000656E7A776572740046756E6B74696F6ED3
:1010C00020756D6B656872656E004D6F64652D31BE
:1010D000004D6F64652D32004D6F64652D33004DFA
:1010E0006F64652D340046757461626100477261FA
:1010F00075706E65722F4A52004D756C7469706C14
:1011000065780033442D506C616E6500322D466C5D
:10111000617020476C6964657200342D466C6170A3
:1011200020476C6964657200506C616E652D3100FA
:10113000506C616E652D32004163726F2D31004439
:10114000656C74612D310048656C692D3132300059
:1011500048656C692D3138300048656C692D39302F
:101160000043617200426F617400426F61742D32FE
:101170004D6F742E00426F61742D334D6F742E00CD
:1011800046756E6374696F6E004561737920313AFC
:1011900031004561737920313A3400546573742D00
:1011A0004D6F6465004261636B004C6F6164204D5C
:1011B0006F64656C0053617665204D6F64656C00EB
:1011C00052656D6F7665204D6F64656C00506F776A
:1011D0006572204F666600537469636B6D6F64655A
:1011E00000536572766F6D6F64650052756E0073A3
:1011F0007469636B6D6F646500736572766F6D6F94
:101200006465006D6F64656C747970650072756EED
:10121000004F75747075742031004F75747075745B
:101220002032004F75747075742033004F757470E0
:1012300075742034005570446F776E2D436F756E52
:10124000746572004D656D6F72792D5377697463A3
:1012500068004175746F6D6174696B004D6F6465F2
:101260006C6C2D45696E7374656C6C756E67656E1C
:10127000004D6F64656C6C2065727374656C6C6591
:101280006E0053797374656D2053657475702F49C2
:101290006E666F00696E7075745F6F7665727669E1
:1012A0006577006F75747075745F6F7665727669B7
:1012B0006577007669727475616C5F696E707574BC
:1012C0007300726576657273655F696E70757473AD
:1012D00000726576657273655F6F7574707574738F
:1012E000004B616C696272696572756E6700446972
:1012F00073706C61792D53657475700053797374D4
:10130000656D2D496E666F73007361766500646567
:101310006C657465004C6F616400536176650044D0
:10132000656C657465004D6F64656C6C2D4E616D08
:1013300065004D6F64656C6C2D49636F6E00476589
:101340006265722D536574757000536572766F2DEA
:1013500053657475700054656C656D65747269656C
:101360002D5365747570004578706572742D4D65E8
:101370006E750054696D65722D4D656E75007265F0
:1013800073657474696D657231005469636B7300C1
:101390004D6F64757300526573657474696D657221
:1013A00031004C6F6767696E672D536368616C74B9
:1013B0006572006C6F676E756D006C6F67706F7330
:1013C00000496E74657276616C6C00416E7A61687A
:1013D0006C20476562657200416E7A61686C2053CB
:1013E0006572766F7300416E7A61686C2054656C2B
:1013F000656D657472696500436F6E6E65637469CF
:101400006F6E2D4944004D6F64656C6C2D5479707E
:10141000004578706F2D46756E6B74696F6E004D68
:101420006F74696F6E2D436F6E74726F6C004569D7
:101430006E73656974696765205765677265647561
:101440007A696572756E67004C696D697465722F93
:1014500057656762656772656E7A65720050504DB8
:101460002D456E636F646572205365747570004D11
:10147000756C746970726F702D456E636F64657200
:10148000005472696D6D65722D416E7A656967658C
:10149000005472696D6D657231005472696D6D65CD
:1014A00072312D52657665727365005472696D6D87
:1014B000657232005472696D6D6572322D526576B7
:1014C00065727365005472696D6D65723300547294
:1014D000696D6D6572332D52657665727365005462
:1014E00072696D6D657234005472696D6D65723428
:1014F0002D526576657273650043656E7465722D55
:10150000576572740053797374656D2D54696D65F8
:101510007200536F66747761726500486172647718
:1015200061726500416B7475656C6C6572204D6FFE
:1015300064656C6C2D537065696368657200416BFE
:101540007475656C6C6573205665727A656963683D
:101550006E6973730053797374696D6572005374A7
:101560006F72616765004D6F64656C2D46696C65CF
:101570000053746F726167652D5061746800416B30
:101580006B752D43616C6962726174696F6E0041A5
:101590006B6B752D4F666673657420312F31305635
:1015A00000416B6B752D5761726E756E6720312F20
:1015B0003130560048696E7465726772756E642DBD
:1015C00042656C6575636874756E670048C3B6687C
:1015D000652065696E6573204D656EC3BC65696E77
:1015E00074726167730048C3B668652064657220D1
:1015F0004B6F70666C65697374650048C3B6686547
:1016000020646572204675C39F6C656973746500BC
:1016100046656E737465722D427265697465004625
:10162000656E737465722D486F65686500446973F3
:10163000706C617920496E7075742D4368616E67B6
:1016400065730054797020646573204D656EC3BC6A
:101650002D456E636F64657273004D6F64656C6CCD
:1016600020286E6F6E652F6C6173742F73656C65C7
:101670006374290053637265656E2D5769647468DD
:101680000053637265656E2D486569676874005222
:101690006F74004772266F756D6C3B6E00426C6113
:1016A00075005472616E73706172656E7A00C39CCE
:1016B00062657274726167756E67732D5765670036
:1016C000C39C62657274726167756E67732D4B613E
:1016D0006E616C0054797020646573204D756C7474
:1016E0006970726F702D50726F746F6B6F6C6C736A
:1016F00000416E7A61686C20646572204D756C746F
:101700006970726F702D4B616EC3A46C6500416E81
:101710007A61686C20646572207A752073656E64E6
:10172000656E64656E204B616EC3A46C6500496E86
:1017300076657274696572656E20646573205050B9
:101740004D2D496D707573657300416E2F41757332
:101750002D536368616C74656E2064657320484620
:101760002D4D6F64756C73004672616D652D5379F4
:101770006E632D466C61672028696E7465726E29F0
:10178000004C2661756D6C3B6E6765206465732047
:1017900053686966742D50756C736573004C2661CF
:1017A000756D6C3B6E6765206465732053796E635D
:1017B0002D50756C736573004C2661756D6C3B6EB6
:1017C0006765206465732043656E7465722D50757E
:1017D0006C736573004D6178696D616C6520446957
:1017E00066666572656E7A207A756D2043656E74E3
:1017F00065722D50756C7365004C494E4B205263D9
:101800005F4D656E636F6465723B004B616E616C2A
:101810002D4E616D6500416B7475656C6C65722D44
:1018200041757367616E67732D57657274005365F8
:1018300072766F2D52657665727365004D6F6475B3
:101840007320284D6964646C652F4F766572616CF6
:101850006C29005472696D6D756E67004C494E4B72
:101860002052635F4174763B004C494E4B205263DB
:101870005F4C696D697465723B004B616E616C20F1
:101880006175662064656D206469657365204675C1
:101890006E6B74696F6E207769726B656E20736F03
:1018A0006C6C004765626572207A756D20416E2F01
:1018B00041757320536368616C74656E2064657252
:1018C0002046756E6B74696F6E004D6978696D6145
:1018D0006C2D4175737363686C61672028312E200D
:1018E0005269636874756E6729004D6978696D6126
:1018F0006C2D4175737363686C61672028322E20EC
:101900005269636874756E67290045696E67616E18
:10191000732D4B616E616C20646573204D69786531
:10192000722773004765626572207A756D20416E7B
:101930002F41757320536368616C74656E20646514
:1019400073204D6978657273004D697865722D4119
:101950006E7465696C0041757367616E67732D4BBA
:10196000616E616C3120646573204D697865722702
:1019700073005765727420646573204175736761E5
:101980006E67732D416E7465696C732028302D313C
:10199000303025290041757367616E67732D4B6187
:1019A0006E616C3220646573204D697865722773AF
:1019B0000041757367616E67732D4B616E616C33A7
:1019C00020646573204D69786572277300417573D3
:1019D00067616E67732D4B616E616C342064657353
:1019E000204D69786572277300382D50756E6B74C1
:1019F0002D4B7572766520283178792D3878793BB2
:101A000020302D3130302529004D6178696D616CB1
:101A10002D4175737363686C61670054797020643D
:101A20006572204578706F2D46756E6B74696F6EA8
:101A30002028686F6368323B20686F636833290031
:101A40005374656967756E670041727420646572CE
:101A5000204D6F74696F6E2D46756E6B74696F6E75
:101A6000202853706565642D494E3B205370656591
:101A7000642D4F75743B204D6F74696F6E2D494E08
:101A80003B204D6F74696F6E2D4F75742900536F35
:101A9000667473746172742D46756E6B74696F6EC3
:101AA0002028302D3130302529004D6978696D614D
:101AB0006C2D476573636877696E6469676B6569E8
:101AC000742028312E205269636874756E6729006E
:101AD0004D6978696D616C2D476573636877696ED0
:101AE0006469676B6569742028322E2052696368C7
:101AF00074756E6729005A69656C2D476562657259
:101B000000546573742D476562657200566572678F
:101B10006C65696368732D576572740054657374DE
:101B20002D46756E6B74696F6E0047656265722D28
:101B30004E616D650047656265722D576572740070
:101B40004D6F64757320285669727475656C6C2FBF
:101B5000416B746976290054797020284C696E6550
:101B600061722F5377697463682F5570446F776E75
:101B70002F4D656D6F727929004F7074696F6E31EA
:101B800020286A65206E61636820547970290052AC
:101B900065766572736520284E6F726D616C2F5289
:101BA00065766572736529004C494E4B2052635F20
:101BB0004475616C726174653B004C494E4B205218
:101BC000635F4578706F3B004C494E4B2052635F1A
:101BD0004D6F74696F6E3B004C494E4B2052635FF2
:101BE0004D697865723B005363616C652D46616B8E
:101BF000746F7200E809010011180100FA0A01006F
:101C0000140F0100EC0D0100F80D0100890A01001C
